 ConEmuBg

 Timestamp is 5b32b0f8 (Wed Jun 27 00:32:40 2018)

 Preferred load address is 10000000

 Start         Length     Name                   Class
 0001:00000000 000184cdH .text$mn                CODE
 0001:000184cd 000000f2H .text$x                 CODE
 0002:00000000 0000022cH .idata$5                DATA
 0002:0000022c 00000004H .00cfg                  DATA
 0002:00000230 00000004H .CRT$XCA                DATA
 0002:00000234 00000004H .CRT$XCZ                DATA
 0002:00000238 00000004H .CRT$XIA                DATA
 0002:0000023c 00000010H .CRT$XIC                DATA
 0002:0000024c 00000004H .CRT$XIZ                DATA
 0002:00000250 00000004H .CRT$XLA                DATA
 0002:00000254 00000004H .CRT$XLZ                DATA
 0002:00000258 00000004H .CRT$XPA                DATA
 0002:0000025c 00000008H .CRT$XPX                DATA
 0002:00000264 00000004H .CRT$XPXA               DATA
 0002:00000268 00000004H .CRT$XPZ                DATA
 0002:0000026c 00000004H .CRT$XTA                DATA
 0002:00000270 00000010H .CRT$XTZ                DATA
 0002:00000274 00000000H .gfids$x                DATA
 0002:00000274 00000000H .gfids$y                DATA
 0002:00000280 00006958H .rdata                  DATA
 0002:00006bd8 00000018H .rdata$T                DATA
 0002:00006bf0 000001e0H .rdata$r                DATA
 0002:00006dd0 0000002cH .rdata$sxdata           DATA
 0002:00006dfc 00000380H .rdata$zzzdbg           DATA
 0002:0000717c 00000004H .rtc$IAA                DATA
 0002:00007180 00000004H .rtc$IZZ                DATA
 0002:00007184 00000004H .rtc$TAA                DATA
 0002:00007188 00000004H .rtc$TZZ                DATA
 0002:0000718c 00000004H .tls                    DATA
 0002:00007190 00000004H .tls$                   DATA
 0002:00007194 00000004H .tls$ZZZ                DATA
 0002:00007198 000005e8H .xdata$x                DATA
 0002:00007780 0000018cH .edata                  DATA
 0002:0000790c 00000078H .idata$2                DATA
 0002:00007984 00000014H .idata$3                DATA
 0002:00007998 0000022cH .idata$4                DATA
 0002:00007bc4 000009aeH .idata$6                DATA
 0003:00000000 00001e50H .data                   DATA
 0003:00001e50 000000c0H .data$r                 DATA
 0003:00001f10 00008bf8H .bss                    DATA
 0004:00000000 000000a0H .rsrc$01                DATA
 0004:000000a0 00000498H .rsrc$02                DATA

  Address         Publics by Value              Rva+Base       Lib:Object

 0000:00000000       __except_list              00000000     <absolute>
 0000:00000000       ___guard_fids_count        00000000     <absolute>
 0000:00000000       ___enclave_config          00000000     <absolute>
 0000:00000000       ___guard_longjmp_count     00000000     <absolute>
 0000:00000000       ___hybrid_code_map_count   00000000     <absolute>
 0000:00000000       ___guard_longjmp_table     00000000     <absolute>
 0000:00000000       ___guard_iat_table         00000000     <absolute>
 0000:00000000       ___hybrid_code_map         00000000     <absolute>
 0000:00000000       ___guard_iat_count         00000000     <absolute>
 0000:00000000       ___hybrid_auxiliary_iat    00000000     <absolute>
 0000:00000000       ___guard_fids_table        00000000     <absolute>
 0000:00000000       ___dynamic_value_reloc_table 00000000     <absolute>
 0000:0000000b       ___safe_se_handler_count   0000000b     <absolute>
 0000:0000002c       __tls_array                0000002c     <absolute>
 0000:00000100       ___guard_flags             00000100     <absolute>
 0000:00000000       ___ImageBase               10000000     <linker-defined>
 0001:00000000       _ConfigureW@4              10001000 f   ConEmuBg.obj
 0001:00000046       _ExitFARW@0                10001046 f   ConEmuBg.obj
 0001:0000006b       ?ExitFARW3@@YGXPAX@Z       1000106b f   ConEmuBg.obj
 0001:00000099       ?ConfigureW3@@YGHPAX@Z     10001099 f   ConEmuBg.obj
 0001:000000da       ??$SafeDelete@UMSectionSimple@@@@YAXAAPAUMSectionSimple@@@Z 100010da f i ConEmuBg.obj
 0001:0000010b       ??$swprintf_c@$0IA@@@YAHAAY0IA@_WPB_WZZ 1000110b f i ConEmuBg.obj
 0001:00000124       ??1MStream@@UAE@XZ         10001124 f i ConEmuBg.obj
 0001:0000015b       ??_EMStream@@UAEPAXI@Z     1000115b f i ConEmuBg.obj
 0001:0000015b       ??_GMStream@@UAEPAXI@Z     1000115b f i ConEmuBg.obj
 0001:0000017d       ?AddRef@MStream@@UAGKXZ    1000117d f i ConEmuBg.obj
 0001:000002c8       ?CheckXmlFile@@YA_N_N@Z    100012c8 f   ConEmuBg.obj
 0001:00000727       ?Clone@MStream@@UAGJPAPAUIStream@@@Z 10001727 f i ConEmuBg.obj
 0001:0000072f       ?Close@CachedImage@@QAEXXZ 1000172f f i ConEmuBg.obj
 0001:000007a3       ?Close@GDIPlusDecoder@@QAEXXZ 100017a3 f i ConEmuBg.obj
 0001:00000854       ?Commit@MStream@@UAGJK@Z   10001854 f i ConEmuBg.obj
 0001:00000866       ?CompareNames@@YA_NPB_WPA_W@Z 10001866 f   ConEmuBg.obj
 0001:00000979       ?LockRegion@MStream@@UAGJT_ULARGE_INTEGER@@0K@Z 10001979 f i ConEmuBg.obj
 0001:00000979       ?UnlockRegion@MStream@@UAGJT_ULARGE_INTEGER@@0K@Z 10001979 f i ConEmuBg.obj
 0001:00000979       ?CopyTo@MStream@@UAGJPAUIStream@@T_ULARGE_INTEGER@@PAT3@2@Z 10001979 f i ConEmuBg.obj
 0001:00000981       ?ExitPlugin@@YAXXZ         10001981 f   ConEmuBg.obj
 0001:000009c7       ?FMatch@@YA_NPB_WPA_W@Z    100019c7 f   ConEmuBg.obj
 0001:00000ad2       ?FillPanelParams@@YAHPAUPaintBackgroundArg@@PAUBkPanelInfo@@PAUDrawInfo@@@Z 10001ad2 f   ConEmuBg.obj
 0001:00001881       ?FormatSize@@YAXT_ULARGE_INTEGER@@PA_W@Z 10002881 f   ConEmuBg.obj
 0001:00001976       ?FreeThreadProc@GDIPlusDecoder@@SGKPAX@Z 10002976 f i ConEmuBg.obj
 0001:00001995       ?GdipDone@@YAXXZ           10002995 f   ConEmuBg.obj
 0001:00001a92       ?GdipInit@@YA_NXZ          10002a92 f   ConEmuBg.obj
 0001:00001b36       ?GetImage@GDIPlusDecoder@@QAEPAUCachedImage@@PB_W@Z 10002b36 f i ConEmuBg.obj
 0001:00001f23       ?GetMsgW@@YAPB_WH@Z        10002f23 f   ConEmuBg.obj
 0001:00001f63       ?GetPluginInfoWcmn@@YGXPAX@Z 10002f63 f   ConEmuBg.obj
 0001:00001f94       ?GetStatusLineCount@@YAHPAUPaintBackgroundArg@@H@Z 10002f94 f   ConEmuBg.obj
 0001:00002148       ?HSV2RGB@@YAXABUHSVColor@@AAURGBColor@@@Z 10003148 f   ConEmuBg.obj
 0001:00002459       ?Init@CachedImage@@QAE_NPB_WPAUHDC__@@IIQAU2@@Z 10003459 f i ConEmuBg.obj
 0001:00002543       ?Init@GDIPlusDecoder@@QAE_NXZ 10003543 f i ConEmuBg.obj
 0001:00002782       ?LoadFarVersion@@YAHXZ     10003782 f   ConEmuBg.obj
 0001:00002abc       ?OnConEmuLoaded@@YGXPAUConEmuLoadedArg@@@Z 10003abc f   ConEmuBg.obj
 0001:00002aec       ?OpenPluginWcmn@@YAPAXHH@Z 10003aec f   ConEmuBg.obj
 0001:00002b19       ?OpenW@@YGPAXPBX@Z         10003b19 f   ConEmuBg.obj
 0001:00002b44       ?PaintConEmuBackground@@YGHPAUPaintBackgroundArg@@@Z 10003b44 f   ConEmuBg.obj
 0001:00002c8d       ?PaintPanel@@YAHPAUPaintBackgroundArg@@HAAKAAH@Z 10003c8d f   ConEmuBg.obj
 0001:00003d32       ?ParseColors@@YAXPB_WHAAY0CA@KAAH@Z 10004d32 f   ConEmuBg.obj
 0001:00003ddd       ?QueryInterface@MStream@@UAGJABU_GUID@@PAPAX@Z 10004ddd f i ConEmuBg.obj
 0001:00003e45       ?RGB2HSV@@YAXABURGBColor@@AAUHSVColor@@@Z 10004e45 f   ConEmuBg.obj
 0001:00003f0b       ?Read@MStream@@UAGJPAXKPAK@Z 10004f0b f i ConEmuBg.obj
 0001:00003f60       ?Release@MStream@@UAGKXZ   10004f60 f i ConEmuBg.obj
 0001:00003f87       ?ReportFail@@YAXPB_W@Z     10004f87 f   ConEmuBg.obj
 0001:0000401f       ?Revert@MStream@@UAGJXZ    1000501f f i ConEmuBg.obj
 0001:00004027       ?Seek@MStream@@UAGJT_LARGE_INTEGER@@KPAT_ULARGE_INTEGER@@@Z 10005027 f i ConEmuBg.obj
 0001:000040a1       ?SetData@MStream@@QAEXPBXK@Z 100050a1 f i ConEmuBg.obj
 0001:000040e0       ?SetSize@MStream@@UAGJT_ULARGE_INTEGER@@@Z 100050e0 f i ConEmuBg.obj
 0001:00004153       ?SettingsLoad@@YAXXZ       10005153 f   ConEmuBg.obj
 0001:000041b2       ?SettingsLoadReg@@YAXPB_W@Z 100051b2 f   ConEmuBg.obj
 0001:0000433a       ?SettingsSave@@YAXXZ       1000533a f   ConEmuBg.obj
 0001:0000436f       ?SettingsSaveReg@@YAXPB_W@Z 1000536f f   ConEmuBg.obj
 0001:0000440e       ?StartPlugin@@YAXH@Z       1000540e f   ConEmuBg.obj
 0001:00004523       ?Stat@MStream@@UAGJPAUtagSTATSTG@@K@Z 10005523 f i ConEmuBg.obj
 0001:0000459b       ?StringCchCatW@@YGJPA_WIPB_W@Z 1000559b f i ConEmuBg.obj
 0001:000045d9       ?StringCchCopyW@@YGJPA_WIPB_W@Z 100055d9 f i ConEmuBg.obj
 0001:0000460d       ?StringCchVPrintfW@@YGJPA_WIPB_WPAD@Z 1000560d f i ConEmuBg.obj
 0001:00004746       ?WasXmlLoaded@@YA_NXZ      10005746 f   ConEmuBg.obj
 0001:00004751       ?Write@MStream@@UAGJPBXKPAK@Z 10005751 f i ConEmuBg.obj
 0001:000047e5       _DllMain@12                100057e5 f   ConEmuBg.obj
 0001:0000483c       _GetMinFarVersionW@0       1000583c f   ConEmuBg.obj
 0001:00004842       _SetStartupInfoW@4         10005842 f   ConEmuBg.obj
 0001:0000489d       ___local_stdio_printf_options 1000589d f i ConEmuBg.obj
 0001:000048a3       __vsnwprintf_l             100058a3 f i ConEmuBg.obj
 0001:00004c15       ?ConfigureW1900@@YAHH@Z    10005c15 f   ConEmuBg1900.obj
 0001:00004c2b       ?ExitFARW1900@@YAXXZ       10005c2b f   ConEmuBg1900.obj
 0001:00004c5a       ?FMatchW1900@@YA_NPB_WPA_W@Z 10005c5a f   ConEmuBg1900.obj
 0001:00004c7a       ?GetMsgW1900@@YAPB_WH@Z    10005c7a f   ConEmuBg1900.obj
 0001:00004ca0       ?GetPluginInfoW1900@@YAXPAX@Z 10005ca0 f   ConEmuBg1900.obj
 0001:00004d04       ?OpenW1900@@YGPAXPBX@Z     10005d04 f   ConEmuBg1900.obj
 0001:00004d04       ?OpenW2800@@YGPAXPBX@Z     10005d04 f   ConEmuBg2800.obj
 0001:00004d28       ?SetStartupInfoW1900@@YAXPAX@Z 10005d28 f   ConEmuBg1900.obj
 0001:00004e1d       ?SettingsLoadW1900@@YAXXZ  10005e1d f   ConEmuBg1900.obj
 0001:00004f70       ?SettingsSaveW1900@@YAXXZ  10005f70 f   ConEmuBg1900.obj
 0001:000053a8       ?ConfigureW2800@@YAHH@Z    100063a8 f   ConEmuBg2800.obj
 0001:000053be       ?ExitFARW2800@@YAXXZ       100063be f   ConEmuBg2800.obj
 0001:000053ed       ?FMatchW2800@@YA_NPB_WPA_W@Z 100063ed f   ConEmuBg2800.obj
 0001:0000540d       ?GetMsgW2800@@YAPB_WH@Z    1000640d f   ConEmuBg2800.obj
 0001:00005433       ?GetPluginInfoW2800@@YAXPAX@Z 10006433 f   ConEmuBg2800.obj
 0001:00005497       ?SetStartupInfoW2800@@YAXPAX@Z 10006497 f   ConEmuBg2800.obj
 0001:0000558c       ?SettingsLoadW2800@@YAXXZ  1000658c f   ConEmuBg2800.obj
 0001:000056d2       ?SettingsSaveW2800@@YAXXZ  100066d2 f   ConEmuBg2800.obj
 0001:000057c1       _GetGlobalInfoW@4          100067c1 f   ConEmuBg2800.obj
 0001:00005b8d       ?ConfigureW995@@YAHH@Z     10006b8d f   ConEmuBg995.obj
 0001:00005ba3       ?ExitFARW995@@YAXXZ        10006ba3 f   ConEmuBg995.obj
 0001:00005be9       ?FMatchW995@@YA_NPB_WPA_W@Z 10006be9 f   ConEmuBg995.obj
 0001:00005c08       ?GetMsgW995@@YAPB_WH@Z     10006c08 f   ConEmuBg995.obj
 0001:00005c2c       ?GetPluginInfoW995@@YAXPAX@Z 10006c2c f   ConEmuBg995.obj
 0001:00005c83       ?SetStartupInfoW995@@YAXPAX@Z 10006c83 f   ConEmuBg995.obj
 0001:00005dc0       ?SettingsLoadW995@@YAXXZ   10006dc0 f   ConEmuBg995.obj
 0001:00005dcd       ?SettingsSaveW995@@YAXXZ   10006dcd f   ConEmuBg995.obj
 0001:00005dda       _OpenPluginW@8             10006dda f   ConEmuBg995.obj
 0001:000061cd       ?FMatchA@@YA_NPBDPAD@Z     100071cd f   ConEmuBgA.obj
 0001:000061ea       ?SettingsLoadA@@YAXXZ      100071ea f   ConEmuBgA.obj
 0001:000061f7       ?SettingsSaveA@@YAXXZ      100071f7 f   ConEmuBgA.obj
 0001:00006204       _Configure@4               10007204 f   ConEmuBgA.obj
 0001:00006221       _ExitFAR@0                 10007221 f   ConEmuBgA.obj
 0001:0000626c       _GetMinFarVersion@0        1000726c f   ConEmuBgA.obj
 0001:00006291       _GetPluginInfo@4           10007291 f   ConEmuBgA.obj
 0001:000062fd       _OpenPlugin@8              100072fd f   ConEmuBgA.obj
 0001:00006314       _SetStartupInfo@4          10007314 f   ConEmuBgA.obj
 0001:0000647e       _GetFileVersionInfoSizeW@8 1000747e f   version:VERSION.dll
 0001:00006484       _GetFileVersionInfoW@16    10007484 f   version:VERSION.dll
 0001:0000648a       _VerQueryValueW@16         1000748a f   version:VERSION.dll
 0001:00006490       ??2@YAPAXI@Z               10007490 f   common-kernel32:Memory.obj
 0001:000064b9       ??_V@YAXPAX@Z              100074b9 f   common-kernel32:Memory.obj
 0001:000064b9       ??3@YAXPAX@Z               100074b9 f   common-kernel32:Memory.obj
 0001:000064b9       ?xf_free@@YAXPAX@Z         100074b9 f   common-kernel32:Memory.obj
 0001:000064d9       ??_U@YAPAXI@Z              100074d9 f   common-kernel32:Memory.obj
 0001:000064d9       ?xf_malloc@@YAPAXI@Z       100074d9 f   common-kernel32:Memory.obj
 0001:000064ef       ?HeapDeinitialize@@YAXXZ   100074ef f   common-kernel32:Memory.obj
 0001:00006507       ?HeapInitialize@@YA_NXZ    10007507 f   common-kernel32:Memory.obj
 0001:00006529       ?xf_calloc@@YAPAXII@Z      10007529 f   common-kernel32:Memory.obj
 0001:00006544       ?StringCchVPrintfA@@YGJPADIPBD0@Z 10007544 f i common-kernel32:MStrSafe.obj
 0001:00006599       ?sprintf_c@@YAHPADHPBDZZ   10007599 f   common-kernel32:MStrSafe.obj
 0001:000065bc       ?swprintf_c@@YAHPA_WHPB_WZZ 100075bc f   common-kernel32:MStrSafe.obj
 0001:000065df       __vsnprintf_l              100075df f i common-kernel32:MStrSafe.obj
 0001:00006611       ?lstrdup@@YAPA_WPB_WI@Z    10007611 f   common-kernel32:MStrDup.obj
 0001:0000665d       ?lstrmerge@@YAPA_WPB_W00000000@Z 1000765d f   common-kernel32:MStrDup.obj
 0001:00006757       ??0MSectionLockSimple@@QAE@XZ 10007757 f   common-kernel32:MSectionSimple.obj
 0001:00006761       ??0MSectionSimple@@QAE@_N@Z 10007761 f   common-kernel32:MSectionSimple.obj
 0001:00006794       ??1MSectionLockSimple@@QAE@XZ 10007794 f   common-kernel32:MSectionSimple.obj
 0001:0000679f       ??1MSectionSimple@@QAE@XZ  1000779f f   common-kernel32:MSectionSimple.obj
 0001:000067b5       ?Lock@MSectionLockSimple@@QAEHPAUMSectionSimple@@K@Z 100077b5 f   common-kernel32:MSectionSimple.obj
 0001:0000681b       ?TryEnter@MSectionSimple@@QAE_NXZ 1000781b f   common-kernel32:MSectionSimple.obj
 0001:0000683a       ?Unlock@MSectionLockSimple@@QAEXXZ 1000783a f   common-kernel32:MSectionSimple.obj
 0001:00006856       ??$sprintf_c@$0CI@@@YAHAAY0CI@DPBDZZ 10007856 f i common-kernel32:WThreads.obj
 0001:0000686c       ?SetThreadName@@YAXKPAD@Z  1000786c f   common-kernel32:WThreads.obj
 0001:000068c5       ?apiCreateThread@@YAPAXP6GKPAX@Z0PAKPBDH@Z 100078c5 f   common-kernel32:WThreads.obj
 0001:000069bd       ?apiTerminateThreadEx@@YAHPAXKPBDH@Z 100079bd f   common-kernel32:WThreads.obj
 0001:00006a91       ?apiThreadHelper@@YGKPAX@Z 10007a91 f   common-kernel32:WThreads.obj
 0001:00006c1d       ??3@YAXPAXI@Z              10007c1d f   LIBCMT:delete_scalar_size.obj
 0001:00006c2b       ___raise_securityfailure   10007c2b f   LIBCMT:gs_report.obj
 0001:00006c53       ___report_gsfailure        10007c53 f   LIBCMT:gs_report.obj
 0001:00006d4e       ___report_rangecheckfailure 10007d4e f   LIBCMT:gs_report.obj
 0001:00006d5a       ___report_securityfailure  10007d5a f   LIBCMT:gs_report.obj
 0001:00006e2a       @__security_check_cookie@4 10007e2a f   LIBCMT:_secchk_.obj
 0001:00006e3b       __EH_epilog3               10007e3b f   LIBCMT:ehprolg3.obj
 0001:00006e50       __EH_epilog3_GS            10007e50 f   LIBCMT:ehprolg3.obj
 0001:00006e61       __EH_prolog3               10007e61 f   LIBCMT:ehprolg3.obj
 0001:00006e95       __EH_prolog3_GS            10007e95 f   LIBCMT:ehprolg3.obj
 0001:00006ecc       __EH_prolog3_catch         10007ecc f   LIBCMT:ehprolg3.obj
 0001:00006f10       __allmul                   10007f10 f   LIBCMT:llmul.obj
 0001:00006f50       __aulldiv                  10007f50 f   LIBCMT:ulldiv.obj
 0001:00006fb8       ??_Gtype_info@@UAEPAXI@Z   10007fb8 f i LIBCMT:std_type_info_static.obj
 0001:00006fb8       ??_Etype_info@@UAEPAXI@Z   10007fb8 f i LIBCMT:std_type_info_static.obj
 0001:00007002       ??$__crt_fast_encode_pointer@P6GHPAU_RTL_CONDITION_VARIABLE@@PAU_RTL_CRITICAL_SECTION@@K@Z@@YAP6GHPAU_RTL_CONDITION_VARIABLE@@PAU_RTL_CRITICAL_SECTION@@K@ZQ6GH01K@Z@Z 10008002 f i LIBCMT:thread_safe_statics.obj
 0001:00007002       ??$__crt_fast_encode_pointer@PAX@@YAPAXQAX@Z 10008002 f i libvcruntime:winapi_downlevel.obj
 0001:00007002       ??$__crt_fast_encode_pointer@PAP6AXXZ@@YAPAP6AXXZQAP6AXXZ@Z 10008002 f i LIBCMT:utility.obj
 0001:00007002       ??$__crt_fast_encode_pointer@P6GXPAU_RTL_CONDITION_VARIABLE@@@Z@@YAP6GXPAU_RTL_CONDITION_VARIABLE@@@ZQ6GX0@Z@Z 10008002 f i LIBCMT:thread_safe_statics.obj
 0001:0000712a       __Init_thread_footer       1000812a f   LIBCMT:thread_safe_statics.obj
 0001:00007174       __Init_thread_header       10008174 f   LIBCMT:thread_safe_statics.obj
 0001:000071c6       __Init_thread_notify       100081c6 f   LIBCMT:thread_safe_statics.obj
 0001:00007208       __Init_thread_wait         10008208 f   LIBCMT:thread_safe_statics.obj
 0001:00007574       __DllMainCRTStartup@12     10008574 f   LIBCMT:dll_dllmain.obj
 0001:000075a0       __SEH_prolog4              100085a0 f   LIBCMT:_sehprolg4_.obj
 0001:000075e6       __SEH_epilog4              100085e6 f   LIBCMT:_sehprolg4_.obj
 0001:0000763f       ___scrt_acquire_startup_lock 1000863f f   LIBCMT:utility.obj
 0001:00007671       ___scrt_dllmain_after_initialize_c 10008671 f   LIBCMT:utility.obj
 0001:0000769c       ___scrt_dllmain_before_initialize_c 1000869c f   LIBCMT:utility.obj
 0001:000076aa       ___scrt_dllmain_crt_thread_attach 100086aa f   LIBCMT:utility.obj
 0001:000076c9       ___scrt_dllmain_crt_thread_detach 100086c9 f   LIBCMT:utility.obj
 0001:000076d6       ___scrt_dllmain_exception_filter 100086d6 f   LIBCMT:utility.obj
 0001:0000770a       ___scrt_dllmain_uninitialize_c 1000870a f   LIBCMT:utility.obj
 0001:0000772d       ___scrt_dllmain_uninitialize_critical 1000872d f   LIBCMT:utility.obj
 0001:0000773a       ___scrt_initialize_crt     1000873a f   LIBCMT:utility.obj
 0001:00007773       ___scrt_initialize_onexit_tables 10008773 f   LIBCMT:utility.obj
 0001:0000781d       ___scrt_is_nonwritable_in_current_image 1000881d f   LIBCMT:utility.obj
 0001:000078a7       ___scrt_release_startup_lock 100088a7 f   LIBCMT:utility.obj
 0001:000078c4       ___scrt_uninitialize_crt   100088c4 f   LIBCMT:utility.obj
 0001:000078ec       __onexit                   100088ec f   LIBCMT:utility.obj
 0001:00007927       _atexit                    10008927 f   LIBCMT:utility.obj
 0001:0000793c       ___scrt_fastfail           1000893c f   LIBCMT:utility_desktop.obj
 0001:00007a58       __crt_debugger_hook        10008a58 f   LIBCMT:utility_desktop.obj
 0001:00007a60       @_guard_check_icall_nop@4  10008a60 f i LIBCMT:guard_support.obj
 0001:00007ab0       ___security_init_cookie    10008ab0 f   LIBCMT:gs_support.obj
 0001:00007afb       ?__scrt_initialize_type_info@@YAXXZ 10008afb f   LIBCMT:tncleanup.obj
 0001:00007b07       ?__scrt_uninitialize_type_info@@YAXXZ 10008b07 f   LIBCMT:tncleanup.obj
 0001:00007b13       ___local_stdio_scanf_options 10008b13 f i LIBCMT:default_local_stdio_options.obj
 0001:00007b19       ___scrt_initialize_default_local_stdio_options 10008b19 f   LIBCMT:default_local_stdio_options.obj
 0001:00007b36       ___scrt_get_dyn_tls_init_callback 10008b36 f   LIBCMT:dyn_tls_init.obj
 0001:00007b3c       __RTC_Initialize           10008b3c f   LIBCMT:_initsect_.obj
 0001:00007b68       __RTC_Terminate            10008b68 f   LIBCMT:_initsect_.obj
 0001:00007b94       ___isa_available_init      10008b94 f   LIBCMT:_cpu_disp_.obj
 0001:00007d2d       __get_startup_argv_mode    10008d2d f   LIBCMT:argv_mode.obj
 0001:00007d31       ___scrt_is_ucrt_dll_in_use 10008d31 f   LIBCMT:ucrt_detection.obj
 0001:00007d3d       _wcschr                    10008d3d f   libvcruntime:wcschr.obj
 0001:00007e07       _wcsrchr                   10008e07 f   libvcruntime:wcsrchr.obj
 0001:00007ea9       _wcsstr                    10008ea9 f   libvcruntime:wcsstr.obj
 0001:0000812c       ?_CallCatchBlock2@@YAPAXPAUEHRegistrationNode@@PBU_s_FuncInfo@@PAXHK@Z 1000912c f   libvcruntime:trnsctrl.obj
 0001:0000818c       ?_CallSETranslator@@YAHPAUEHExceptionRecord@@PAUEHRegistrationNode@@PAX2PBU_s_FuncInfo@@H1@Z 1000918c f   libvcruntime:trnsctrl.obj
 0001:00008269       ?_GetRangeOfTrysToCheck@@YAPBU_s_TryBlockMapEntry@@PBU_s_FuncInfo@@HHPAI1@Z 10009269 f   libvcruntime:trnsctrl.obj
 0001:000082e1       ?_JumpToContinuation@@YGXPAXPAUEHRegistrationNode@@@Z 100092e1 f   libvcruntime:trnsctrl.obj
 0001:00008313       ?_UnwindNestedFrames@@YGXPAUEHRegistrationNode@@PAUEHExceptionRecord@@@Z 10009313 f   libvcruntime:trnsctrl.obj
 0001:00008368       __CatchGuardHandler        10009368 f   libvcruntime:trnsctrl.obj
 0001:00008399       __CreateFrameInfo          10009399 f   libvcruntime:trnsctrl.obj
 0001:000083bd       __FindAndUnlinkFrame       100093bd f   libvcruntime:trnsctrl.obj
 0001:00008402       __TranslatorGuardHandler   10009402 f   libvcruntime:trnsctrl.obj
 0001:000084a1       ___CxxFrameHandler3        100094a1 f   libvcruntime:trnsctrl.obj
 0001:000084e0       _memmove                   100094e0 f   libvcruntime:memmove.obj
 0001:00008a60       _memset                    10009a60 f   libvcruntime:memset.obj
 0001:00008bc0       _strchr                    10009bc0 f   libvcruntime:strchr.obj
 0001:00008c2e       ___from_strstr_to_strchr   10009c2e     libvcruntime:strchr.obj
 0001:00008cf0       _strrchr                   10009cf0 f   libvcruntime:strrchr.obj
 0001:00008e70       __except_handler4          10009e70 f   libvcruntime:_chandler4_.obj
 0001:00008fc7       ___vcrt_initialize         10009fc7 f   libvcruntime:initialization.obj
 0001:00008ff0       ___vcrt_thread_attach      10009ff0 f   libvcruntime:initialization.obj
 0001:00008ffb       ___vcrt_thread_detach      10009ffb f   libvcruntime:initialization.obj
 0001:00009006       ___vcrt_uninitialize       1000a006 f   libvcruntime:initialization.obj
 0001:00009025       ___vcrt_uninitialize_critical 1000a025 f   libvcruntime:initialization.obj
 0001:0000902d       ___std_type_info_compare   1000a02d f   libvcruntime:std_type_info.obj
 0001:00009069       ___std_type_info_destroy_list 1000a069 f   libvcruntime:std_type_info.obj
 0001:0000908c       ___vcrt_freefls@4          1000a08c f   libvcruntime:per_thread_data.obj
 0001:000090a8       ___vcrt_freeptd            1000a0a8 f   libvcruntime:per_thread_data.obj
 0001:000090eb       ___vcrt_getptd             1000a0eb f   libvcruntime:per_thread_data.obj
 0001:000090f9       ___vcrt_getptd_noexit      1000a0f9 f   libvcruntime:per_thread_data.obj
 0001:0000918b       ___vcrt_initialize_ptd     1000a18b f   libvcruntime:per_thread_data.obj
 0001:000091cf       ___vcrt_uninitialize_ptd   1000a1cf f   libvcruntime:per_thread_data.obj
 0001:000091f0       __CallSettingFrame@12      1000a1f0 f   libvcruntime:lowhelpr.obj
 0001:00009217       __NLG_Return               1000a217     libvcruntime:lowhelpr.obj
 0001:0000923c       ??0bad_exception@std@@QAE@ABV01@@Z 1000a23c f i libvcruntime:frame.obj
 0001:00009257       ??0bad_exception@std@@QAE@XZ 1000a257 f i libvcruntime:frame.obj
 0001:0000926f       ??0exception@std@@QAE@ABV01@@Z 1000a26f f i libvcruntime:frame.obj
 0001:0000929b       ??1bad_exception@std@@UAE@XZ 1000a29b f i libvcruntime:frame.obj
 0001:000092ac       ??8type_info@@QBE_NABV0@@Z 1000a2ac f i libvcruntime:frame.obj
 0001:000092cb       ??_Gexception@std@@UAEPAXI@Z 1000a2cb f i libvcruntime:frame.obj
 0001:000092cb       ??_Ebad_exception@std@@UAEPAXI@Z 1000a2cb f i libvcruntime:frame.obj
 0001:000092cb       ??_Eexception@std@@UAEPAXI@Z 1000a2cb f i libvcruntime:frame.obj
 0001:000092cb       ??_Gbad_exception@std@@UAEPAXI@Z 1000a2cb f i libvcruntime:frame.obj
 0001:00009ae9       ?_CallMemberFunction1@@YGXQAX00@Z 1000aae9 f i libvcruntime:frame.obj
 0001:00009af9       ?_CallMemberFunction2@@YGXQAX00H@Z 1000aaf9 f i libvcruntime:frame.obj
 0001:00009b0c       ?what@exception@std@@UBEPBDXZ 1000ab0c f i libvcruntime:frame.obj
 0001:00009b19       ___BuildCatchObject        1000ab19 f   libvcruntime:frame.obj
 0001:00009ba8       ___BuildCatchObjectHelper  1000aba8 f   libvcruntime:frame.obj
 0001:00009cdc       ___FrameUnwindToState      1000acdc f   libvcruntime:frame.obj
 0001:00009da9       ___InternalCxxFrameHandler 1000ada9 f   libvcruntime:frame.obj
 0001:00009ea6       ___TypeMatch               1000aea6 f   libvcruntime:frame.obj
 0001:00009f34       ___except_validate_context_record 1000af34 f   libvcruntime:jbcxrval.obj
 0001:00009f64       ___except_validate_jump_buffer 1000af64 f   libvcruntime:jbcxrval.obj
 0001:00009fa0       __local_unwind4            1000afa0 f   libvcruntime:_exsup4_.obj
 0001:0000a078       __seh_longjmp_unwind4@4    1000b078 f   libvcruntime:_exsup4_.obj
 0001:0000a0a0       @_EH4_CallFilterFunc@8     1000b0a0 f   libvcruntime:_exsup4_.obj
 0001:0000a0b8       @_EH4_TransferToHandler@8  1000b0b8 f   libvcruntime:_exsup4_.obj
 0001:0000a0d4       @_EH4_GlobalUnwind2@8      1000b0d4 f   libvcruntime:_exsup4_.obj
 0001:0000a0f0       @_EH4_LocalUnwind@16       1000b0f0 f   libvcruntime:_exsup4_.obj
 0001:0000a107       ___vcrt_initialize_locks   1000b107 f   libvcruntime:locks.obj
 0001:0000a143       ___vcrt_uninitialize_locks 1000b143 f   libvcruntime:locks.obj
 0001:0000a2a7       ___vcrt_FlsAlloc           1000b2a7 f   libvcruntime:winapi_downlevel.obj
 0001:0000a2e2       ___vcrt_FlsFree            1000b2e2 f   libvcruntime:winapi_downlevel.obj
 0001:0000a31d       ___vcrt_FlsGetValue        1000b31d f   libvcruntime:winapi_downlevel.obj
 0001:0000a358       ___vcrt_FlsSetValue        1000b358 f   libvcruntime:winapi_downlevel.obj
 0001:0000a396       ___vcrt_InitializeCriticalSectionEx 1000b396 f   libvcruntime:winapi_downlevel.obj
 0001:0000a3dd       ___vcrt_initialize_winapi_thunks 1000b3dd f   libvcruntime:winapi_downlevel.obj
 0001:0000a406       ___vcrt_uninitialize_winapi_thunks 1000b406 f   libvcruntime:winapi_downlevel.obj
 0001:0000a438       ___vcrt_initialize_pure_virtual_call_handler 1000b438 f   libvcruntime:purevirt_data.obj
 0001:0000a450       __global_unwind2           1000b450 f   libvcruntime:_exsup_.obj
 0001:0000a4b6       __local_unwind2            1000b4b6 f   libvcruntime:_exsup_.obj
 0001:0000a53a       __abnormal_termination     1000b53a f   libvcruntime:_exsup_.obj
 0001:0000a560       __NLG_Notify1              1000b560 f   libvcruntime:_exsup_.obj
 0001:0000a56c       __NLG_Notify               1000b56c f   libvcruntime:_exsup_.obj
 0001:0000a583       __NLG_Dispatch2            1000b583     libvcruntime:_exsup_.obj
 0001:0000a583       __NLG_Dispatch             1000b583     libvcruntime:_exsup_.obj
 0001:0000a58b       __NLG_Call                 1000b58b f   libvcruntime:_exsup_.obj
 0001:0000a58d       __NLG_Return2              1000b58d     libvcruntime:_exsup_.obj
 0001:0000a58e       _unexpected                1000b58e f   libvcruntime:unexpected.obj
 0001:0000a5ab       ___DestructExceptionObject 1000b5ab f   libvcruntime:ehhelpers.obj
 0001:0000a641       ?_CallMemberFunction0@@YGXQAX0@Z 1000b641 f i libvcruntime:ehhelpers.obj
 0001:0000a64e       __IsExceptionObjectToBeDestroyed 1000b64e f   libvcruntime:ehhelpers.obj
 0001:0000a674       ___AdjustPointer           1000b674 f   libvcruntime:ehhelpers.obj
 0001:0000a699       ___FrameUnwindFilter       1000b699 f   libvcruntime:ehhelpers.obj
 0001:0000a6de       ___std_exception_copy      1000b6de f   libvcruntime:std_exception.obj
 0001:0000a741       ___std_exception_destroy   1000b741 f   libvcruntime:std_exception.obj
 0001:0000a760       __CxxThrowException@8      1000b760 f   libvcruntime:throw.obj
 0001:0000a7d0       _memcpy                    1000b7d0 f   libvcruntime:memcpy.obj
 0001:0000ad44       ??$is_overflow_condition@K@__crt_strtox@@YA_NIK@Z 1000bd44 f i libucrt:strtox.obj
 0001:0000ad77       ??$make_c_string_character_source@_WPAPA_W@__crt_strtox@@YA?AV?$c_string_character_source@_W@0@QB_WQAPA_W@Z 1000bd77 f i libucrt:strtox.obj
 0001:0000ad77       ??$make_c_string_character_source@DPAPAD@__crt_strtox@@YA?AV?$c_string_character_source@D@0@QBDQAPAD@Z 1000bd77 f i libucrt:strtox.obj
 0001:0000ad92       ??$parse_integer@KV?$c_string_character_source@D@__crt_strtox@@@__crt_strtox@@YAKQAU__crt_locale_pointers@@V?$c_string_character_source@D@0@H_N@Z 1000bd92 f i libucrt:strtox.obj
 0001:0000afba       ??$parse_integer@KV?$c_string_character_source@_W@__crt_strtox@@@__crt_strtox@@YAKQAU__crt_locale_pointers@@V?$c_string_character_source@_W@0@H_N@Z 1000bfba f i libucrt:strtox.obj
 0001:0000b69f       ??0_LocaleUpdate@@QAE@QAU__crt_locale_pointers@@@Z 1000c69f f i libucrt:strtox.obj
 0001:0000b722       ?unget@?$c_string_character_source@D@__crt_strtox@@QAEXD@Z 1000c722 f i libucrt:strtox.obj
 0001:0000b74a       ?unget@?$c_string_character_source@_W@__crt_strtox@@QAEX_W@Z 1000c74a f i libucrt:strtox.obj
 0001:0000b776       ?validate@?$string_output_adapter@_W@__crt_stdio_output@@QBE_NXZ 1000c776 f i libucrt:output.obj
 0001:0000b776       ?validate@?$c_string_character_source@_W@__crt_strtox@@QBE_NXZ 1000c776 f i libucrt:strtox.obj
 0001:0000b776       ?validate@?$string_output_adapter@D@__crt_stdio_output@@QBE_NXZ 1000c776 f i libucrt:output.obj
 0001:0000b776       ?validate@?$c_string_character_source@D@__crt_strtox@@QBE_NXZ 1000c776 f i libucrt:strtox.obj
 0001:0000b791       __chvalidchk_l             1000c791 f i libucrt:strtox.obj
 0001:0000b7bb       __ischartype_l             1000c7bb f i libucrt:strtox.obj
 0001:0000b7ee       _strtol                    1000c7ee f   libucrt:strtox.obj
 0001:0000b81a       _wcstol                    1000c81a f   libucrt:strtox.obj
 0001:0000b846       _wcstoul                   1000c846 f   libucrt:strtox.obj
 0001:0000bb73       ??$count@D@formatting_buffer@__crt_stdio_output@@QBEIXZ 1000cb73 f i libucrt:output.obj
 0001:0000bb8b       ??$ensure_buffer_is_big_enough@D@formatting_buffer@__crt_stdio_output@@QAE_NI@Z 1000cb8b f i libucrt:output.obj
 0001:0000bc11       ??$is_wide_character_specifier@D@__crt_stdio_output@@YA_N_KDW4length_modifier@0@@Z 1000cc11 f i libucrt:output.obj
 0001:0000bc51       ??$is_wide_character_specifier@_W@__crt_stdio_output@@YA_N_K_WW4length_modifier@0@@Z 1000cc51 f i libucrt:output.obj
 0001:0000bca0       ??$scratch_data@D@formatting_buffer@__crt_stdio_output@@QAEPADXZ 1000cca0 f i libucrt:output.obj
 0001:0000bcbe       ??$type_case_integer_parse_into_buffer@I@?$output_processor@DV?$string_output_adapter@D@__crt_stdio_output@@V?$standard_base@DV?$string_output_adapter@D@__crt_stdio_output@@@2@@__crt_stdio_output@@AAEXII_N@Z 1000ccbe f i libucrt:output.obj
 0001:0000bcbe       ??$type_case_integer_parse_into_buffer@I@?$output_processor@_WV?$string_output_adapter@_W@__crt_stdio_output@@V?$standard_base@_WV?$string_output_adapter@_W@__crt_stdio_output@@@2@@__crt_stdio_output@@AAEXII_N@Z 1000ccbe f i libucrt:output.obj
 0001:0000bd33       ??$type_case_integer_parse_into_buffer@_K@?$output_processor@_WV?$string_output_adapter@_W@__crt_stdio_output@@V?$standard_base@_WV?$string_output_adapter@_W@__crt_stdio_output@@@2@@__crt_stdio_output@@AAEX_KI_N@Z 1000cd33 f i libucrt:output.obj
 0001:0000bd33       ??$type_case_integer_parse_into_buffer@_K@?$output_processor@DV?$string_output_adapter@D@__crt_stdio_output@@V?$standard_base@DV?$string_output_adapter@D@__crt_stdio_output@@@2@@__crt_stdio_output@@AAEX_KI_N@Z 1000cd33 f i libucrt:output.obj
 0001:0000bdbb       ??$write_multiple_characters@V?$string_output_adapter@D@__crt_stdio_output@@D@__crt_stdio_output@@YAXABV?$string_output_adapter@D@0@DHQAH@Z 1000cdbb f i libucrt:output.obj
 0001:0000bde7       ??$write_multiple_characters@V?$string_output_adapter@_W@__crt_stdio_output@@D@__crt_stdio_output@@YAXABV?$string_output_adapter@_W@0@DHQAH@Z 1000cde7 f i libucrt:output.obj
 0001:0000be18       ??0?$common_data@D@__crt_stdio_output@@IAE@XZ 1000ce18 f i libucrt:output.obj
 0001:0000be5f       ??0?$common_data@_W@__crt_stdio_output@@IAE@XZ 1000ce5f f i libucrt:output.obj
 0001:0000beab       ??0?$output_adapter_data@DV?$string_output_adapter@D@__crt_stdio_output@@@__crt_stdio_output@@IAE@ABV?$string_output_adapter@D@1@_KQBDQAU__crt_locale_pointers@@QAD@Z 1000ceab f i libucrt:output.obj
 0001:0000bee7       ??0?$output_adapter_data@_WV?$string_output_adapter@_W@__crt_stdio_output@@@__crt_stdio_output@@IAE@ABV?$string_output_adapter@_W@1@_KQB_WQAU__crt_locale_pointers@@QAD@Z 1000cee7 f i libucrt:output.obj
 0001:0000bf23       ??0?$output_processor@DV?$string_output_adapter@D@__crt_stdio_output@@V?$standard_base@DV?$string_output_adapter@D@__crt_stdio_output@@@2@@__crt_stdio_output@@QAE@ABV?$string_output_adapter@D@1@_KQBDQAU__crt_locale_pointers@@QAD@Z 1000cf23 f i libucrt:output.obj
 0001:0000bf58       ??0?$output_processor@_WV?$string_output_adapter@_W@__crt_stdio_output@@V?$standard_base@_WV?$string_output_adapter@_W@__crt_stdio_output@@@2@@__crt_stdio_output@@QAE@ABV?$string_output_adapter@_W@1@_KQB_WQAU__crt_locale_pointers@@QAD@Z 1000cf58 f i libucrt:output.obj
 0001:0000bf8d       ??1formatting_buffer@__crt_stdio_output@@QAE@XZ 1000cf8d f i libucrt:output.obj
 0001:0000bfa7       ??4?$__crt_unique_heap_ptr@DU__crt_internal_free_policy@@@@QAEAAV0@$$QAV0@@Z 1000cfa7 f i libucrt:output.obj
 0001:0000bfcb       ?crop_zeroes@__crt_stdio_output@@YAXPADQAU__crt_locale_pointers@@@Z 1000cfcb f i libucrt:output.obj
 0001:0000c022       ?find_next_state@?$output_processor@DV?$string_output_adapter@D@__crt_stdio_output@@V?$standard_base@DV?$string_output_adapter@D@__crt_stdio_output@@@2@@__crt_stdio_output@@ABE?AW4state@2@DW432@@Z 1000d022 f i libucrt:output.obj
 0001:0000c054       ?find_next_state@?$output_processor@_WV?$string_output_adapter@_W@__crt_stdio_output@@V?$standard_base@_WV?$string_output_adapter@_W@__crt_stdio_output@@@2@@__crt_stdio_output@@ABE?AW4state@2@_WW432@@Z 1000d054 f i libucrt:output.obj
 0001:0000c088       ?force_decimal_point@__crt_stdio_output@@YAXPADQAU__crt_locale_pointers@@@Z 1000d088 f i libucrt:output.obj
 0001:0000c0e4       ?parse_int_from_format_string@?$output_processor@DV?$string_output_adapter@D@__crt_stdio_output@@V?$standard_base@DV?$string_output_adapter@D@__crt_stdio_output@@@2@@__crt_stdio_output@@AAE_NQAH@Z 1000d0e4 f i libucrt:output.obj
 0001:0000c140       ?parse_int_from_format_string@?$output_processor@_WV?$string_output_adapter@_W@__crt_stdio_output@@V?$standard_base@_WV?$string_output_adapter@_W@__crt_stdio_output@@@2@@__crt_stdio_output@@AAE_NQAH@Z 1000d140 f i libucrt:output.obj
 0001:0000c19e       ?process@?$output_processor@DV?$string_output_adapter@D@__crt_stdio_output@@V?$standard_base@DV?$string_output_adapter@D@__crt_stdio_output@@@2@@__crt_stdio_output@@QAEHXZ 1000d19e f i libucrt:output.obj
 0001:0000c2ba       ?process@?$output_processor@_WV?$string_output_adapter@_W@__crt_stdio_output@@V?$standard_base@_WV?$string_output_adapter@_W@__crt_stdio_output@@@2@@__crt_stdio_output@@QAEHXZ 1000d2ba f i libucrt:output.obj
 0001:0000c3da       ?state_case_flag@?$output_processor@DV?$string_output_adapter@D@__crt_stdio_output@@V?$standard_base@DV?$string_output_adapter@D@__crt_stdio_output@@@2@@__crt_stdio_output@@AAE_NXZ 1000d3da f i libucrt:output.obj
 0001:0000c417       ?state_case_flag@?$output_processor@_WV?$string_output_adapter@_W@__crt_stdio_output@@V?$standard_base@_WV?$string_output_adapter@_W@__crt_stdio_output@@@2@@__crt_stdio_output@@AAE_NXZ 1000d417 f i libucrt:output.obj
 0001:0000c454       ?state_case_normal@?$output_processor@DV?$string_output_adapter@D@__crt_stdio_output@@V?$standard_base@DV?$string_output_adapter@D@__crt_stdio_output@@@2@@__crt_stdio_output@@AAE_NXZ 1000d454 f i libucrt:output.obj
 0001:0000c473       ?state_case_normal@?$output_processor@_WV?$string_output_adapter@_W@__crt_stdio_output@@V?$standard_base@_WV?$string_output_adapter@_W@__crt_stdio_output@@@2@@__crt_stdio_output@@AAE_NXZ 1000d473 f i libucrt:output.obj
 0001:0000c492       ?state_case_normal_common@?$output_processor@DV?$string_output_adapter@D@__crt_stdio_output@@V?$standard_base@DV?$string_output_adapter@D@__crt_stdio_output@@@2@@__crt_stdio_output@@AAE_NXZ 1000d492 f i libucrt:output.obj
 0001:0000c4bc       ?state_case_normal_common@?$output_processor@_WV?$string_output_adapter@_W@__crt_stdio_output@@V?$standard_base@_WV?$string_output_adapter@_W@__crt_stdio_output@@@2@@__crt_stdio_output@@AAE_NXZ 1000d4bc f i libucrt:output.obj
 0001:0000c4d7       ?state_case_normal_tchar@?$output_processor@DV?$string_output_adapter@D@__crt_stdio_output@@V?$standard_base@DV?$string_output_adapter@D@__crt_stdio_output@@@2@@__crt_stdio_output@@AAE_ND@Z 1000d4d7 f i libucrt:output.obj
 0001:0000c538       ?state_case_precision@?$output_processor@DV?$string_output_adapter@D@__crt_stdio_output@@V?$standard_base@DV?$string_output_adapter@D@__crt_stdio_output@@@2@@__crt_stdio_output@@AAE_NXZ 1000d538 f i libucrt:output.obj
 0001:0000c560       ?state_case_precision@?$output_processor@_WV?$string_output_adapter@_W@__crt_stdio_output@@V?$standard_base@_WV?$string_output_adapter@_W@__crt_stdio_output@@@2@@__crt_stdio_output@@AAE_NXZ 1000d560 f i libucrt:output.obj
 0001:0000c589       ?state_case_size@?$output_processor@DV?$string_output_adapter@D@__crt_stdio_output@@V?$standard_base@DV?$string_output_adapter@D@__crt_stdio_output@@@2@@__crt_stdio_output@@AAE_NXZ 1000d589 f i libucrt:output.obj
 0001:0000c6f2       ?state_case_size@?$output_processor@_WV?$string_output_adapter@_W@__crt_stdio_output@@V?$standard_base@_WV?$string_output_adapter@_W@__crt_stdio_output@@@2@@__crt_stdio_output@@AAE_NXZ 1000d6f2 f i libucrt:output.obj
 0001:0000c86e       ?state_case_type@?$output_processor@DV?$string_output_adapter@D@__crt_stdio_output@@V?$standard_base@DV?$string_output_adapter@D@__crt_stdio_output@@@2@@__crt_stdio_output@@AAE_NXZ 1000d86e f i libucrt:output.obj
 0001:0000ca9d       ?state_case_type@?$output_processor@_WV?$string_output_adapter@_W@__crt_stdio_output@@V?$standard_base@_WV?$string_output_adapter@_W@__crt_stdio_output@@@2@@__crt_stdio_output@@AAE_NXZ 1000da9d f i libucrt:output.obj
 0001:0000ccfa       ?state_case_width@?$output_processor@DV?$string_output_adapter@D@__crt_stdio_output@@V?$standard_base@DV?$string_output_adapter@D@__crt_stdio_output@@@2@@__crt_stdio_output@@AAE_NXZ 1000dcfa f i libucrt:output.obj
 0001:0000cd25       ?state_case_width@?$output_processor@_WV?$string_output_adapter@_W@__crt_stdio_output@@V?$standard_base@_WV?$string_output_adapter@_W@__crt_stdio_output@@@2@@__crt_stdio_output@@AAE_NXZ 1000dd25 f i libucrt:output.obj
 0001:0000cd51       ?to_integer_size@__crt_stdio_output@@YAIW4length_modifier@1@@Z 1000dd51 f i libucrt:output.obj
 0001:0000cdad       ?type_case_Z@?$output_processor@DV?$string_output_adapter@D@__crt_stdio_output@@V?$standard_base@DV?$string_output_adapter@D@__crt_stdio_output@@@2@@__crt_stdio_output@@AAE_NXZ 1000ddad f i libucrt:output.obj
 0001:0000ce10       ?type_case_Z@?$output_processor@_WV?$string_output_adapter@_W@__crt_stdio_output@@V?$standard_base@_WV?$string_output_adapter@_W@__crt_stdio_output@@@2@@__crt_stdio_output@@AAE_NXZ 1000de10 f i libucrt:output.obj
 0001:0000ce73       ?type_case_a@?$output_processor@DV?$string_output_adapter@D@__crt_stdio_output@@V?$standard_base@DV?$string_output_adapter@D@__crt_stdio_output@@@2@@__crt_stdio_output@@AAE_NXZ 1000de73 f i libucrt:output.obj
 0001:0000cfcd       ?type_case_a@?$output_processor@_WV?$string_output_adapter@_W@__crt_stdio_output@@V?$standard_base@_WV?$string_output_adapter@_W@__crt_stdio_output@@@2@@__crt_stdio_output@@AAE_NXZ 1000dfcd f i libucrt:output.obj
 0001:0000d13f       ?type_case_c_tchar@?$output_processor@DV?$string_output_adapter@D@__crt_stdio_output@@V?$standard_base@DV?$string_output_adapter@D@__crt_stdio_output@@@2@@__crt_stdio_output@@AAE_ND@Z 1000e13f f i libucrt:output.obj
 0001:0000d1cf       ?type_case_c_tchar@?$output_processor@_WV?$string_output_adapter@_W@__crt_stdio_output@@V?$standard_base@_WV?$string_output_adapter@_W@__crt_stdio_output@@@2@@__crt_stdio_output@@AAE_N_W@Z 1000e1cf f i libucrt:output.obj
 0001:0000d267       ?type_case_integer@?$output_processor@_WV?$string_output_adapter@_W@__crt_stdio_output@@V?$standard_base@_WV?$string_output_adapter@_W@__crt_stdio_output@@@2@@__crt_stdio_output@@AAE_NI_N@Z 1000e267 f i libucrt:output.obj
 0001:0000d267       ?type_case_integer@?$output_processor@DV?$string_output_adapter@D@__crt_stdio_output@@V?$standard_base@DV?$string_output_adapter@D@__crt_stdio_output@@@2@@__crt_stdio_output@@AAE_NI_N@Z 1000e267 f i libucrt:output.obj
 0001:0000d3b1       ?type_case_n@?$output_processor@_WV?$string_output_adapter@_W@__crt_stdio_output@@V?$standard_base@_WV?$string_output_adapter@_W@__crt_stdio_output@@@2@@__crt_stdio_output@@AAE_NXZ 1000e3b1 f i libucrt:output.obj
 0001:0000d3b1       ?type_case_n@?$output_processor@DV?$string_output_adapter@D@__crt_stdio_output@@V?$standard_base@DV?$string_output_adapter@D@__crt_stdio_output@@@2@@__crt_stdio_output@@AAE_NXZ 1000e3b1 f i libucrt:output.obj
 0001:0000d425       ?type_case_o@?$output_processor@_WV?$string_output_adapter@_W@__crt_stdio_output@@V?$standard_base@_WV?$string_output_adapter@_W@__crt_stdio_output@@@2@@__crt_stdio_output@@AAE_NXZ 1000e425 f i libucrt:output.obj
 0001:0000d425       ?type_case_o@?$output_processor@DV?$string_output_adapter@D@__crt_stdio_output@@V?$standard_base@DV?$string_output_adapter@D@__crt_stdio_output@@@2@@__crt_stdio_output@@AAE_NXZ 1000e425 f i libucrt:output.obj
 0001:0000d444       ?type_case_p@?$output_processor@DV?$string_output_adapter@D@__crt_stdio_output@@V?$standard_base@DV?$string_output_adapter@D@__crt_stdio_output@@@2@@__crt_stdio_output@@AAE_NXZ 1000e444 f i libucrt:output.obj
 0001:0000d444       ?type_case_p@?$output_processor@_WV?$string_output_adapter@_W@__crt_stdio_output@@V?$standard_base@_WV?$string_output_adapter@_W@__crt_stdio_output@@@2@@__crt_stdio_output@@AAE_NXZ 1000e444 f i libucrt:output.obj
 0001:0000d45c       ?type_case_s@?$output_processor@DV?$string_output_adapter@D@__crt_stdio_output@@V?$standard_base@DV?$string_output_adapter@D@__crt_stdio_output@@@2@@__crt_stdio_output@@AAE_NXZ 1000e45c f i libucrt:output.obj
 0001:0000d4cf       ?type_case_s@?$output_processor@_WV?$string_output_adapter@_W@__crt_stdio_output@@V?$standard_base@_WV?$string_output_adapter@_W@__crt_stdio_output@@@2@@__crt_stdio_output@@AAE_NXZ 1000e4cf f i libucrt:output.obj
 0001:0000d543       ?type_case_s_compute_narrow_string_length@?$output_processor@_WV?$string_output_adapter@_W@__crt_stdio_output@@V?$standard_base@_WV?$string_output_adapter@_W@__crt_stdio_output@@@2@@__crt_stdio_output@@ABEHH_W@Z 1000e543 f i libucrt:output.obj
 0001:0000d583       ?write_character@?$string_output_adapter@D@__crt_stdio_output@@QBE_NDQAH@Z 1000e583 f i libucrt:output.obj
 0001:0000d5c5       ?write_character@?$string_output_adapter@_W@__crt_stdio_output@@QBE_N_WQAH@Z 1000e5c5 f i libucrt:output.obj
 0001:0000d60a       ?write_stored_string_tchar@?$output_processor@DV?$string_output_adapter@D@__crt_stdio_output@@V?$standard_base@DV?$string_output_adapter@D@__crt_stdio_output@@@2@@__crt_stdio_output@@AAE_ND@Z 1000e60a f i libucrt:output.obj
 0001:0000d6b1       ?write_stored_string_tchar@?$output_processor@_WV?$string_output_adapter@_W@__crt_stdio_output@@V?$standard_base@_WV?$string_output_adapter@_W@__crt_stdio_output@@@2@@__crt_stdio_output@@AAE_N_W@Z 1000e6b1 f i libucrt:output.obj
 0001:0000d73c       ?write_string@?$string_output_adapter@D@__crt_stdio_output@@QBEXQBDHQAH1@Z 1000e73c f i libucrt:output.obj
 0001:0000d7cf       ?write_string@?$string_output_adapter@_W@__crt_stdio_output@@QBEXQB_WHQAH1@Z 1000e7cf f i libucrt:output.obj
 0001:0000d869       ___stdio_common_vsprintf   1000e869 f   libucrt:output.obj
 0001:0000d88d       ___stdio_common_vswprintf  1000e88d f   libucrt:output.obj
 0001:0000d8b1       _wcsncmp                   1000e8b1 f   libucrt:wcsncmp.obj
 0001:0000d8eb       __initterm                 1000e8eb f   libucrt:initterm.obj
 0001:0000d947       __initterm_e               1000e947 f   libucrt:initterm.obj
 0001:0000d98c       __seh_filter_dll           1000e98c f   libucrt:exception_filter.obj
 0001:0000d9ac       __seh_filter_exe           1000e9ac f   libucrt:exception_filter.obj
 0001:0000dd3a       ___acrt_initialize_thread_local_exit_callback 1000ed3a f   libucrt:exit.obj
 0001:0000dd49       __cexit                    1000ed49 f   libucrt:exit.obj
 0001:0000dd58       __exit                     1000ed58 f   libucrt:exit.obj
 0001:0000dd6e       __is_c_termination_complete 1000ed6e f   libucrt:exit.obj
 0001:0000e00d       ___acrt_allocate_buffer_for_argv 1000f00d f   libucrt:argv_parsing.obj
 0001:0000e062       __configure_narrow_argv    1000f062 f   libucrt:argv_parsing.obj
 0001:0000e1c6       ??$uninitialize@A6AXAAPAPAD@Z@?$dual_state_global@PAPAD@__crt_state_management@@QAEXA6AXAAPAPAD@Z@Z 1000f1c6 f i libucrt:environment_initialization.obj
 0001:0000e1c6       ??$uninitialize@A6AXAAPAPA_W@Z@?$dual_state_global@PAPA_W@__crt_state_management@@QAEXA6AXAAPAPA_W@Z@Z 1000f1c6 f i libucrt:environment_initialization.obj
 0001:0000e23c       ?initialize@?$dual_state_global@P6AXPB_W00II@Z@__crt_state_management@@QAEXQ6AXPB_W00II@Z@Z 1000f23c f i libucrt:invalid_parameter.obj
 0001:0000e23c       ?initialize@?$dual_state_global@P6AHPAU_exception@@@Z@__crt_state_management@@QAEXQ6AHPAU_exception@@@Z@Z 1000f23c f i libucrt:matherr.obj
 0001:0000e23c       ?initialize@?$dual_state_global@PAPAD@__crt_state_management@@QAEXQAPAD@Z 1000f23c f i libucrt:environment_initialization.obj
 0001:0000e23c       ?initialize@?$dual_state_global@P6AXH@Z@__crt_state_management@@QAEXQ6AXH@Z@Z 1000f23c f i libucrt:signal.obj
 0001:0000e23c       ?initialize@?$dual_state_global@P6AHI@Z@__crt_state_management@@QAEXQ6AHI@Z@Z 1000f23c f i libucrt:new_handler.obj
 0001:0000e23c       ?initialize@?$dual_state_global@PAU__crt_locale_data@@@__crt_state_management@@QAEXQAU__crt_locale_data@@@Z 1000f23c f i libucrt:initialization.obj
 0001:0000e26d       ___dcrt_uninitialize_environments_nolock 1000f26d f   libucrt:environment_initialization.obj
 0001:0000e2a4       __initialize_narrow_environment 1000f2a4 f   libucrt:environment_initialization.obj
 0001:0000e2a9       ??$?RV<lambda_800076c951b434888f4765a74a194fcc>@@AAV<lambda_4e60a939b0d047cfe11ddc22648dfba9>@@V<lambda_6dbb1268764f43b569ce7b67e331d33a>@@@?$__crt_seh_guarded_call@H@@QAEH$$QAV<lambda_800076c951b434888f4765a74a194fcc>@@AAV<lambda_4e60a939b0d047cfe11ddc22648dfba9>@@$$QAV<lambda_6dbb1268764f43b569ce7b67e331d33a>@@@Z 1000f2a9 f i libucrt:onexit.obj
 0001:0000e2fa       ??$?RV<lambda_995298e7d72eb4c2aab26c0585b3abe5>@@AAV<lambda_275893d493268fdec8709772e3fcec0e>@@V<lambda_293819299cbf9a7022e18b56a874bb5c>@@@?$__crt_seh_guarded_call@H@@QAEH$$QAV<lambda_995298e7d72eb4c2aab26c0585b3abe5>@@AAV<lambda_275893d493268fdec8709772e3fcec0e>@@$$QAV<lambda_293819299cbf9a7022e18b56a874bb5c>@@@Z 1000f2fa f i libucrt:onexit.obj
 0001:0000e34b       ??$__acrt_lock_and_call@V<lambda_275893d493268fdec8709772e3fcec0e>@@@@YAHW4__acrt_lock_id@@$$QAV<lambda_275893d493268fdec8709772e3fcec0e>@@@Z 1000f34b f i libucrt:onexit.obj
 0001:0000e373       ??$__acrt_lock_and_call@V<lambda_4e60a939b0d047cfe11ddc22648dfba9>@@@@YAHW4__acrt_lock_id@@$$QAV<lambda_4e60a939b0d047cfe11ddc22648dfba9>@@@Z 1000f373 f i libucrt:onexit.obj
 0001:0000e39b       ??$__crt_fast_encode_pointer@P6AHXZ@@YAP6AHXZQ6AHXZ@Z 1000f39b f i libucrt:onexit.obj
 0001:0000e61b       __crt_atexit               1000f61b f   libucrt:onexit.obj
 0001:0000e631       __execute_onexit_table     1000f631 f   libucrt:onexit.obj
 0001:0000e64e       __initialize_onexit_table  1000f64e f   libucrt:onexit.obj
 0001:0000e68b       __register_onexit_function 1000f68b f   libucrt:onexit.obj
 0001:0000e6db       ___acrt_uninitialize_command_line 1000f6db f   libucrt:argv_data.obj
 0001:0000e7a3       ___acrt_initialize         1000f7a3 f   libucrt:initialization.obj
 0001:0000e7b5       ___acrt_thread_attach      1000f7b5 f   libucrt:initialization.obj
 0001:0000e7c0       ___acrt_thread_detach      1000f7c0 f   libucrt:initialization.obj
 0001:0000e7c8       ___acrt_uninitialize       1000f7c8 f   libucrt:initialization.obj
 0001:0000e7da       ___acrt_uninitialize_critical 1000f7da f   libucrt:initialization.obj
 0001:0000e7ec       _terminate                 1000f7ec f   libucrt:terminate.obj
 0001:0000e828       _free                      1000f828 f   libucrt:free.obj
 0001:0000e82d       _malloc                    1000f82d f   libucrt:malloc.obj
 0001:0000e838       _strcpy_s                  1000f838 f   libucrt:strcpy_s.obj
 0001:0000e892       _abort                     1000f892 f   libucrt:abort.obj
 0001:0000e8d5       _calloc                    1000f8d5 f   libucrt:calloc.obj
 0001:0000e8e0       _strncmp                   1000f8e0 f   libucrt:strncmp.obj
 0001:0000e958       ___acrt_call_reportfault   1000f958 f   libucrt:invalid_parameter.obj
 0001:0000ea93       ___acrt_initialize_invalid_parameter_handler 1000fa93 f   libucrt:invalid_parameter.obj
 0001:0000eaa7       __invalid_parameter        1000faa7 f   libucrt:invalid_parameter.obj
 0001:0000eb22       __invalid_parameter_noinfo 1000fb22 f   libucrt:invalid_parameter.obj
 0001:0000eb32       __invoke_watson            1000fb32 f   libucrt:invalid_parameter.obj
 0001:0000eb65       ___acrt_errno_from_os_error 1000fb65 f   libucrt:errno.obj
 0001:0000eba8       ___acrt_errno_map_os_error 1000fba8 f   libucrt:errno.obj
 0001:0000ebcb       ___doserrno                1000fbcb f   libucrt:errno.obj
 0001:0000ebde       __errno                    1000fbde f   libucrt:errno.obj
 0001:0000ebf1       ___pctype_func             1000fbf1 f   libucrt:ctype.obj
 0001:0000ec17       _iswctype                  1000fc17 f   libucrt:iswctype.obj
 0001:0000ec76       __isctype_l                1000fc76 f   libucrt:isctype.obj
 0001:0000ed48       ??$?RV<lambda_3518db117f0e7cdb002338c5d3c47b6c>@@AAV<lambda_b2ea41f6bbb362cd97d94c6828d90b61>@@V<lambda_abdedf541bb04549bc734292b4a045d4>@@@?$__crt_seh_guarded_call@X@@QAEX$$QAV<lambda_3518db117f0e7cdb002338c5d3c47b6c>@@AAV<lambda_b2ea41f6bbb362cd97d94c6828d90b61>@@$$QAV<lambda_abdedf541bb04549bc734292b4a045d4>@@@Z 1000fd48 f i libucrt:per_thread_data.obj
 0001:0000ed98       ??$?RV<lambda_51b6e8b1eb166f2a3faf91f424b38130>@@AAV<lambda_6250bd4b2a391816dd638c3bf72b0bcb>@@V<lambda_0b5a4a3e68152e1d9b943535f5f47bed>@@@?$__crt_seh_guarded_call@X@@QAEX$$QAV<lambda_51b6e8b1eb166f2a3faf91f424b38130>@@AAV<lambda_6250bd4b2a391816dd638c3bf72b0bcb>@@$$QAV<lambda_0b5a4a3e68152e1d9b943535f5f47bed>@@@Z 1000fd98 f i libucrt:per_thread_data.obj
 0001:0000edf9       ??$?RV<lambda_5b71d36f03204c0beab531769a5b5694>@@AAV<lambda_be2b3da3f62db62e9dad5dc70221a656>@@V<lambda_8f9ce462984622f9bf76b59e2aaaf805>@@@?$__crt_seh_guarded_call@X@@QAEX$$QAV<lambda_5b71d36f03204c0beab531769a5b5694>@@AAV<lambda_be2b3da3f62db62e9dad5dc70221a656>@@$$QAV<lambda_8f9ce462984622f9bf76b59e2aaaf805>@@@Z 1000fdf9 f i libucrt:per_thread_data.obj
 0001:0000ee44       ??$?RV<lambda_9df27f884b057bc3edfc946cb5b7cf47>@@AAV<lambda_e69574bed617af4e071282c136b37893>@@V<lambda_cc0d902bcbbeb830f749456577db4721>@@@?$__crt_seh_guarded_call@X@@QAEX$$QAV<lambda_9df27f884b057bc3edfc946cb5b7cf47>@@AAV<lambda_e69574bed617af4e071282c136b37893>@@$$QAV<lambda_cc0d902bcbbeb830f749456577db4721>@@@Z 1000fe44 f i libucrt:per_thread_data.obj
 0001:0000ee8c       ??$__acrt_lock_and_call@V<lambda_6250bd4b2a391816dd638c3bf72b0bcb>@@@@YAXW4__acrt_lock_id@@$$QAV<lambda_6250bd4b2a391816dd638c3bf72b0bcb>@@@Z 1000fe8c f i libucrt:per_thread_data.obj
 0001:0000eeb4       ??$__acrt_lock_and_call@V<lambda_b2ea41f6bbb362cd97d94c6828d90b61>@@@@YAXW4__acrt_lock_id@@$$QAV<lambda_b2ea41f6bbb362cd97d94c6828d90b61>@@@Z 1000feb4 f i libucrt:per_thread_data.obj
 0001:0000eedc       ??$__acrt_lock_and_call@V<lambda_be2b3da3f62db62e9dad5dc70221a656>@@@@YAXW4__acrt_lock_id@@$$QAV<lambda_be2b3da3f62db62e9dad5dc70221a656>@@@Z 1000fedc f i libucrt:per_thread_data.obj
 0001:0000ef04       ??$__acrt_lock_and_call@V<lambda_e69574bed617af4e071282c136b37893>@@@@YAXW4__acrt_lock_id@@$$QAV<lambda_e69574bed617af4e071282c136b37893>@@@Z 1000ff04 f i libucrt:per_thread_data.obj
 0001:0000f0ba       ___acrt_freeptd            100100ba f   libucrt:per_thread_data.obj
 0001:0000f0e6       ___acrt_getptd             100100e6 f   libucrt:per_thread_data.obj
 0001:0000f16a       ___acrt_getptd_noexit      1001016a f   libucrt:per_thread_data.obj
 0001:0000f1ef       ___acrt_initialize_ptd     100101ef f   libucrt:per_thread_data.obj
 0001:0000f21b       ___acrt_uninitialize_ptd   1001021b f   libucrt:per_thread_data.obj
 0001:0000f235       ___acrt_update_locale_info 10010235 f   libucrt:locale_update.obj
 0001:0000f262       ___acrt_update_multibyte_info 10010262 f   libucrt:locale_update.obj
 0001:0000f28f       ___acrt_set_locale_changed 1001028f f   libucrt:wsetlocale.obj
 0001:0000f29a       ___acrt_uninitialize_locale 1001029a f   libucrt:wsetlocale.obj
 0001:0000f2ec       __isdigit_l                100102ec f i libucrt:_ctype.obj
 0001:0000f324       _isdigit                   10010324 f i libucrt:_ctype.obj
 0001:0000f4b8       __tolower_l                100104b8 f   libucrt:tolower_toupper.obj
 0001:0000f4d2       _tolower                   100104d2 f   libucrt:tolower_toupper.obj
 0001:0000f502       __free_base                10010502 f   libucrt:free_base.obj
 0001:0000f53c       __malloc_base              1001053c f   libucrt:malloc_base.obj
 0001:0000f58a       __mbtowc_l                 1001058a f   libucrt:mbtowc.obj
 0001:0000f684       _mbtowc                    10010684 f   libucrt:mbtowc.obj
 0001:0000f69e       __wctomb_s_l               1001069e f   libucrt:wctomb.obj
 0001:0000f7bf       _wctomb_s                  100107bf f   libucrt:wctomb.obj
 0001:0000f7dc       _strnlen                   100107dc f   libucrt:strnlen.obj
 0001:0000f903       _wcsnlen                   10010903 f   libucrt:strnlen.obj
 0001:0000faba       ?__acrt_fp_classify@@YA?AW4__acrt_fp_class@@ABN@Z 10010aba f i libucrt:cvt.obj
 0001:0000fb26       ?__acrt_fp_is_negative@@YA_NABN@Z 10010b26 f i libucrt:cvt.obj
 0001:00010385       ___acrt_fp_format          10011385 f   libucrt:cvt.obj
 0001:000104cf       __fileno                   100114cf f   libucrt:fileno.obj
 0001:000104f5       ___acrt_initialize_stdio   100114f5 f   libucrt:_file.obj
 0001:000105bd       ___acrt_uninitialize_stdio 100115bd f   libucrt:_file.obj
 0001:00010609       __lock_file                10011609 f   libucrt:_file.obj
 0001:0001061d       __unlock_file              1001161d f   libucrt:_file.obj
 0001:00010631       __get_printf_count_output  10011631 f   libucrt:printf_count_output.obj
 0001:000107b2       ___acrt_initialize_lowio   100117b2 f   libucrt:ioinit.obj
 0001:00010808       ___acrt_uninitialize_lowio 10011808 f   libucrt:ioinit.obj
 0001:00010834       ___acrt_initialize_locks   10011834 f   libucrt:locks.obj
 0001:00010875       ___acrt_lock               10011875 f   libucrt:locks.obj
 0001:0001088c       ___acrt_uninitialize_locks 1001188c f   libucrt:locks.obj
 0001:000108bd       ___acrt_unlock             100118bd f   libucrt:locks.obj
 0001:000109eb       ___acrt_FlsAlloc@4         100119eb f   libucrt:winapi_thunks.obj
 0001:00010a41       ___acrt_FlsFree@4          10011a41 f   libucrt:winapi_thunks.obj
 0001:00010a97       ___acrt_FlsGetValue@4      10011a97 f   libucrt:winapi_thunks.obj
 0001:00010aed       ___acrt_FlsSetValue@8      10011aed f   libucrt:winapi_thunks.obj
 0001:00010b46       ___acrt_InitializeCriticalSectionEx@12 10011b46 f   libucrt:winapi_thunks.obj
 0001:00010ba8       ___acrt_LCMapStringEx@36   10011ba8 f   libucrt:winapi_thunks.obj
 0001:00010c30       ___acrt_LocaleNameToLCID@8 10011c30 f   libucrt:winapi_thunks.obj
 0001:00010c8c       ___acrt_initialize_winapi_thunks 10011c8c f   libucrt:winapi_thunks.obj
 0001:00010cb2       ___acrt_is_packaged_app    10011cb2 f   libucrt:winapi_thunks.obj
 0001:00010d39       ___acrt_uninitialize_winapi_thunks 10011d39 f   libucrt:winapi_thunks.obj
 0001:00010d6f       __calloc_base              10011d6f f   libucrt:calloc_base.obj
 0001:0001118e       ??1?$argument_list@D@?A0xb0e4b824@@QAE@XZ 1001218e f i libucrt:argv_wildcards.obj
 0001:000111b3       ?append@?$argument_list@D@?A0xb0e4b824@@QAEHQAD@Z 100121b3 f i libucrt:argv_wildcards.obj
 0001:000111e8       ?expand_if_necessary@?$argument_list@D@?A0xb0e4b824@@AAEHXZ 100121e8 f i libucrt:argv_wildcards.obj
 0001:0001126f       ___acrt_expand_narrow_argv_wildcards 1001226f f   libucrt:argv_wildcards.obj
 0001:0001127a       ??$?RV<lambda_978dc153c237d78434369da87b74ff60>@@AAV<lambda_ad1ced32f4ac17aa236e5ef05d6b3b7c>@@V<lambda_4a8533e2866a575feecb8298ce776b0d>@@@?$__crt_seh_guarded_call@X@@QAEX$$QAV<lambda_978dc153c237d78434369da87b74ff60>@@AAV<lambda_ad1ced32f4ac17aa236e5ef05d6b3b7c>@@$$QAV<lambda_4a8533e2866a575feecb8298ce776b0d>@@@Z 1001227a f i libucrt:mbctype.obj
 0001:000112bd       ??$__acrt_lock_and_call@V<lambda_ad1ced32f4ac17aa236e5ef05d6b3b7c>@@@@YAXW4__acrt_lock_id@@$$QAV<lambda_ad1ced32f4ac17aa236e5ef05d6b3b7c>@@@Z 100122bd f i libucrt:mbctype.obj
 0001:00011754       ___acrt_initialize_multibyte 10012754 f   libucrt:mbctype.obj
 0001:00011772       ___acrt_update_thread_multibyte_data 10012772 f   libucrt:mbctype.obj
 0001:00011814       __setmbcp_nolock           10012814 f   libucrt:mbctype.obj
 0001:00011adf       __ismbblead                10012adf f   libucrt:ismbbyte.obj
 0001:00011af7       ___acrt_initialize_command_line 10012af7 f   libucrt:argv_data.obj
 0001:00011b47       ___dcrt_get_narrow_environment_from_os 10012b47 f   libucrt:get_environment_from_os.obj
 0001:00011bca       __recalloc                 10012bca f   libucrt:recalloc.obj
 0001:00011bd5       __recalloc_base            10012bd5 f   libucrt:recalloc.obj
 0001:00011c42       ___acrt_initialize_heap    10012c42 f   libucrt:heap_handle.obj
 0001:00011c53       ___acrt_uninitialize_heap  10012c53 f   libucrt:heap_handle.obj
 0001:00011c5d       ___acrt_execute_initializers 10012c5d f   libucrt:shared_initialization.obj
 0001:00011ce0       ___acrt_execute_uninitializers 10012ce0 f   libucrt:shared_initialization.obj
 0001:00011d2d       ___acrt_initialize_new_handler 10012d2d f   libucrt:new_handler.obj
 0001:00011d41       __callnewh                 10012d41 f   libucrt:new_handler.obj
 0001:00011d85       __query_new_handler        10012d85 f   libucrt:new_handler.obj
 0001:00011dd7       ??$?RV<lambda_a048d3beccc847880fc8490e18b82769>@@AAV<lambda_ec61778202f4f5fc7e7711acc23c3bca>@@V<lambda_f7496a158712204296dd6628a163878e>@@@?$__crt_seh_guarded_call@P6AXH@Z@@QAEP6AXH@Z$$QAV<lambda_a048d3beccc847880fc8490e18b82769>@@AAV<lambda_ec61778202f4f5fc7e7711acc23c3bca>@@$$QAV<lambda_f7496a158712204296dd6628a163878e>@@@Z 10012dd7 f i libucrt:signal.obj
 0001:00011e31       ??$__acrt_lock_and_call@V<lambda_ec61778202f4f5fc7e7711acc23c3bca>@@@@YAP6AXH@ZW4__acrt_lock_id@@$$QAV<lambda_ec61778202f4f5fc7e7711acc23c3bca>@@@Z 10012e31 f i libucrt:signal.obj
 0001:00011ec3       ___acrt_get_sigabrt_handler 10012ec3 f   libucrt:signal.obj
 0001:00011eda       ___acrt_initialize_signal_handlers 10012eda f   libucrt:signal.obj
 0001:00011f15       ___fpecode                 10012f15 f   libucrt:signal.obj
 0001:00011f1e       _raise                     10012f1e f   libucrt:signal.obj
 0001:00012126       ___acrt_has_user_matherr   10013126 f   libucrt:matherr.obj
 0001:0001213f       ___acrt_initialize_user_matherr 1001313f f   libucrt:matherr.obj
 0001:00012153       ___acrt_invoke_user_matherr 10013153 f   libucrt:matherr.obj
 0001:0001219c       __isleadbyte_l             1001319c f i libucrt:_wctype.obj
 0001:000121d5       ___acrt_GetStringTypeA     100131d5 f   libucrt:getstringtypea.obj
 0001:000122f2       __freea_crt                100132f2 f i libucrt:getstringtypea.obj
 0001:00012312       ___acrt_add_locale_ref     10013312 f   libucrt:locale_refcounting.obj
 0001:0001238f       ___acrt_free_locale        1001338f f   libucrt:locale_refcounting.obj
 0001:000124d9       ___acrt_locale_add_lc_time_reference 100134d9 f   libucrt:locale_refcounting.obj
 0001:00012502       ___acrt_locale_free_lc_time_if_unreferenced 10013502 f   libucrt:locale_refcounting.obj
 0001:00012532       ___acrt_locale_release_lc_time_reference 10013532 f   libucrt:locale_refcounting.obj
 0001:0001255b       ___acrt_release_locale_ref 1001355b f   libucrt:locale_refcounting.obj
 0001:000125dc       ___acrt_update_thread_locale_data 100135dc f   libucrt:locale_refcounting.obj
 0001:00012653       __updatetlocinfoEx_nolock  10013653 f   libucrt:locale_refcounting.obj
 0001:000126a3       ___acrt_locale_free_monetary 100136a3 f   libucrt:initmon.obj
 0001:000127a1       ___acrt_locale_free_numeric 100137a1 f   libucrt:initnum.obj
 0001:00012846       ___acrt_locale_free_time   10013846 f   libucrt:inittime.obj
 0001:00012b47       ___acrt_LCMapStringA       10013b47 f   libucrt:lcmapstringa.obj
 0001:00012b92       __query_new_mode           10013b92 f   libucrt:new_mode.obj
 0001:00012b98       ___acrt_fp_strflt_to_string 10013b98 f   libucrt:_fptostr.obj
 0001:00012c54       ??0scoped_fp_state_reset@?A0x48fbfdd4@@QAE@XZ 10013c54 f i libucrt:cfout.obj
 0001:00012c80       ?divide@__crt_strtox@@YA_KAAUbig_integer@1@ABU21@@Z 10013c80 f i libucrt:cfout.obj
 0001:0001312e       ___acrt_fltout             1001412e f   libucrt:cfout.obj
 0001:000144ca       __fcloseall                100154ca f   libucrt:closeall.obj
 0001:0001456a       ___acrt_stdio_flush_nolock 1001556a f   libucrt:fflush.obj
 0001:000145d0       __fflush_nolock            100155d0 f   libucrt:fflush.obj
 0001:00014617       __flushall                 10015617 f   libucrt:fflush.obj
 0001:000146f8       ___acrt_stdio_free_buffer_nolock 100156f8 f   libucrt:_freebuf.obj
 0001:00014736       __isatty                   10015736 f   libucrt:isatty.obj
 0001:0001478c       ___acrt_lowio_create_handle_array 1001578c f   libucrt:osfinfo.obj
 0001:00014806       ___acrt_lowio_destroy_handle_array 10015806 f   libucrt:osfinfo.obj
 0001:0001483b       ___acrt_lowio_ensure_fh_exists 1001583b f   libucrt:osfinfo.obj
 0001:000148d3       ___acrt_lowio_lock_fh      100158d3 f   libucrt:osfinfo.obj
 0001:000148f6       ___acrt_lowio_unlock_fh    100158f6 f   libucrt:osfinfo.obj
 0001:00014919       __free_osfhnd              10015919 f   libucrt:osfinfo.obj
 0001:000149aa       __get_osfhandle            100159aa f   libucrt:osfinfo.obj
 0001:00014ad0       ___acrt_DownlevelLocaleNameToLCID 10015ad0 f   libucrt:lcidtoname_downlevel.obj
 0001:00014be0       _qsort                     10015be0 f   libucrt:qsort.obj
 0001:0001502b       _strncpy_s                 1001602b f   libucrt:strncpy_s.obj
 0001:00015040       _strpbrk                   10016040 f   libucrt:strpbrk.obj
 0001:00015080       __mbsdec                   10016080 f   libucrt:mbsdec.obj
 0001:00015097       __mbsdec_l                 10016097 f   libucrt:mbsdec.obj
 0001:00015133       __msize                    10016133 f   libucrt:msize.obj
 0001:00015166       __realloc_base             10016166 f   libucrt:realloc_base.obj
 0001:000151cf       ___strncnt                 100161cf f   libucrt:strncnt.obj
 0001:000151eb       _fegetenv                  100161eb f   libucrt:fegetenv.obj
 0001:00015208       _fesetenv                  10016208 f   libucrt:fesetenv.obj
 0001:00015251       _feholdexcept              10016251 f   libucrt:feholdexcept.obj
 0001:000152a0       _log10                     100162a0 f   libucrt:log10.obj
 0001:000152e0       __CIlog10                  100162e0 f   libucrt:log10.obj
 0001:0001531b       __CIlog10_default          1001631b f   libucrt:log10.obj
 0001:0001532f       __log10_default            1001632f     libucrt:log10.obj
 0001:000153f0       _ceil                      100163f0 f   libucrt:ceil_pentium4.obj
 0001:00015430       __ceil_pentium4            10016430 f   libucrt:ceil_pentium4.obj
 0001:00015a9d       __write                    10016a9d f   libucrt:write.obj
 0001:00015b88       __write_nolock             10016b88 f   libucrt:write.obj
 0001:00015e12       __lseeki64_nolock          10016e12 f   libucrt:lseek.obj
 0001:00015e2d       __fclose_nolock            10016e2d f   libucrt:fclose.obj
 0001:00015ea3       _fclose                    10016ea3 f   libucrt:fclose.obj
 0001:00015f23       ??$?RV<lambda_61cee617f5178ae960314fd4d05640a0>@@AAV<lambda_6978c1fb23f02e42e1d9e99668cc68aa>@@V<lambda_9cd88cf8ad10232537feb2133f08c833>@@@?$__crt_seh_guarded_call@H@@QAEH$$QAV<lambda_61cee617f5178ae960314fd4d05640a0>@@AAV<lambda_6978c1fb23f02e42e1d9e99668cc68aa>@@$$QAV<lambda_9cd88cf8ad10232537feb2133f08c833>@@@Z 10016f23 f i libucrt:commit.obj
 0001:00015fbb       ??$__acrt_lowio_lock_fh_and_call@V<lambda_6978c1fb23f02e42e1d9e99668cc68aa>@@@@YAHH$$QAV<lambda_6978c1fb23f02e42e1d9e99668cc68aa>@@@Z 10016fbb f i libucrt:commit.obj
 0001:00015fe3       __commit                   10016fe3 f   libucrt:commit.obj
 0001:00016052       __query_app_type           10017052 f   libucrt:report_runtime_error.obj
 0001:000162fb       __getfpcontrolword         100172fb f   libucrt:_fenvutils.obj
 0001:0001633e       __getfpstatusword          1001733e f   libucrt:_fenvutils.obj
 0001:000163e6       __setfpcontrolword         100173e6 f   libucrt:_fenvutils.obj
 0001:00016466       __setfpstatusword          10017466 f   libucrt:_fenvutils.obj
 0001:000164e6       __clearfp                  100174e6 f   libucrt:ieee87.obj
 0001:000165c4       ___acrt_initialize_sse2    100175c4 f   libucrt:mathfcns.obj
 0001:000165e0       __CIlog10_pentium4         100175e0 f   libucrt:log10_pentium4.obj
 0001:000165f8       __log10_pentium4           100175f8     libucrt:log10_pentium4.obj
 0001:00016881       __fFEXP                    10017881     libucrt:87tran.obj
 0001:000168d8       __rtinfpopse               100178d8     libucrt:87tran.obj
 0001:000168da       __rtinfnpopse              100178da     libucrt:87tran.obj
 0001:000168ea       __fFLN                     100178ea     libucrt:87tran.obj
 0001:0001699f       __rtinfpop                 1001799f     libucrt:87tran.obj
 0001:000169a1       __rtinfnpop                100179a1     libucrt:87tran.obj
 0001:000169be       __ffexpm1                  100179be     libucrt:87tran.obj
 0001:00016a70       __trandisp1                10017a70 f   libucrt:87disp.obj
 0001:00016ad7       __trandisp2                10017ad7 f   libucrt:87disp.obj
 0001:00016b63       __rttospopde               10017b63     libucrt:87disp.obj
 0001:00016b68       __rttospop                 10017b68     libucrt:87disp.obj
 0001:00016b6a       __rtnospop                 10017b6a     libucrt:87disp.obj
 0001:00016b6c       __rttosnpop                10017b6c     libucrt:87disp.obj
 0001:00016b6d       __rtnospopde               10017b6d     libucrt:87disp.obj
 0001:00016b74       __rtzeropop                10017b74     libucrt:87disp.obj
 0001:00016b76       __rtzeronpop               10017b76     libucrt:87disp.obj
 0001:00016b7b       __rtzerospop               10017b7b     libucrt:87disp.obj
 0001:00016b88       __rtonepop                 10017b88     libucrt:87disp.obj
 0001:00016b8a       __rtonenpop                10017b8a     libucrt:87disp.obj
 0001:00016b8f       __tosnan1                  10017b8f     libucrt:87disp.obj
 0001:00016bba       __nosnan2                  10017bba     libucrt:87disp.obj
 0001:00016bbc       __tosnan2                  10017bbc     libucrt:87disp.obj
 0001:00016be4       __nan2                     10017be4     libucrt:87disp.obj
 0001:00016c23       __rtindfpop                10017c23     libucrt:87disp.obj
 0001:00016c25       __rtindfnpop               10017c25     libucrt:87disp.obj
 0001:00016c36       __rttosnpopde              10017c36     libucrt:87disp.obj
 0001:00016c40       __rtatan2inf               10017c40     libucrt:87disp.obj
 0001:00016c5d       __rtchsifneg               10017c5d     libucrt:87disp.obj
 0001:00016c70       __twoToTOS                 10017c70 f   libucrt:common.obj
 0001:00016c85       __load_CW                  10017c85 f   libucrt:common.obj
 0001:00016c9c       __convertTOStoQNaN         10017c9c f   libucrt:common.obj
 0001:00016cb5       __fload_withFB             10017cb5 f   libucrt:common.obj
 0001:00016cf8       __checkTOS_withFB          10017cf8 f   libucrt:common.obj
 0001:00016d0e       __fast_exit                10017d0e f   libucrt:common.obj
 0001:00016d1b       __math_exit                10017d1b f   libucrt:common.obj
 0001:00016d45       __check_overflow_exit      10017d45 f   libucrt:common.obj
 0001:00016d59       __check_range_exit         10017d59 f   libucrt:common.obj
 0001:00016e00       __startTwoArgErrorHandling 10017e00 f   libucrt:genexcep.obj
 0001:00016e17       __startOneArgErrorHandling 10017e17 f   libucrt:genexcep.obj
 0001:00016e56       ___libm_error_support      10017e56 f   libucrt:libm_error.obj
 0001:0001706e       __ceil_default             1001806e f   libucrt:ceil.obj
 0001:00017127       __putwch_nolock            10018127 f   libucrt:putwch.obj
 0001:0001716c       ??$?RV<lambda_123407a5e2ac06da108355a851863b7a>@@AAV<lambda_2fe9b910cf3cbf4a0ab98a02ba45b3ec>@@V<lambda_ae55bdf541ad94d75914d381c370e64d>@@@?$__crt_seh_guarded_call@H@@QAEH$$QAV<lambda_123407a5e2ac06da108355a851863b7a>@@AAV<lambda_2fe9b910cf3cbf4a0ab98a02ba45b3ec>@@$$QAV<lambda_ae55bdf541ad94d75914d381c370e64d>@@@Z 1001816c f i libucrt:close.obj
 0001:000171ee       ??$__acrt_lowio_lock_fh_and_call@V<lambda_2fe9b910cf3cbf4a0ab98a02ba45b3ec>@@@@YAHH$$QAV<lambda_2fe9b910cf3cbf4a0ab98a02ba45b3ec>@@@Z 100181ee f i libucrt:close.obj
 0001:00017216       __close                    10018216 f   libucrt:close.obj
 0001:00017295       __close_nolock             10018295 f   libucrt:close.obj
 0001:00017331       ?__acrt_stdio_free_stream@@YAXV__crt_stdio_stream@@@Z 10018331 f   libucrt:stream.obj
 0001:00017370       ___ascii_strnicmp          10018370 f   libucrt:_strnicm.obj
 0001:000173d1       __clrfp                    100183d1 f   libucrt:fpctrl.obj
 0001:000173e4       __ctrlfp                   100183e4 f   libucrt:fpctrl.obj
 0001:00017410       __set_statfp               10018410 f   libucrt:fpctrl.obj
 0001:0001746b       __statfp                   1001846b f   libucrt:fpctrl.obj
 0001:0001747d       __d_inttype                1001847d f   libucrt:powhlp.obj
 0001:000174e7       __powhlp                   100184e7 f   libucrt:powhlp.obj
 0001:00017612       __87except                 10018612 f   libucrt:87except.obj
 0001:0001771d       __frnd                     1001871d f   libucrt:frnd.obj
 0001:00017733       __errcode                  10018733 f   libucrt:fpexcept.obj
 0001:00017767       __except1                  10018767 f   libucrt:fpexcept.obj
 0001:00017835       __handle_exc               10018835 f   libucrt:fpexcept.obj
 0001:00017a15       __raise_exc                10018a15 f   libucrt:fpexcept.obj
 0001:00017a38       __raise_exc_ex             10018a38 f   libucrt:fpexcept.obj
 0001:00017d29       __set_errno_from_matherr   10018d29 f   libucrt:fpexcept.obj
 0001:00017d58       __umatherr                 10018d58 f   libucrt:fpexcept.obj
 0001:00017dfa       __decomp                   10018dfa f   libucrt:util.obj
 0001:00017ece       __set_exp                  10018ece f   libucrt:util.obj
 0001:00017efd       __sptype                   10018efd f   libucrt:util.obj
 0001:00017f5b       ___dcrt_lowio_initialize_console_output 10018f5b f   libucrt:initcon.obj
 0001:00017f7a       ___dcrt_terminate_console_output 10018f7a f   libucrt:initcon.obj
 0001:00017f91       __fpclass                  10018f91 f   libucrt:ieeemisc.obj
 0001:00018035       _IsProcessorFeaturePresent@4 10019035 f   kernel32:KERNEL32.dll
 0001:00018040       __FindPESection            10019040 f   LIBCMT:pesect.obj
 0001:00018090       __IsNonwritableInCurrentImage 10019090 f   LIBCMT:pesect.obj
 0001:00018150       __ValidateImageBase        10019150 f   LIBCMT:pesect.obj
 0001:00018190       __aulldvrm                 10019190 f   LIBCMT:ulldvrm.obj
 0001:00018230       __SEH_prolog4_GS           10019230 f   LIBCMT:_sehprolg4gs_.obj
 0001:00018279       __SEH_epilog4_GS           10019279 f   LIBCMT:_sehprolg4gs_.obj
 0001:00018290       __alldvrm                  10019290 f   LIBCMT:lldvrm.obj
 0001:00018370       __aullshr                  10019370 f   LIBCMT:ullshr.obj
 0001:00018390       __alloca_probe_16          10019390 f   LIBCMT:alloca16.obj
 0001:000183a6       __alloca_probe_8           100193a6     LIBCMT:alloca16.obj
 0001:000183c0       __allshl                   100193c0 f   LIBCMT:llshl.obj
 0001:000183e0       __ftol2_sse                100193e0 f   LIBCMT:_ftol2_.obj
 0001:000183e9       __ftol2_pentium4           100193e9 f   LIBCMT:_ftol2_.obj
 0001:000183fc       __ftol2_sse_excpt          100193fc f   LIBCMT:_ftol2_.obj
 0001:00018420       __ftol2                    10019420 f   LIBCMT:_ftol2_.obj
 0001:000184a0       __chkstk                   100194a0 f   LIBCMT:chkstk.obj
 0001:000184a0       __alloca_probe             100194a0 f   LIBCMT:chkstk.obj
 0002:00000000       __imp__RegQueryValueExW@24 1001a000     advapi32:ADVAPI32.dll
 0002:00000004       __imp__RegOpenKeyExW@20    1001a004     advapi32:ADVAPI32.dll
 0002:00000008       __imp__RegCreateKeyExW@36  1001a008     advapi32:ADVAPI32.dll
 0002:0000000c       __imp__RegCloseKey@4       1001a00c     advapi32:ADVAPI32.dll
 0002:00000010       __imp__RegSetValueExW@24   1001a010     advapi32:ADVAPI32.dll
 0002:00000014       \177ADVAPI32_NULL_THUNK_DATA 1001a014     advapi32:ADVAPI32.dll
 0002:00000018       __imp__SetTextColor@8      1001a018     gdi32:GDI32.dll
 0002:0000001c       __imp__StretchBlt@44       1001a01c     gdi32:GDI32.dll
 0002:00000020       __imp__SetBkMode@8         1001a020     gdi32:GDI32.dll
 0002:00000024       __imp__SelectObject@8      1001a024     gdi32:GDI32.dll
 0002:00000028       __imp__DeleteObject@4      1001a028     gdi32:GDI32.dll
 0002:0000002c       __imp__DeleteDC@4          1001a02c     gdi32:GDI32.dll
 0002:00000030       __imp__CreateSolidBrush@4  1001a030     gdi32:GDI32.dll
 0002:00000034       __imp__CreateFontIndirectW@4 1001a034     gdi32:GDI32.dll
 0002:00000038       __imp__CreateCompatibleDC@4 1001a038     gdi32:GDI32.dll
 0002:0000003c       __imp__CreateCompatibleBitmap@12 1001a03c     gdi32:GDI32.dll
 0002:00000040       __imp__BitBlt@36           1001a040     gdi32:GDI32.dll
 0002:00000044       \177GDI32_NULL_THUNK_DATA  1001a044     gdi32:GDI32.dll
 0002:00000048       __imp__GetLocalTime@4      1001a048     kernel32:KERNEL32.dll
 0002:0000004c       __imp__SystemTimeToFileTime@8 1001a04c     kernel32:KERNEL32.dll
 0002:00000050       __imp__lstrcmpW@8          1001a050     kernel32:KERNEL32.dll
 0002:00000054       __imp__lstrcmpiW@8         1001a054     kernel32:KERNEL32.dll
 0002:00000058       __imp__lstrcpynW@12        1001a058     kernel32:KERNEL32.dll
 0002:0000005c       __imp__lstrcpyW@8          1001a05c     kernel32:KERNEL32.dll
 0002:00000060       __imp__lstrlenW@4          1001a060     kernel32:KERNEL32.dll
 0002:00000064       __imp__LoadLibraryW@4      1001a064     kernel32:KERNEL32.dll
 0002:00000068       __imp__GetModuleFileNameW@12 1001a068     kernel32:KERNEL32.dll
 0002:0000006c       __imp__ExpandEnvironmentStringsW@12 1001a06c     kernel32:KERNEL32.dll
 0002:00000070       __imp__OutputDebugStringW@4 1001a070     kernel32:KERNEL32.dll
 0002:00000074       __imp__GetDriveTypeW@4     1001a074     kernel32:KERNEL32.dll
 0002:00000078       __imp__GetTempPathW@8      1001a078     kernel32:KERNEL32.dll
 0002:0000007c       __imp__GetDiskFreeSpaceExW@16 1001a07c     kernel32:KERNEL32.dll
 0002:00000080       __imp__CreateFileW@28      1001a080     kernel32:KERNEL32.dll
 0002:00000084       __imp__FindFirstChangeNotificationW@12 1001a084     kernel32:KERNEL32.dll
 0002:00000088       __imp__CloseHandle@4       1001a088     kernel32:KERNEL32.dll
 0002:0000008c       __imp__FindCloseChangeNotification@4 1001a08c     kernel32:KERNEL32.dll
 0002:00000090       __imp__WideCharToMultiByte@32 1001a090     kernel32:KERNEL32.dll
 0002:00000094       __imp__ReadConsoleOutputW@20 1001a094     kernel32:KERNEL32.dll
 0002:00000098       __imp__GetConsoleScreenBufferInfo@8 1001a098     kernel32:KERNEL32.dll
 0002:0000009c       __imp__lstrcpynA@12        1001a09c     kernel32:KERNEL32.dll
 0002:000000a0       __imp__lstrcpyA@8          1001a0a0     kernel32:KERNEL32.dll
 0002:000000a4       __imp__lstrlenA@4          1001a0a4     kernel32:KERNEL32.dll
 0002:000000a8       __imp__MultiByteToWideChar@24 1001a0a8     kernel32:KERNEL32.dll
 0002:000000ac       __imp__SetFilePointerEx@20 1001a0ac     kernel32:KERNEL32.dll
 0002:000000b0       __imp__GetConsoleMode@8    1001a0b0     kernel32:KERNEL32.dll
 0002:000000b4       __imp__GetConsoleCP@0      1001a0b4     kernel32:KERNEL32.dll
 0002:000000b8       __imp__WriteFile@20        1001a0b8     kernel32:KERNEL32.dll
 0002:000000bc       __imp__HeapSize@12         1001a0bc     kernel32:KERNEL32.dll
 0002:000000c0       __imp__SetStdHandle@8      1001a0c0     kernel32:KERNEL32.dll
 0002:000000c4       __imp__ReadFile@20         1001a0c4     kernel32:KERNEL32.dll
 0002:000000c8       __imp__GetStdHandle@4      1001a0c8     kernel32:KERNEL32.dll
 0002:000000cc       __imp__GetFileInformationByHandle@8 1001a0cc     kernel32:KERNEL32.dll
 0002:000000d0       __imp__WaitForSingleObject@8 1001a0d0     kernel32:KERNEL32.dll
 0002:000000d4       __imp__GetLastError@0      1001a0d4     kernel32:KERNEL32.dll
 0002:000000d8       __imp__GetCurrentProcessId@0 1001a0d8     kernel32:KERNEL32.dll
 0002:000000dc       __imp__GetProcessHeap@0    1001a0dc     kernel32:KERNEL32.dll
 0002:000000e0       __imp__HeapFree@12         1001a0e0     kernel32:KERNEL32.dll
 0002:000000e4       __imp__HeapReAlloc@16      1001a0e4     kernel32:KERNEL32.dll
 0002:000000e8       __imp__HeapAlloc@12        1001a0e8     kernel32:KERNEL32.dll
 0002:000000ec       __imp__GetProcAddress@8    1001a0ec     kernel32:KERNEL32.dll
 0002:000000f0       __imp__VirtualProtect@16   1001a0f0     kernel32:KERNEL32.dll
 0002:000000f4       __imp__FreeLibrary@4       1001a0f4     kernel32:KERNEL32.dll
 0002:000000f8       __imp__FlushFileBuffers@4  1001a0f8     kernel32:KERNEL32.dll
 0002:000000fc       __imp__DecodePointer@4     1001a0fc     kernel32:KERNEL32.dll
 0002:00000100       __imp__WriteConsoleW@20    1001a100     kernel32:KERNEL32.dll
 0002:00000104       __imp__FindNextChangeNotification@4 1001a104     kernel32:KERNEL32.dll
 0002:00000108       __imp__InitializeCriticalSection@4 1001a108     kernel32:KERNEL32.dll
 0002:0000010c       __imp__FreeEnvironmentStringsW@4 1001a10c     kernel32:KERNEL32.dll
 0002:00000110       __imp__GetEnvironmentStringsW@0 1001a110     kernel32:KERNEL32.dll
 0002:00000114       __imp__GetCommandLineW@0   1001a114     kernel32:KERNEL32.dll
 0002:00000118       __imp__HeapCreate@12       1001a118     kernel32:KERNEL32.dll
 0002:0000011c       __imp__HeapDestroy@4       1001a11c     kernel32:KERNEL32.dll
 0002:00000120       __imp__DebugBreak@0        1001a120     kernel32:KERNEL32.dll
 0002:00000124       __imp__EnterCriticalSection@4 1001a124     kernel32:KERNEL32.dll
 0002:00000128       __imp__LeaveCriticalSection@4 1001a128     kernel32:KERNEL32.dll
 0002:0000012c       __imp__TryEnterCriticalSection@4 1001a12c     kernel32:KERNEL32.dll
 0002:00000130       __imp__DeleteCriticalSection@4 1001a130     kernel32:KERNEL32.dll
 0002:00000134       __imp__Sleep@4             1001a134     kernel32:KERNEL32.dll
 0002:00000138       __imp__GetTickCount@0      1001a138     kernel32:KERNEL32.dll
 0002:0000013c       __imp__RaiseException@16   1001a13c     kernel32:KERNEL32.dll
 0002:00000140       __imp__CreateThread@24     1001a140     kernel32:KERNEL32.dll
 0002:00000144       __imp__GetCurrentThreadId@0 1001a144     kernel32:KERNEL32.dll
 0002:00000148       __imp__TerminateThread@8   1001a148     kernel32:KERNEL32.dll
 0002:0000014c       __imp__SetLastError@4      1001a14c     kernel32:KERNEL32.dll
 0002:00000150       __imp__ResumeThread@4      1001a150     kernel32:KERNEL32.dll
 0002:00000154       __imp__IsDebuggerPresent@0 1001a154     kernel32:KERNEL32.dll
 0002:00000158       __imp__UnhandledExceptionFilter@4 1001a158     kernel32:KERNEL32.dll
 0002:0000015c       __imp__SetUnhandledExceptionFilter@4 1001a15c     kernel32:KERNEL32.dll
 0002:00000160       __imp__GetCurrentProcess@0 1001a160     kernel32:KERNEL32.dll
 0002:00000164       __imp__TerminateProcess@8  1001a164     kernel32:KERNEL32.dll
 0002:00000168       __imp__IsProcessorFeaturePresent@4 1001a168     kernel32:KERNEL32.dll
 0002:0000016c       __imp__InitializeCriticalSectionAndSpinCount@8 1001a16c     kernel32:KERNEL32.dll
 0002:00000170       __imp__SetEvent@4          1001a170     kernel32:KERNEL32.dll
 0002:00000174       __imp__ResetEvent@4        1001a174     kernel32:KERNEL32.dll
 0002:00000178       __imp__WaitForSingleObjectEx@12 1001a178     kernel32:KERNEL32.dll
 0002:0000017c       __imp__CreateEventW@16     1001a17c     kernel32:KERNEL32.dll
 0002:00000180       __imp__GetModuleHandleW@4  1001a180     kernel32:KERNEL32.dll
 0002:00000184       __imp__GetStartupInfoW@4   1001a184     kernel32:KERNEL32.dll
 0002:00000188       __imp__QueryPerformanceCounter@4 1001a188     kernel32:KERNEL32.dll
 0002:0000018c       __imp__GetSystemTimeAsFileTime@4 1001a18c     kernel32:KERNEL32.dll
 0002:00000190       __imp__InitializeSListHead@4 1001a190     kernel32:KERNEL32.dll
 0002:00000194       __imp__RtlUnwind@16        1001a194     kernel32:KERNEL32.dll
 0002:00000198       __imp__InterlockedFlushSList@4 1001a198     kernel32:KERNEL32.dll
 0002:0000019c       __imp__EncodePointer@4     1001a19c     kernel32:KERNEL32.dll
 0002:000001a0       __imp__TlsAlloc@0          1001a1a0     kernel32:KERNEL32.dll
 0002:000001a4       __imp__TlsGetValue@4       1001a1a4     kernel32:KERNEL32.dll
 0002:000001a8       __imp__TlsSetValue@8       1001a1a8     kernel32:KERNEL32.dll
 0002:000001ac       __imp__TlsFree@4           1001a1ac     kernel32:KERNEL32.dll
 0002:000001b0       __imp__LoadLibraryExW@12   1001a1b0     kernel32:KERNEL32.dll
 0002:000001b4       __imp__ExitProcess@4       1001a1b4     kernel32:KERNEL32.dll
 0002:000001b8       __imp__GetModuleHandleExW@12 1001a1b8     kernel32:KERNEL32.dll
 0002:000001bc       __imp__GetModuleFileNameA@12 1001a1bc     kernel32:KERNEL32.dll
 0002:000001c0       __imp__GetStringTypeW@16   1001a1c0     kernel32:KERNEL32.dll
 0002:000001c4       __imp__GetACP@0            1001a1c4     kernel32:KERNEL32.dll
 0002:000001c8       __imp__GetFileType@4       1001a1c8     kernel32:KERNEL32.dll
 0002:000001cc       __imp__LCMapStringW@24     1001a1cc     kernel32:KERNEL32.dll
 0002:000001d0       __imp__FindClose@4         1001a1d0     kernel32:KERNEL32.dll
 0002:000001d4       __imp__FindFirstFileExA@24 1001a1d4     kernel32:KERNEL32.dll
 0002:000001d8       __imp__FindNextFileA@8     1001a1d8     kernel32:KERNEL32.dll
 0002:000001dc       __imp__IsValidCodePage@4   1001a1dc     kernel32:KERNEL32.dll
 0002:000001e0       __imp__GetOEMCP@0          1001a1e0     kernel32:KERNEL32.dll
 0002:000001e4       __imp__GetCPInfo@8         1001a1e4     kernel32:KERNEL32.dll
 0002:000001e8       __imp__GetCommandLineA@0   1001a1e8     kernel32:KERNEL32.dll
 0002:000001ec       \177KERNEL32_NULL_THUNK_DATA 1001a1ec     kernel32:KERNEL32.dll
 0002:000001f0       __imp__CharUpperBuffW@8    1001a1f0     user32:USER32.dll
 0002:000001f4       __imp__CharLowerBuffW@8    1001a1f4     user32:USER32.dll
 0002:000001f8       __imp__GetDC@4             1001a1f8     user32:USER32.dll
 0002:000001fc       __imp__FillRect@12         1001a1fc     user32:USER32.dll
 0002:00000200       __imp__MessageBoxW@16      1001a200     user32:USER32.dll
 0002:00000204       __imp__ReleaseDC@8         1001a204     user32:USER32.dll
 0002:00000208       __imp__DrawTextW@20        1001a208     user32:USER32.dll
 0002:0000020c       \177USER32_NULL_THUNK_DATA 1001a20c     user32:USER32.dll
 0002:00000210       __imp__GetFileVersionInfoW@16 1001a210     version:VERSION.dll
 0002:00000214       __imp__VerQueryValueW@16   1001a214     version:VERSION.dll
 0002:00000218       __imp__GetFileVersionInfoSizeW@8 1001a218     version:VERSION.dll
 0002:0000021c       \177VERSION_NULL_THUNK_DATA 1001a21c     version:VERSION.dll
 0002:00000220       __imp__CoUninitialize@0    1001a220     ole32:ole32.dll
 0002:00000224       __imp__CoInitialize@4      1001a224     ole32:ole32.dll
 0002:00000228       \177ole32_NULL_THUNK_DATA  1001a228     ole32:ole32.dll
 0002:0000022c       ___guard_check_icall_fptr  1001a22c     LIBCMT:guard_support.obj
 0002:00000230       ___xc_a                    1001a230     LIBCMT:initializers.obj
 0002:00000234       ___xc_z                    1001a234     LIBCMT:initializers.obj
 0002:00000238       ___xi_a                    1001a238     LIBCMT:initializers.obj
 0002:00000240       ___acrt_stdio_initializer  1001a240     libucrt:stdio_initializer.obj
 0002:00000244       ___acrt_multibyte_initializer 1001a244     libucrt:multibyte_initializer.obj
 0002:00000248       ___acrt_tran_sse2_initializer 1001a248     libucrt:sse2_initializer.obj
 0002:0000024c       ___xi_z                    1001a24c     LIBCMT:initializers.obj
 0002:00000250       ___xl_a                    1001a250     LIBCMT:tlssup.obj
 0002:00000254       ___xl_z                    1001a254     LIBCMT:tlssup.obj
 0002:00000258       ___xp_a                    1001a258     LIBCMT:initializers.obj
 0002:0000025c       ___acrt_locale_terminator  1001a25c     libucrt:locale_initializer.obj
 0002:00000260       ___dcrt_console_output_terminator 1001a260     libucrt:console_output_initializer.obj
 0002:00000264       ___acrt_stdio_terminator   1001a264     libucrt:stdio_initializer.obj
 0002:00000268       ___xp_z                    1001a268     LIBCMT:initializers.obj
 0002:0000026c       ___xt_a                    1001a26c     LIBCMT:initializers.obj
 0002:00000270       ___xt_z                    1001a270     LIBCMT:initializers.obj
 0002:00000280       ??_C@_1BO@DPOJIDLN@?$AAB?$AAa?$AAc?$AAk?$AAg?$AAr?$AAo?$AAu?$AAn?$AAd?$AA?4?$AAx?$AAm?$AAl?$AA?$AA@ 1001a280     ConEmuBg.obj
 0002:000002a0       ??_C@_1BM@GCLEPEKO@?$AAP?$AAl?$AAu?$AAg?$AAi?$AAn?$AAE?$AAn?$AAa?$AAb?$AAl?$AAe?$AAd?$AA?$AA@ 1001a2a0     ConEmuBg.obj
 0002:000002bc       ??_C@_1BM@NBLKFLKP@?$AAX?$AAm?$AAl?$AAC?$AAo?$AAn?$AAf?$AAi?$AAg?$AAF?$AAi?$AAl?$AAe?$AA?$AA@ 1001a2bc     ConEmuBg.obj
 0002:000002d8       ??_C@_08BCACMCCB@ExitFARW?$AA@ 1001a2d8     ConEmuBg.obj
 0002:000002e4       ??_C@_0L@DJCGGOCO@ConfigureW?$AA@ 1001a2e4     ConEmuBg.obj
 0002:000002f0       ??_C@_11LOCGONAA@?$AA?$AA@ 1001a2f0     ConEmuBg.obj
 0002:000002f8       ??_7MStream@@6B@           1001a2f8     ConEmuBg.obj
 0002:00000334       ??_C@_13FPGAJAPJ@?$AA?2?$AA?$AA@ 1001a334     ConEmuBg.obj
 0002:00000338       ??_C@_1FG@DPPGENBC@?$AAL?$AAo?$AAa?$AAd?$AAA?$AAp?$AAp?$AAV?$AAe?$AAr?$AAs?$AAi?$AAo?$AAn?$AA?4?$AAV?$AAe?$AAr?$AAQ?$AAu?$AAe?$AAr?$AAy?$AAV?$AAa?$AAl?$AAu?$AAe?$AA?$CI?$AA?$CC?$AA?2?$AA?$CC@ 1001a338     ConEmuBg.obj
 0002:00000390       ??_C@_1FK@HILEEFML@?$AAL?$AAo?$AAa?$AAd?$AAA?$AAp?$AAp?$AAV?$AAe?$AAr?$AAs?$AAi?$AAo?$AAn?$AA?4?$AAG?$AAe?$AAt?$AAF?$AAi?$AAl?$AAe?$AAV?$AAe?$AAr?$AAs?$AAi?$AAo?$AAn?$AAI?$AAn?$AAf@ 1001a390     ConEmuBg.obj
 0002:000003f0       ??_C@_1GC@BINFLBDC@?$AAL?$AAo?$AAa?$AAd?$AAA?$AAp?$AAp?$AAV?$AAe?$AAr?$AAs?$AAi?$AAo?$AAn?$AA?5?$AAf?$AAa?$AAi?$AAl?$AAe?$AAd?$AA?$CB?$AA?5?$AAC?$AAa?$AAn?$AA?8?$AAt?$AA?5?$AAa?$AAl?$AAl@ 1001a3f0     ConEmuBg.obj
 0002:00000458       ??_C@_1GC@CPPHDKJK@?$AAL?$AAo?$AAa?$AAd?$AAA?$AAp?$AAp?$AAV?$AAe?$AAr?$AAs?$AAi?$AAo?$AAn?$AA?4?$AAG?$AAe?$AAt?$AAF?$AAi?$AAl?$AAe?$AAV?$AAe?$AAr?$AAs?$AAi?$AAo?$AAn?$AAI?$AAn?$AAf@ 1001a458     ConEmuBg.obj
 0002:000004c0       ??_C@_1EG@IINOBDEG@?$AAI?$AAn?$AAv?$AAa?$AAl?$AAi?$AAd?$AA?5?$AAa?$AAs?$AAM?$AAo?$AAd?$AAu?$AAl?$AAe?$AAP?$AAa?$AAt?$AAh?$AA?5?$AAw?$AAa?$AAs?$AA?5?$AAs?$AAp?$AAe?$AAc?$AAi?$AAf?$AAi@ 1001a4c0     ConEmuBg.obj
 0002:00000508       ??_C@_1CA@GGFPMHLH@?$AA?6?$AAE?$AAr?$AAr?$AAC?$AAo?$AAd?$AAe?$AA?$DN?$AA0?$AAx?$AA?$CF?$AA0?$AA8?$AAX?$AA?$AA@ 1001a508     ConEmuBg.obj
 0002:00000528       ??_C@_1FG@LNADFPCE@?$AAL?$AAo?$AAa?$AAd?$AAF?$AAa?$AAr?$AAV?$AAe?$AAr?$AAs?$AAi?$AAo?$AAn?$AA?4?$AAG?$AAe?$AAt?$AAM?$AAo?$AAd?$AAu?$AAl?$AAe?$AAF?$AAi?$AAl?$AAe?$AAN?$AAa?$AAm?$AAe@ 1001a528     ConEmuBg.obj
 0002:00000580       ??_C@_1CC@JLFNPNCD@?$AAC?$AAo?$AAn?$AAE?$AAm?$AAu?$AAB?$AAg?$AA?0?$AA?5?$AAP?$AAI?$AAD?$AA?$DN?$AA?$CF?$AAu?$AA?$AA@ 1001a580     ConEmuBg.obj
 0002:000005a4       ??_C@_1O@DPFEOIGE@?$AA?$DM?$AAN?$AAU?$AAL?$AAL?$AA?$DO?$AA?$AA@ 1001a5a4     ConEmuBg.obj
 0002:000005b4       ??_C@_1BI@NADJHDOD@?$AA?6?$AAE?$AAx?$AAp?$AAa?$AAn?$AAd?$AAe?$AAd?$AA?3?$AA?5?$AA?$AA@ 1001a5b4     ConEmuBg.obj
 0002:000005cc       ??_C@_1CA@DIJECNLO@?$AA?6?$AAC?$AAo?$AAn?$AAf?$AAi?$AAg?$AA?5?$AAv?$AAa?$AAl?$AAu?$AAe?$AA?3?$AA?5?$AA?$AA@ 1001a5cc     ConEmuBg.obj
 0002:000005f0       ??_C@_1GC@JKFCNIDB@?$AAT?$AAo?$AAo?$AA?5?$AAl?$AAo?$AAn?$AAg?$AA?5?$AAx?$AAm?$AAl?$AA?5?$AAp?$AAa?$AAt?$AAh?$AA?5?$AAa?$AAf?$AAt?$AAe?$AAr?$AA?5?$AAE?$AAx?$AAp?$AAa?$AAn?$AAd?$AAE?$AAn@ 1001a5f0     ConEmuBg.obj
 0002:00000658       ??_C@_1EE@OPEIBADO@?$AAC?$AAa?$AAn?$AA?8?$AAt?$AA?5?$AAi?$AAn?$AAi?$AAt?$AAi?$AAa?$AAl?$AAi?$AAz?$AAe?$AA?5?$AAn?$AAa?$AAm?$AAe?$AA?5?$AAo?$AAf?$AA?5?$AAx?$AAm?$AAl?$AA?5?$AAf?$AAi?$AAl@ 1001a658     ConEmuBg.obj
 0002:000006a0       ??_C@_1EA@MFDKJDBE@?$AAC?$AAo?$AAn?$AAf?$AAi?$AAg?$AAu?$AAr?$AAa?$AAt?$AAi?$AAo?$AAn?$AA?5?$AAx?$AAm?$AAl?$AA?5?$AAf?$AAi?$AAl?$AAe?$AA?5?$AAi?$AAs?$AA?5?$AAe?$AAm?$AAp?$AAt?$AAy?$AA?$AA@ 1001a6a0     ConEmuBg.obj
 0002:000006e0       ??_C@_1FM@NIEBMEBA@?$AAC?$AAa?$AAn?$AA?8?$AAt?$AA?5?$AAa?$AAl?$AAl?$AAo?$AAc?$AAa?$AAt?$AAe?$AA?5?$AA?$CF?$AAu?$AA?5?$AAb?$AAy?$AAt?$AAe?$AAs?$AA?5?$AAf?$AAo?$AAr?$AA?5?$AAx?$AAm?$AAl?$AA?5@ 1001a6e0     ConEmuBg.obj
 0002:00000740       ??_C@_1GA@PEKCNEOL@?$AAC?$AAa?$AAn?$AA?8?$AAt?$AA?5?$AAr?$AAe?$AAa?$AAd?$AA?5?$AA?$CF?$AAu?$AA?5?$AAb?$AAy?$AAt?$AAe?$AAs?$AA?5?$AAf?$AAr?$AAo?$AAm?$AA?5?$AAx?$AAm?$AAl?$AA?5?$AAc?$AAo?$AAn@ 1001a740     ConEmuBg.obj
 0002:000007a0       ??_C@_1HE@IENNFNAG@?$AAC?$AAo?$AAn?$AAf?$AAi?$AAg?$AAu?$AAr?$AAa?$AAt?$AAi?$AAo?$AAn?$AA?5?$AAx?$AAm?$AAl?$AA?5?$AAf?$AAi?$AAl?$AAe?$AA?5?$AAw?$AAa?$AAs?$AA?5?$AAn?$AAo?$AAt?$AA?5?$AAf@ 1001a7a0     ConEmuBg.obj
 0002:00000818       ??_C@_1HA@MHONNEJA@?$AAC?$AAr?$AAe?$AAa?$AAt?$AAe?$AAC?$AAo?$AAm?$AAp?$AAa?$AAt?$AAi?$AAb?$AAl?$AAe?$AA?$FL?$AAD?$AAC?$AA?$HM?$AAB?$AAi?$AAt?$AAm?$AAa?$AAp?$AA?$FN?$AA?5?$AAf?$AAa?$AAi?$AAl@ 1001a818     ConEmuBg.obj
 0002:00000888       ??_C@_1GC@KCIBPHOM@?$AAG?$AAe?$AAt?$AAM?$AAo?$AAd?$AAu?$AAl?$AAe?$AAF?$AAi?$AAl?$AAe?$AAN?$AAa?$AAm?$AAe?$AA?5?$AAf?$AAa?$AAi?$AAl?$AAe?$AAd?$AA?5?$AAi?$AAn?$AA?5?$AAG?$AAD?$AAI?$AAP@ 1001a888     ConEmuBg.obj
 0002:000008ec       ??_C@_1BI@LOJECBFD@?$AAG?$AAd?$AAi?$AAP?$AAl?$AAu?$AAs?$AA?4?$AAd?$AAl?$AAl?$AA?$AA@ 1001a8ec     ConEmuBg.obj
 0002:00000904       ??_C@_1CO@CNEBCEFN@?$AAG?$AAd?$AAi?$AAP?$AAl?$AAu?$AAs?$AA?4?$AAd?$AAl?$AAl?$AA?5?$AAn?$AAo?$AAt?$AA?5?$AAf?$AAo?$AAu?$AAn?$AAd?$AA?$CB?$AA?$AA@ 1001a904     ConEmuBg.obj
 0002:00000934       ??_C@_0P@NIGHOHPH@GdiplusStartup?$AA@ 1001a934     ConEmuBg.obj
 0002:00000944       ??_C@_0BA@OMKIAPCJ@GdiplusShutdown?$AA@ 1001a944     ConEmuBg.obj
 0002:00000954       ??_C@_0BJ@IPKMAACN@GdipCreateBitmapFromFile?$AA@ 1001a954     ConEmuBg.obj
 0002:00000970       ??_C@_0BC@DPLNHGNM@GdipGetImageWidth?$AA@ 1001a970     ConEmuBg.obj
 0002:00000984       ??_C@_0BD@JIGBIPOH@GdipGetImageHeight?$AA@ 1001a984     ConEmuBg.obj
 0002:00000998       ??_C@_0BB@MGCHKKMH@GdipDisposeImage?$AA@ 1001a998     ConEmuBg.obj
 0002:000009ac       ??_C@_0P@DANGKLEH@GdipDrawImageI?$AA@ 1001a9ac     ConEmuBg.obj
 0002:000009bc       ??_C@_0BC@PACDIGJN@GdipCreateFromHDC?$AA@ 1001a9bc     ConEmuBg.obj
 0002:000009d0       ??_C@_0BD@MFGJCODH@GdipDeleteGraphics?$AA@ 1001a9d0     ConEmuBg.obj
 0002:000009e4       ??_C@_09EJEFPMLL@GdipGetDC?$AA@ 1001a9e4     ConEmuBg.obj
 0002:000009f0       ??_C@_0O@KHJJFDII@GdipReleaseDC?$AA@ 1001a9f0     ConEmuBg.obj
 0002:00000a00       ??_C@_0BM@MMIJHLFD@GdipGetImageGraphicsContext?$AA@ 1001aa00     ConEmuBg.obj
 0002:00000a1c       ??_C@_0BI@GEKGFIAG@GdipBitmapConvertFormat?$AA@ 1001aa1c     ConEmuBg.obj
 0002:00000a34       ??_C@_1CM@JMKADHIE@?$AAG?$AAd?$AAi?$AAp?$AAl?$AAu?$AAs?$AAS?$AAt?$AAa?$AAr?$AAt?$AAu?$AAp?$AA?5?$AAf?$AAa?$AAi?$AAl?$AAe?$AAd?$AA?$AA@ 1001aa34     ConEmuBg.obj
 0002:00000a60       ??_C@_1EG@ENHOOKPB@?$AAF?$AAu?$AAn?$AAc?$AAt?$AAi?$AAo?$AAn?$AAs?$AA?5?$AAn?$AAo?$AAt?$AA?5?$AAf?$AAo?$AAu?$AAn?$AAd?$AA?5?$AAi?$AAn?$AA?5?$AAG?$AAd?$AAi?$AAP?$AAl?$AAu?$AAs?$AA?4?$AAd@ 1001aa60     ConEmuBg.obj
 0002:00000aa8       ??_C@_0BD@FCCFIJEI@Bg?3?3FreeThreadProc?$AA@ 1001aaa8     ConEmuBg.obj
 0002:00000abc       ??_C@_0DH@FMEJPGLI@t?3?2vcproject?2maximus5?2conemu?2src@ 1001aabc     ConEmuBg.obj
 0002:00000af8       ??_C@_1EK@HIHBLDLC@?$AAC?$AAa?$AAn?$AA?8?$AAt?$AA?5?$AAa?$AAl?$AAl?$AAo?$AAc?$AAa?$AAt?$AAe?$AA?5?$AAm?$AAe?$AAm?$AAo?$AAr?$AAy?$AA?5?$AAf?$AAo?$AAr?$AA?5?$AAs?$AAz?$AAF?$AAu?$AAl?$AAl@ 1001aaf8     ConEmuBg.obj
 0002:00000b44       ??_C@_1DI@MGMDCCIK@?$AAC?$AAa?$AAn?$AA?8?$AAt?$AA?5?$AAl?$AAo?$AAa?$AAd?$AA?5?$AAi?$AAm?$AAa?$AAg?$AAe?$AA?0?$AA?5?$AAE?$AAr?$AAr?$AA?$DN?$AA?$CF?$AAi?$AA?6?$AA?$CF?$AAs?$AA?$AA@ 1001ab44     ConEmuBg.obj
 0002:00000b7c       ??_C@_1DO@BMBIALGO@?$AAG?$AAe?$AAt?$AAI?$AAm?$AAa?$AAg?$AAe?$AAS?$AAi?$AAz?$AAe?$AA?5?$AAf?$AAa?$AAi?$AAl?$AAe?$AAd?$AA?0?$AA?5?$AAE?$AAr?$AAr?$AA?$DN?$AA?$CF?$AAi?$AA?6?$AA?$CF?$AAs?$AA?$AA@ 1001ab7c     ConEmuBg.obj
 0002:00000bc0       ??_C@_1EG@KBBKNBAB@?$AAC?$AAr?$AAe?$AAa?$AAt?$AAe?$AAC?$AAo?$AAm?$AAp?$AAa?$AAt?$AAi?$AAb?$AAl?$AAe?$AA?$FL?$AAD?$AAC?$AA?$HM?$AAB?$AAi?$AAt?$AAm?$AAa?$AAp?$AA?$FN?$AA?5?$AAf?$AAa?$AAi?$AAl@ 1001abc0     ConEmuBg.obj
 0002:00000c08       ??_C@_1EI@MNPBDJFF@?$AAG?$AAd?$AAi?$AAp?$AAC?$AAr?$AAe?$AAa?$AAt?$AAe?$AAF?$AAr?$AAo?$AAm?$AAH?$AAD?$AAC?$AA?5?$AAf?$AAa?$AAi?$AAl?$AAe?$AAd?$AA?0?$AA?5?$AAE?$AAr?$AAr?$AA?$DN?$AA?$CF?$AAi@ 1001ac08     ConEmuBg.obj
 0002:00000c50       ??_C@_1EC@FCMECJAF@?$AAG?$AAd?$AAi?$AAp?$AAD?$AAr?$AAa?$AAw?$AAI?$AAm?$AAa?$AAg?$AAe?$AAI?$AA?5?$AAf?$AAa?$AAi?$AAl?$AAe?$AAd?$AA?0?$AA?5?$AAE?$AAr?$AAr?$AA?$DN?$AA?$CF?$AAi?$AA?6?$AA?$CF?$AAs@ 1001ac50     ConEmuBg.obj
 0002:00000c94       ??_C@_1DI@COJKFCDM@?$AAG?$AAd?$AAi?$AAp?$AAG?$AAe?$AAt?$AAD?$AAC?$AA?5?$AAf?$AAa?$AAi?$AAl?$AAe?$AAd?$AA?0?$AA?5?$AAE?$AAr?$AAr?$AA?$DN?$AA?$CF?$AAi?$AA?6?$AA?$CF?$AAs?$AA?$AA@ 1001ac94     ConEmuBg.obj
 0002:00000cd0       ??_C@_1EM@FGINKPEA@?$AAC?$AAa?$AAn?$AA?8?$AAt?$AA?5?$AAa?$AAl?$AAl?$AAo?$AAc?$AAa?$AAt?$AAe?$AA?5?$AAm?$AAe?$AAm?$AAo?$AAr?$AAy?$AA?5?$AAf?$AAo?$AAr?$AA?5?$AAC?$AAa?$AAc?$AAh?$AAe?$AAd@ 1001acd0     ConEmuBg.obj
 0002:00000d1c       ??_C@_1BI@DCLCNAFM@?$AAx?$AAm?$AAl?$AAl?$AAi?$AAt?$AAe?$AA?4?$AAd?$AAl?$AAl?$AA?$AA@ 1001ad1c     ConEmuBg.obj
 0002:00000d34       ??_C@_1CM@BLKKKOJI@?$AAx?$AAm?$AAl?$AAl?$AAi?$AAt?$AAe?$AA?4?$AAd?$AAl?$AAl?$AA?5?$AAn?$AAo?$AAt?$AA?5?$AAf?$AAo?$AAu?$AAn?$AAd?$AA?$AA@ 1001ad34     ConEmuBg.obj
 0002:00000d60       ??_C@_0BA@EICHKACL@CreateXmlReader?$AA@ 1001ad60     ConEmuBg.obj
 0002:00000d70       ??_C@_1GM@NPCBAKPP@?$AAf?$AAu?$AAn?$AAc?$AAt?$AAi?$AAo?$AAn?$AA?5?$AAC?$AAr?$AAe?$AAa?$AAt?$AAe?$AAX?$AAm?$AAl?$AAR?$AAe?$AAa?$AAd?$AAe?$AAr?$AA?5?$AAi?$AAn?$AA?5?$AAt?$AAh?$AAe?$AA?5@ 1001ad70     ConEmuBg.obj
 0002:00000ddc       __GUID_7279fc81_709d_4095_b63d_69fe4b0d9030 1001addc     ConEmuBg.obj
 0002:00000dec       ??_C@_1O@FLJJBOMO@?$AA?2?$AAT?$AAE?$AAM?$AAP?$AA?2?$AA?$AA@ 1001adec     ConEmuBg.obj
 0002:00000dfc       ??_C@_1O@IANIHGAM@?$AAw?$AAi?$AAn?$AAd?$AAo?$AAw?$AA?$AA@ 1001adfc     ConEmuBg.obj
 0002:00000e0c       ??_C@_1M@HCONLDPB@?$AAp?$AAa?$AAn?$AAe?$AAl?$AA?$AA@ 1001ae0c     ConEmuBg.obj
 0002:00000e18       ??_C@_19FHBCDCCA@?$AAt?$AAy?$AAp?$AAe?$AA?$AA@ 1001ae18     ConEmuBg.obj
 0002:00000e24       ??_C@_1O@OCKFCHPL@?$AAP?$AAA?$AAN?$AAE?$AAL?$AAS?$AA?$AA@ 1001ae24     ConEmuBg.obj
 0002:00000e34       ??_C@_1M@HLGJKDIH@?$AAP?$AAA?$AAN?$AAE?$AAL?$AA?$AA@ 1001ae34     ConEmuBg.obj
 0002:00000e40       ??_C@_1O@PEPCDNON@?$AAE?$AAD?$AAI?$AAT?$AAO?$AAR?$AA?$AA@ 1001ae40     ConEmuBg.obj
 0002:00000e50       ??_C@_1O@EFKGOBLP@?$AAV?$AAI?$AAE?$AAW?$AAE?$AAR?$AA?$AA@ 1001ae50     ConEmuBg.obj
 0002:00000e60       ??_C@_1M@EKGBHJEJ@?$AAD?$AAR?$AAI?$AAV?$AAE?$AA?$AA@ 1001ae60     ConEmuBg.obj
 0002:00000e6c       ??_C@_1O@BDNPEFIG@?$AAP?$AAL?$AAU?$AAG?$AAI?$AAN?$AA?$AA@ 1001ae6c     ConEmuBg.obj
 0002:00000e7c       ??_C@_19EINGHGNA@?$AAT?$AAR?$AAE?$AAE?$AA?$AA@ 1001ae7c     ConEmuBg.obj
 0002:00000e88       ??_C@_1M@KIGDKMPO@?$AAQ?$AAV?$AAI?$AAE?$AAW?$AA?$AA@ 1001ae88     ConEmuBg.obj
 0002:00000e94       ??_C@_19FILLMKCG@?$AAI?$AAN?$AAF?$AAO?$AA?$AA@ 1001ae94     ConEmuBg.obj
 0002:00000ea0       ??_C@_1BE@FAHOEFOG@?$AAd?$AAr?$AAi?$AAv?$AAe?$AAt?$AAy?$AAp?$AAe?$AA?$AA@ 1001aea0     ConEmuBg.obj
 0002:00000eb4       ??_C@_1BI@BCACJIAB@?$AAN?$AAO?$AA_?$AAR?$AAO?$AAO?$AAT?$AA_?$AAD?$AAI?$AAR?$AA?$AA@ 1001aeb4     ConEmuBg.obj
 0002:00000ecc       ??_C@_1BE@JMGCMLBE@?$AAR?$AAE?$AAM?$AAO?$AAV?$AAA?$AAB?$AAL?$AAE?$AA?$AA@ 1001aecc     ConEmuBg.obj
 0002:00000ee0       ??_C@_1M@PEPLLLCM@?$AAF?$AAI?$AAX?$AAE?$AAD?$AA?$AA@ 1001aee0     ConEmuBg.obj
 0002:00000eec       ??_C@_1O@OAMNPHFH@?$AAR?$AAE?$AAM?$AAO?$AAT?$AAE?$AA?$AA@ 1001aeec     ConEmuBg.obj
 0002:00000efc       ??_C@_1M@NEPFDHKI@?$AAC?$AAD?$AAR?$AAO?$AAM?$AA?$AA@ 1001aefc     ConEmuBg.obj
 0002:00000f08       ??_C@_1BA@EJELCCEN@?$AAR?$AAA?$AAM?$AAD?$AAI?$AAS?$AAK?$AA?$AA@ 1001af08     ConEmuBg.obj
 0002:00000f18       ??_C@_1BC@FAFPDLON@?$AAp?$AAa?$AAt?$AAh?$AAt?$AAy?$AAp?$AAe?$AA?$AA@ 1001af18     ConEmuBg.obj
 0002:00000f2c       ??_C@_19LFDMGLCC@?$AAT?$AAE?$AAM?$AAP?$AA?$AA@ 1001af2c     ConEmuBg.obj
 0002:00000f38       ??_C@_1BE@FDJCBAKA@?$AAp?$AAa?$AAt?$AAh?$AAm?$AAa?$AAt?$AAc?$AAh?$AA?$AA@ 1001af38     ConEmuBg.obj
 0002:00000f4c       ??_C@_1O@JODKLKCF@?$AAf?$AAo?$AAr?$AAm?$AAa?$AAt?$AA?$AA@ 1001af4c     ConEmuBg.obj
 0002:00000f5c       ??_C@_1BC@LGPIFEA@?$AAd?$AAi?$AAs?$AAa?$AAb?$AAl?$AAe?$AAd?$AA?$AA@ 1001af5c     ConEmuBg.obj
 0002:00000f70       ??_C@_1M@EENKLIPJ@?$AAc?$AAo?$AAl?$AAo?$AAr?$AA?$AA@ 1001af70     ConEmuBg.obj
 0002:00000f7c       ??_C@_17PAHGLGBB@?$AAr?$AAg?$AAb?$AA?$AA@ 1001af7c     ConEmuBg.obj
 0002:00000f84       ??_C@_1BC@NNDMOMJF@?$AAr?$AAg?$AAb?$AA_?$AAd?$AAa?$AAr?$AAk?$AA?$AA@ 1001af84     ConEmuBg.obj
 0002:00000f98       ??_C@_1BE@OGMDEBBA@?$AAr?$AAg?$AAb?$AA_?$AAl?$AAi?$AAg?$AAh?$AAt?$AA?$AA@ 1001af98     ConEmuBg.obj
 0002:00000fac       ??_C@_17NMNENAKF@?$AAb?$AAg?$AAr?$AA?$AA@ 1001afac     ConEmuBg.obj
 0002:00000fb4       ??_C@_1BC@JFCNIMOB@?$AAb?$AAg?$AAr?$AA_?$AAd?$AAa?$AAr?$AAk?$AA?$AA@ 1001afb4     ConEmuBg.obj
 0002:00000fc8       ??_C@_1BE@OACCNEKL@?$AAb?$AAg?$AAr?$AA_?$AAl?$AAi?$AAg?$AAh?$AAt?$AA?$AA@ 1001afc8     ConEmuBg.obj
 0002:00000fdc       ??_C@_1M@OAJKEOAM@?$AAs?$AAh?$AAi?$AAf?$AAt?$AA?$AA@ 1001afdc     ConEmuBg.obj
 0002:00000fe8       ??_C@_17IHBDLLG@?$AAy?$AAe?$AAs?$AA?$AA@ 1001afe8     ConEmuBg.obj
 0002:00000ff0       ??_C@_1M@LPGODFOM@?$AAs?$AAp?$AAa?$AAc?$AAe?$AA?$AA@ 1001aff0     ConEmuBg.obj
 0002:00000ffc       ??_C@_1M@GACLNJGJ@?$AAl?$AAa?$AAr?$AAg?$AAe?$AA?$AA@ 1001affc     ConEmuBg.obj
 0002:00001008       ??_C@_17FDPGNGBJ@?$AAo?$AAf?$AAf?$AA?$AA@ 1001b008     ConEmuBg.obj
 0002:00001010       ??_C@_1M@NFEAPLNL@?$AAt?$AAi?$AAt?$AAl?$AAe?$AA?$AA@ 1001b010     ConEmuBg.obj
 0002:0000101c       ??_C@_1M@CNKDNHCK@?$AA?5?$AA?7?$AA?$AN?$AA?6?$AA?$CL?$AA?$AA@ 1001b01c     ConEmuBg.obj
 0002:00001028       ??_C@_1O@DFDGIFKD@?$AAV?$AAO?$AAL?$AAU?$AAM?$AAE?$AA?$AA@ 1001b028     ConEmuBg.obj
 0002:00001038       ??_C@_1BG@CACAJBGP@?$AAV?$AAO?$AAL?$AAU?$AAM?$AAE?$AAS?$AAI?$AAZ?$AAE?$AA?$AA@ 1001b038     ConEmuBg.obj
 0002:00001050       ??_C@_1BG@DCPGEGPA@?$AAV?$AAO?$AAL?$AAU?$AAM?$AAE?$AAF?$AAR?$AAE?$AAE?$AA?$AA@ 1001b050     ConEmuBg.obj
 0002:00001068       ??_C@_1BI@FHFKHMCH@?$AAP?$AAA?$AAN?$AAE?$AAL?$AAF?$AAO?$AAR?$AAM?$AAA?$AAT?$AA?$AA@ 1001b068     ConEmuBg.obj
 0002:00001080       ??_C@_17EHOCEIDI@?$AAi?$AAm?$AAg?$AA?$AA@ 1001b080     ConEmuBg.obj
 0002:00001088       ??_C@_17DCNMIAEN@?$AAr?$AAe?$AAf?$AA?$AA@ 1001b088     ConEmuBg.obj
 0002:00001090       ??_C@_13OPKGLAFF@?$AAB?$AA?$AA@ 1001b090     ConEmuBg.obj
 0002:00001094       ??_C@_15BKLPDEEF@?$AAK?$AAB?$AA?$AA@ 1001b094     ConEmuBg.obj
 0002:0000109c       ??_C@_15MMOGNHFI@?$AAM?$AAB?$AA?$AA@ 1001b09c     ConEmuBg.obj
 0002:000010a4       ??_C@_15GNHNPEDO@?$AAG?$AAB?$AA?$AA@ 1001b0a4     ConEmuBg.obj
 0002:000010ac       ??_C@_15OIDPIEAL@?$AAT?$AAB?$AA?$AA@ 1001b0ac     ConEmuBg.obj
 0002:000010b4       ??_C@_15HDKOMGBN@?$AAP?$AAB?$AA?$AA@ 1001b0b4     ConEmuBg.obj
 0002:000010bc       ??_C@_1BC@MFPHLBKH@?$AA?$CF?$AAu?$AA?4?$AA?$CF?$AAu?$AA?5?$AA?$CF?$AAs?$AA?$AA@ 1001b0bc     ConEmuBg.obj
 0002:000010d0       ??_C@_1M@MDEFCCAF@?$AA?$CF?$AAu?$AA?5?$AA?$CF?$AAs?$AA?$AA@ 1001b0d0     ConEmuBg.obj
 0002:000010dc       ??_C@_19DKAIAFPE@?$AAL?$AAe?$AAf?$AAt?$AA?$AA@ 1001b0dc     ConEmuBg.obj
 0002:000010e8       ??_C@_1M@KDEMMBOH@?$AAR?$AAi?$AAg?$AAh?$AAt?$AA?$AA@ 1001b0e8     ConEmuBg.obj
 0002:000010f8       ??_C@_1FK@LJOGCJPM@?$AAC?$AAo?$AAn?$AAE?$AAm?$AAu?$AAB?$AAk?$AA?3?$AA?5?$AAD?$AAi?$AAs?$AAa?$AAb?$AAl?$AAe?$AAd?$AA?5?$AA?$CF?$AAs?$AA?5?$AA?9?$AA?5?$AA?$HL?$AA?$CF?$AAi?$AA?0?$AA?$CF?$AAi?$AA?0?$AA?$CF@ 1001b0f8     ConEmuBg.obj
 0002:00001154       ??_C@_1BO@KJOLJEJK@?$AAi?$AAm?$AAg?$AA?1?$AAp?$AAl?$AAu?$AAg?$AAi?$AAn?$AA?4?$AAp?$AAn?$AAg?$AA?$AA@ 1001b154     ConEmuBg.obj
 0002:00001174       ??_C@_1DA@JALAODAO@?$AAi?$AAm?$AAg?$AA?1?$AAd?$AAr?$AAi?$AAv?$AAe?$AA_?$AAr?$AAe?$AAm?$AAo?$AAv?$AAa?$AAb?$AAl?$AAe?$AA?4?$AAp?$AAn?$AAg?$AA?$AA@ 1001b174     ConEmuBg.obj
 0002:000011a4       ??_C@_1CM@FDAGABBA@?$AAi?$AAm?$AAg?$AA?1?$AAd?$AAr?$AAi?$AAv?$AAe?$AA_?$AAn?$AAe?$AAt?$AAw?$AAo?$AAr?$AAk?$AA?4?$AAp?$AAn?$AAg?$AA?$AA@ 1001b1a4     ConEmuBg.obj
 0002:000011d0       ??_C@_1CI@DLJJCGCI@?$AAi?$AAm?$AAg?$AA?1?$AAd?$AAr?$AAi?$AAv?$AAe?$AA_?$AAc?$AAd?$AAr?$AAo?$AAm?$AA?4?$AAp?$AAn?$AAg?$AA?$AA@ 1001b1d0     ConEmuBg.obj
 0002:000011f8       ??_C@_1CM@NJAGAAPF@?$AAi?$AAm?$AAg?$AA?1?$AAd?$AAr?$AAi?$AAv?$AAe?$AA_?$AAr?$AAa?$AAm?$AAd?$AAi?$AAs?$AAk?$AA?4?$AAp?$AAn?$AAg?$AA?$AA@ 1001b1f8     ConEmuBg.obj
 0002:00001224       ??_C@_1CI@FIJFGDPK@?$AAi?$AAm?$AAg?$AA?1?$AAd?$AAr?$AAi?$AAv?$AAe?$AA_?$AAf?$AAi?$AAx?$AAe?$AAd?$AA?4?$AAp?$AAn?$AAg?$AA?$AA@ 1001b224     ConEmuBg.obj
 0002:00001250       ??_C@_1EI@KDEPAOIE@?$AAC?$AAo?$AAn?$AAE?$AAm?$AAu?$AAB?$AAk?$AA?3?$AA?5?$AA?$CF?$AAs?$AA?5?$AA?9?$AA?5?$AA?$HL?$AA?$CF?$AAi?$AA?0?$AA?$CF?$AAi?$AA?0?$AA?$CF?$AAi?$AA?0?$AA?$CF?$AAi?$AA?$CJ?$AA?5?$AA?$CD?$AA?$CF?$AA0@ 1001b250     ConEmuBg.obj
 0002:00001298       ??_C@_1M@KAKMLIHO@?$AAA?$AAr?$AAi?$AAa?$AAl?$AA?$AA@ 1001b298     ConEmuBg.obj
 0002:000012a8       ??_C@_1FE@OJCEMPCK@?$AAC?$AAo?$AAn?$AAE?$AAm?$AAu?$AAB?$AAk?$AA?3?$AA?5?$AAI?$AAn?$AAv?$AAi?$AAs?$AAi?$AAb?$AAl?$AAe?$AA?5?$AAL?$AAe?$AAf?$AAt?$AA?5?$AA?9?$AA?5?$AA?$HL?$AA?$CF?$AAi?$AA?0?$AA?$CF@ 1001b2a8     ConEmuBg.obj
 0002:00001300       ??_C@_1FG@IGPHDCHD@?$AAC?$AAo?$AAn?$AAE?$AAm?$AAu?$AAB?$AAk?$AA?3?$AA?5?$AAI?$AAn?$AAv?$AAi?$AAs?$AAi?$AAb?$AAl?$AAe?$AA?5?$AAR?$AAi?$AAg?$AAh?$AAt?$AA?5?$AA?9?$AA?5?$AA?$HL?$AA?$CF?$AAi?$AA?0@ 1001b300     ConEmuBg.obj
 0002:00001360       __xmm@00000000000000080000000000000000 1001b360     ConEmuBg1900.obj
 0002:00001370       __xmm@00000000000000090000000000000007 1001b370     ConEmuBg1900.obj
 0002:00001380       ??_C@_1CE@PJKCDLK@?$AAC?$AAo?$AAn?$AAE?$AAm?$AAu?$AA?5?$AAB?$AAa?$AAc?$AAk?$AAg?$AAr?$AAo?$AAu?$AAn?$AAd?$AA?$AA@ 1001b380     ConEmuBg2800.obj
 0002:000013a8       ??_C@_1GC@GCGDBDMO@?$AAP?$AAa?$AAi?$AAn?$AAt?$AA?5?$AAF?$AAa?$AAr?$AA?5?$AAp?$AAa?$AAn?$AAe?$AAl?$AAs?$AA?5?$AAb?$AAa?$AAc?$AAk?$AAg?$AAr?$AAo?$AAu?$AAn?$AAd?$AA?5?$AAi?$AAn?$AA?5?$AAt@ 1001b3a8     ConEmuBg2800.obj
 0002:0000140c       ??_C@_1DE@DJEAMLPH@?$AAC?$AAo?$AAn?$AAE?$AAm?$AAu?$AA?4?$AAM?$AAa?$AAx?$AAi?$AAm?$AAu?$AAs?$AA5?$AA?$EA?$AAg?$AAm?$AAa?$AAi?$AAl?$AA?4?$AAc?$AAo?$AAm?$AA?$AA@ 1001b40c     ConEmuBg2800.obj
 0002:00001440       ??_C@_1BE@POBJGOHE@?$AAC?$AAo?$AAn?$AAE?$AAm?$AAu?$AAB?$AAg?$AA?2?$AA?$AA@ 1001b440     ConEmuBg995.obj
 0002:00001454       _IID_IUnknown              1001b454     uuid:unknwn_i.obj
 0002:00001464       _IID_ISequentialStream     1001b464     uuid:objidl_i.obj
 0002:00001474       _IID_IStream               1001b474     uuid:objidl_i.obj
 0002:00001484       ??_C@_00CNPNBAHC@?$AA@     1001b484     common-kernel32:MStrDup.obj
 0002:00001488       ??_C@_05LCABBMOG@?$CFs?3?$CFi?$AA@ 1001b488     common-kernel32:WThreads.obj
 0002:0000149c       ??_7type_info@@6B@         1001b49c     LIBCMT:std_type_info_static.obj
 0002:000014a0       ??_C@_1EC@JIJBPKFM@?$AAa?$AAp?$AAi?$AA?9?$AAm?$AAs?$AA?9?$AAw?$AAi?$AAn?$AA?9?$AAc?$AAo?$AAr?$AAe?$AA?9?$AAs?$AAy?$AAn?$AAc?$AAh?$AA?9?$AAl?$AA1?$AA?9?$AA2?$AA?9?$AA0?$AA?4?$AAd?$AAl?$AAl@ 1001b4a0     LIBCMT:thread_safe_statics.obj
 0002:000014e4       ??_C@_1BK@MGMFAEKH@?$AAk?$AAe?$AAr?$AAn?$AAe?$AAl?$AA3?$AA2?$AA?4?$AAd?$AAl?$AAl?$AA?$AA@ 1001b4e4     LIBCMT:thread_safe_statics.obj
 0002:00001500       ??_C@_0BM@HLJJNPAH@InitializeConditionVariable?$AA@ 1001b500     LIBCMT:thread_safe_statics.obj
 0002:0000151c       ??_C@_0BJ@JEBJOJFJ@SleepConditionVariableCS?$AA@ 1001b51c     LIBCMT:thread_safe_statics.obj
 0002:00001538       ??_C@_0BJ@PGPPEPCC@WakeAllConditionVariable?$AA@ 1001b538     LIBCMT:thread_safe_statics.obj
 0002:00001554       __pDefaultRawDllMain       1001b554     LIBCMT:dll_dllmain.obj
 0002:00001554       __pRawDllMain              1001b554     LIBCMT:dll_dllmain.obj
 0002:0000155c       ??_7exception@std@@6B@     1001b55c     libvcruntime:frame.obj
 0002:00001564       ??_C@_0BC@EOODALEL@Unknown?5exception?$AA@ 1001b564     libvcruntime:frame.obj
 0002:0000157c       ??_7bad_exception@std@@6B@ 1001b57c     libvcruntime:frame.obj
 0002:00001584       ??_C@_0O@DPKOEFFH@bad?5exception?$AA@ 1001b584     libvcruntime:frame.obj
 0002:000015a0       ??_C@_1DM@KHCHBNEB@?$AAa?$AAp?$AAi?$AA?9?$AAm?$AAs?$AA?9?$AAw?$AAi?$AAn?$AA?9?$AAc?$AAo?$AAr?$AAe?$AA?9?$AAf?$AAi?$AAb?$AAe?$AAr?$AAs?$AA?9?$AAl?$AA1?$AA?9?$AA1?$AA?9?$AA1?$AA?$AA@ 1001b5a0     libvcruntime:winapi_downlevel.obj
 0002:000015dc       ??_C@_1DK@LPPGFMPP@?$AAa?$AAp?$AAi?$AA?9?$AAm?$AAs?$AA?9?$AAw?$AAi?$AAn?$AA?9?$AAc?$AAo?$AAr?$AAe?$AA?9?$AAs?$AAy?$AAn?$AAc?$AAh?$AA?9?$AAl?$AA1?$AA?9?$AA2?$AA?9?$AA0?$AA?$AA@ 1001b5dc     libvcruntime:winapi_downlevel.obj
 0002:00001618       ??_C@_1BC@GDMECMAK@?$AAk?$AAe?$AAr?$AAn?$AAe?$AAl?$AA3?$AA2?$AA?$AA@ 1001b618     libvcruntime:winapi_downlevel.obj
 0002:0000162c       ??_C@_1BA@PFFKHIOG@?$AAa?$AAp?$AAi?$AA?9?$AAm?$AAs?$AA?9?$AA?$AA@ 1001b62c     libvcruntime:winapi_downlevel.obj
 0002:0000163c       ??_C@_1BA@IAIFMGEF@?$AAe?$AAx?$AAt?$AA?9?$AAm?$AAs?$AA?9?$AA?$AA@ 1001b63c     libvcruntime:winapi_downlevel.obj
 0002:00001654       ??_C@_08KNHFBNJ@FlsAlloc?$AA@ 1001b654     libvcruntime:winapi_downlevel.obj
 0002:00001668       ??_C@_07PEJMOBNF@FlsFree?$AA@ 1001b668     libvcruntime:winapi_downlevel.obj
 0002:00001678       ??_C@_0M@GDNOONDI@FlsGetValue?$AA@ 1001b678     libvcruntime:winapi_downlevel.obj
 0002:0000168c       ??_C@_0M@JCPCPOEF@FlsSetValue?$AA@ 1001b68c     libvcruntime:winapi_downlevel.obj
 0002:000016a0       ??_C@_0BM@HCFOFFN@InitializeCriticalSectionEx?$AA@ 1001b6a0     libvcruntime:winapi_downlevel.obj
 0002:00001858       ??_C@_08EHJDFFNH@__based?$CI?$AA@ 1001b858     libvcruntime:undname.obj
 0002:00001864       ??_C@_07KOLFKCDI@__cdecl?$AA@ 1001b864     libvcruntime:undname.obj
 0002:0000186c       ??_C@_08GHMPAG@__pascal?$AA@ 1001b86c     libvcruntime:undname.obj
 0002:00001878       ??_C@_09IFJBGAPI@__stdcall?$AA@ 1001b878     libvcruntime:undname.obj
 0002:00001884       ??_C@_0L@NPHFGOKO@__thiscall?$AA@ 1001b884     libvcruntime:undname.obj
 0002:00001890       ??_C@_0L@JMKHOMEK@__fastcall?$AA@ 1001b890     libvcruntime:undname.obj
 0002:0000189c       ??_C@_0N@BCKKPABJ@__vectorcall?$AA@ 1001b89c     libvcruntime:undname.obj
 0002:000018ac       ??_C@_09HIJEGCPM@__clrcall?$AA@ 1001b8ac     libvcruntime:undname.obj
 0002:000018b8       ??_C@_06GHPCKEAG@__eabi?$AA@ 1001b8b8     libvcruntime:undname.obj
 0002:000018c0       ??_C@_07EECFKIPL@__swift?$AA@ 1001b8c0     libvcruntime:undname.obj
 0002:000018c8       ??_C@_07JOMMBBKO@__ptr64?$AA@ 1001b8c8     libvcruntime:undname.obj
 0002:000018d0       ??_C@_0L@PILCLIHE@__restrict?$AA@ 1001b8d0     libvcruntime:undname.obj
 0002:000018dc       ??_C@_0M@GFIIJFMG@__unaligned?$AA@ 1001b8dc     libvcruntime:undname.obj
 0002:000018e8       ??_C@_09DHDLOLLB@restrict?$CI?$AA@ 1001b8e8     libvcruntime:undname.obj
 0002:000018f4       ??_C@_04NIHEBCM@?5new?$AA@ 1001b8f4     libvcruntime:undname.obj
 0002:000018fc       ??_C@_07FPCDHGMM@?5delete?$AA@ 1001b8fc     libvcruntime:undname.obj
 0002:00001904       ??_C@_01NEMOKFLO@?$DN?$AA@ 1001b904     libvcruntime:undname.obj
 0002:00001908       ??_C@_02GPIOPFAK@?$DO?$DO?$AA@ 1001b908     libvcruntime:undname.obj
 0002:0000190c       ??_C@_02FODMEDOG@?$DM?$DM?$AA@ 1001b90c     libvcruntime:undname.obj
 0002:00001910       ??_C@_01DCLJPIOD@?$CB?$AA@ 1001b910     libvcruntime:undname.obj
 0002:00001914       ??_C@_02EGOFBIJA@?$DN?$DN?$AA@ 1001b914     libvcruntime:undname.obj
 0002:00001918       ??_C@_02FDNJECIE@?$CB?$DN?$AA@ 1001b918     libvcruntime:undname.obj
 0002:0000191c       ??_C@_02GPECMEKF@?$FL?$FN?$AA@ 1001b91c     libvcruntime:undname.obj
 0002:00001920       ??_C@_08LHJFAFGD@operator?$AA@ 1001b920     libvcruntime:undname.obj
 0002:0000192c       ??_C@_02HBOOOICD@?9?$DO?$AA@ 1001b92c     libvcruntime:undname.obj
 0002:00001930       ??_C@_01NBENCBCI@?$CK?$AA@ 1001b930     libvcruntime:undname.obj
 0002:00001934       ??_C@_02ECNGHCIF@?$CL?$CL?$AA@ 1001b934     libvcruntime:undname.obj
 0002:00001938       ??_C@_02BAABKJLB@?9?9?$AA@ 1001b938     libvcruntime:undname.obj
 0002:0000193c       ??_C@_01JOAMLHOP@?9?$AA@   1001b93c     libvcruntime:undname.obj
 0002:00001940       ??_C@_01MIFGBAGJ@?$CL?$AA@ 1001b940     libvcruntime:undname.obj
 0002:00001944       ??_C@_01HNPIGOCE@?$CG?$AA@ 1001b944     libvcruntime:undname.obj
 0002:00001948       ??_C@_03MNHNFDLC@?9?$DO?$CK?$AA@ 1001b948     libvcruntime:undname.obj
 0002:0000194c       ??_C@_01KMDKNFGN@?1?$AA@   1001b94c     libvcruntime:undname.obj
 0002:00001950       ??_C@_01FGNFDNOH@?$CF?$AA@ 1001b950     libvcruntime:undname.obj
 0002:00001954       ??_C@_01MNNFJEPP@?$DM?$AA@ 1001b954     libvcruntime:undname.obj
 0002:00001958       ??_C@_02EHCHHCKH@?$DM?$DN?$AA@ 1001b958     libvcruntime:undname.obj
 0002:0000195c       ??_C@_01PPODPGHN@?$DO?$AA@ 1001b95c     libvcruntime:undname.obj
 0002:00001960       ??_C@_02EEKDKGMJ@?$DO?$DN?$AA@ 1001b960     libvcruntime:undname.obj
 0002:00001964       ??_C@_01IHBHIGKO@?0?$AA@   1001b964     libvcruntime:undname.obj
 0002:00001968       ??_C@_02HCKGKOFO@?$CI?$CJ?$AA@ 1001b968     libvcruntime:undname.obj
 0002:0000196c       ??_C@_01PJKLJHI@?$HO?$AA@  1001b96c     libvcruntime:undname.obj
 0002:00001970       ??_C@_01JKBOJNNK@?$FO?$AA@ 1001b970     libvcruntime:undname.obj
 0002:00001974       ??_C@_01DNKMNLPK@?$HM?$AA@ 1001b974     libvcruntime:undname.obj
 0002:00001978       ??_C@_02PPKAJPJL@?$CG?$CG?$AA@ 1001b978     libvcruntime:undname.obj
 0002:0000197c       ??_C@_02NONPIBCD@?$HM?$HM?$AA@ 1001b97c     libvcruntime:undname.obj
 0002:00001980       ??_C@_02FPIMKNGF@?$CK?$DN?$AA@ 1001b980     libvcruntime:undname.obj
 0002:00001984       ??_C@_02FOEOMHFC@?$CL?$DN?$AA@ 1001b984     libvcruntime:undname.obj
 0002:00001988       ??_C@_02FKMDLLOA@?9?$DN?$AA@ 1001b988     libvcruntime:undname.obj
 0002:0000198c       ??_C@_02FJEHGPIO@?1?$DN?$AA@ 1001b98c     libvcruntime:undname.obj
 0002:00001990       ??_C@_02FENAOKFI@?$CF?$DN?$AA@ 1001b990     libvcruntime:undname.obj
 0002:00001994       ??_C@_03IKFCCPFF@?$DO?$DO?$DN?$AA@ 1001b994     libvcruntime:undname.obj
 0002:00001998       ??_C@_03CDNPDDLA@?$DM?$DM?$DN?$AA@ 1001b998     libvcruntime:undname.obj
 0002:0000199c       ??_C@_02FGJGFEAB@?$CG?$DN?$AA@ 1001b99c     libvcruntime:undname.obj
 0002:000019a0       ??_C@_02DHLNPPGH@?$HM?$DN?$AA@ 1001b9a0     libvcruntime:undname.obj
 0002:000019a4       ??_C@_02MHEGNOJ@?$FO?$DN?$AA@ 1001b9a4     libvcruntime:undname.obj
 0002:000019a8       ??_C@_09IFPLHPGF@?$GAvftable?8?$AA@ 1001b9a8     libvcruntime:undname.obj
 0002:000019b4       ??_C@_09BLBHBJP@?$GAvbtable?8?$AA@ 1001b9b4     libvcruntime:undname.obj
 0002:000019c0       ??_C@_07FEEIOKP@?$GAvcall?8?$AA@ 1001b9c0     libvcruntime:undname.obj
 0002:000019c8       ??_C@_08LLFFHHDJ@?$GAtypeof?8?$AA@ 1001b9c8     libvcruntime:undname.obj
 0002:000019d4       ??_C@_0BF@KDPPACIK@?$GAlocal?5static?5guard?8?$AA@ 1001b9d4     libvcruntime:undname.obj
 0002:000019ec       ??_C@_08OBABFOLI@?$GAstring?8?$AA@ 1001b9ec     libvcruntime:undname.obj
 0002:000019f8       ??_C@_0BD@JDLKDPAB@?$GAvbase?5destructor?8?$AA@ 1001b9f8     libvcruntime:undname.obj
 0002:00001a0c       ??_C@_0BN@DEGPLNFK@?$GAvector?5deleting?5destructor?8?$AA@ 1001ba0c     libvcruntime:undname.obj
 0002:00001a2c       ??_C@_0BO@OBMKPJIG@?$GAdefault?5constructor?5closure?8?$AA@ 1001ba2c     libvcruntime:undname.obj
 0002:00001a4c       ??_C@_0BN@IMDCHIKM@?$GAscalar?5deleting?5destructor?8?$AA@ 1001ba4c     libvcruntime:undname.obj
 0002:00001a6c       ??_C@_0BO@PFGOCPJJ@?$GAvector?5constructor?5iterator?8?$AA@ 1001ba6c     libvcruntime:undname.obj
 0002:00001a8c       ??_C@_0BN@LFPFMEDL@?$GAvector?5destructor?5iterator?8?$AA@ 1001ba8c     libvcruntime:undname.obj
 0002:00001aac       ??_C@_0CE@IKBNEHA@?$GAvector?5vbase?5constructor?5iterat@ 1001baac     libvcruntime:undname.obj
 0002:00001ad0       ??_C@_0BL@NILFHHPC@?$GAvirtual?5displacement?5map?8?$AA@ 1001bad0     libvcruntime:undname.obj
 0002:00001aec       ??_C@_0CB@JONCMFFK@?$GAeh?5vector?5constructor?5iterator?8@ 1001baec     libvcruntime:undname.obj
 0002:00001b10       ??_C@_0CA@GCEOPDGL@?$GAeh?5vector?5destructor?5iterator?8?$AA@ 1001bb10     libvcruntime:undname.obj
 0002:00001b30       ??_C@_0CH@OOJPLCPH@?$GAeh?5vector?5vbase?5constructor?5ite@ 1001bb30     libvcruntime:undname.obj
 0002:00001b58       ??_C@_0BL@LLKPOHJI@?$GAcopy?5constructor?5closure?8?$AA@ 1001bb58     libvcruntime:undname.obj
 0002:00001b74       ??_C@_0BA@KBCDOMBN@?$GAudt?5returning?8?$AA@ 1001bb74     libvcruntime:undname.obj
 0002:00001b84       ??_C@_03KLGMFNMG@?$GAEH?$AA@ 1001bb84     libvcruntime:undname.obj
 0002:00001b88       ??_C@_05KHLCHHI@?$GARTTI?$AA@ 1001bb88     libvcruntime:undname.obj
 0002:00001b90       ??_C@_0BA@KKLDJDLB@?$GAlocal?5vftable?8?$AA@ 1001bb90     libvcruntime:undname.obj
 0002:00001ba0       ??_C@_0CE@IIHCMGGL@?$GAlocal?5vftable?5constructor?5closu@ 1001bba0     libvcruntime:undname.obj
 0002:00001bc4       ??_C@_06FHBGPFGH@?5new?$FL?$FN?$AA@ 1001bbc4     libvcruntime:undname.obj
 0002:00001bcc       ??_C@_09LBNFPBCA@?5delete?$FL?$FN?$AA@ 1001bbcc     libvcruntime:undname.obj
 0002:00001bd8       ??_C@_0P@HJKNJFNN@?$GAomni?5callsig?8?$AA@ 1001bbd8     libvcruntime:undname.obj
 0002:00001be8       ??_C@_0BL@CNOONJFP@?$GAplacement?5delete?5closure?8?$AA@ 1001bbe8     libvcruntime:undname.obj
 0002:00001c04       ??_C@_0BN@CKNJLHMB@?$GAplacement?5delete?$FL?$FN?5closure?8?$AA@ 1001bc04     libvcruntime:undname.obj
 0002:00001c24       ??_C@_0CG@CFDHKGGD@?$GAmanaged?5vector?5constructor?5iter@ 1001bc24     libvcruntime:undname.obj
 0002:00001c4c       ??_C@_0CF@IMGKMJNO@?$GAmanaged?5vector?5destructor?5itera@ 1001bc4c     libvcruntime:undname.obj
 0002:00001c74       ??_C@_0CG@HLDDJMAG@?$GAeh?5vector?5copy?5constructor?5iter@ 1001bc74     libvcruntime:undname.obj
 0002:00001c9c       ??_C@_0CM@FCBBDIGB@?$GAeh?5vector?5vbase?5copy?5constructo@ 1001bc9c     libvcruntime:undname.obj
 0002:00001cc8       ??_C@_0BL@CLIPGLGB@?$GAdynamic?5initializer?5for?5?8?$AA@ 1001bcc8     libvcruntime:undname.obj
 0002:00001ce4       ??_C@_0CB@PDBIFEP@?$GAdynamic?5atexit?5destructor?5for?5?8@ 1001bce4     libvcruntime:undname.obj
 0002:00001d08       ??_C@_0CD@CGAJBKEJ@?$GAvector?5copy?5constructor?5iterato@ 1001bd08     libvcruntime:undname.obj
 0002:00001d2c       ??_C@_0CJ@GJELGAMM@?$GAvector?5vbase?5copy?5constructor?5i@ 1001bd2c     libvcruntime:undname.obj
 0002:00001d58       ??_C@_0CL@FGIJHLCE@?$GAmanaged?5vector?5copy?5constructor@ 1001bd58     libvcruntime:undname.obj
 0002:00001d84       ??_C@_0BM@PMGGMLDN@?$GAlocal?5static?5thread?5guard?8?$AA@ 1001bd84     libvcruntime:undname.obj
 0002:00001da0       ??_C@_0N@BDNMDMOL@operator?5?$CC?$CC?5?$AA@ 1001bda0     libvcruntime:undname.obj
 0002:00001db0       ??_C@_0BC@GGEBGALA@operator?5co_await?$AA@ 1001bdb0     libvcruntime:undname.obj
 0002:00001dc4       ??_C@_0BC@DAFEJGAK@?5Type?5Descriptor?8?$AA@ 1001bdc4     libvcruntime:undname.obj
 0002:00001dd8       ??_C@_0BM@LDKODKLH@?5Base?5Class?5Descriptor?5at?5?$CI?$AA@ 1001bdd8     libvcruntime:undname.obj
 0002:00001df4       ??_C@_0BD@LGICGFMM@?5Base?5Class?5Array?8?$AA@ 1001bdf4     libvcruntime:undname.obj
 0002:00001e08       ??_C@_0BN@MECKDCOJ@?5Class?5Hierarchy?5Descriptor?8?$AA@ 1001be08     libvcruntime:undname.obj
 0002:00001e28       ??_C@_0BK@CFCOFLF@?5Complete?5Object?5Locator?8?$AA@ 1001be28     libvcruntime:undname.obj
 0002:00001e44       __pDestructExceptionObject 1001be44     libvcruntime:ehhelpers.obj
 0002:00001e68       _standard_lookup_table     1001be68     libucrt:output.obj
 0002:00001ec4       ??_C@_06OJHGLDPL@?$CInull?$CJ?$AA@ 1001bec4     libucrt:output.obj
 0002:00001ecc       ??_C@_1O@CEDCILHN@?$AA?$CI?$AAn?$AAu?$AAl?$AAl?$AA?$CJ?$AA?$AA@ 1001becc     libucrt:output.obj
 0002:00001ee0       ___acrt_exception_action_table 1001bee0     libucrt:exception_filter.obj
 0002:00001f70       ___acrt_signal_action_table_count 1001bf70     libucrt:exception_filter.obj
 0002:00001f74       ___acrt_signal_action_first_fpe_index 1001bf74     libucrt:exception_filter.obj
 0002:00001f78       ___acrt_signal_action_fpe_count 1001bf78     libucrt:exception_filter.obj
 0002:00001f7c       ??_C@_1BI@BGOHAHKC@?$AAm?$AAs?$AAc?$AAo?$AAr?$AAe?$AAe?$AA?4?$AAd?$AAl?$AAl?$AA?$AA@ 1001bf7c     libucrt:exit.obj
 0002:00001f94       ??_C@_0P@MIGLKIOC@CorExitProcess?$AA@ 1001bf94     libucrt:exit.obj
 0002:00002188       __wctype                   1001c188     libucrt:ctype.obj
 0002:00002390       ___newctype                1001c390     libucrt:ctype.obj
 0002:00002690       ___newclmap                1001c690     libucrt:ctype.obj
 0002:00002810       ___newcumap                1001c810     libucrt:ctype.obj
 0002:00002990       ??_C@_03KOEHGMDN@Sun?$AA@  1001c990     libucrt:nlsdata.obj
 0002:00002994       ??_C@_03PDAGKDH@Mon?$AA@   1001c994     libucrt:nlsdata.obj
 0002:00002998       ??_C@_03NAGEINEP@Tue?$AA@  1001c998     libucrt:nlsdata.obj
 0002:0000299c       ??_C@_03MHOMLAJA@Wed?$AA@  1001c99c     libucrt:nlsdata.obj
 0002:000029a0       ??_C@_03IOFIKPDN@Thu?$AA@  1001c9a0     libucrt:nlsdata.obj
 0002:000029a4       ??_C@_03IDIOELNC@Fri?$AA@  1001c9a4     libucrt:nlsdata.obj
 0002:000029a8       ??_C@_03FEFJNEK@Sat?$AA@   1001c9a8     libucrt:nlsdata.obj
 0002:000029ac       ??_C@_06OOPIFAJ@Sunday?$AA@ 1001c9ac     libucrt:nlsdata.obj
 0002:000029b4       ??_C@_06JLEDEDGH@Monday?$AA@ 1001c9b4     libucrt:nlsdata.obj
 0002:000029bc       ??_C@_07BAAGCFCM@Tuesday?$AA@ 1001c9bc     libucrt:nlsdata.obj
 0002:000029c4       ??_C@_09DLIGFAKA@Wednesday?$AA@ 1001c9c4     libucrt:nlsdata.obj
 0002:000029d0       ??_C@_08HACCIKIA@Thursday?$AA@ 1001c9d0     libucrt:nlsdata.obj
 0002:000029dc       ??_C@_06JECMNKMI@Friday?$AA@ 1001c9dc     libucrt:nlsdata.obj
 0002:000029e4       ??_C@_08INBOOONO@Saturday?$AA@ 1001c9e4     libucrt:nlsdata.obj
 0002:000029f0       ??_C@_03JIHJHPIE@Jan?$AA@  1001c9f0     libucrt:nlsdata.obj
 0002:000029f4       ??_C@_03HJBDCHOM@Feb?$AA@  1001c9f4     libucrt:nlsdata.obj
 0002:000029f8       ??_C@_03ODNJBKGA@Mar?$AA@  1001c9f8     libucrt:nlsdata.obj
 0002:000029fc       ??_C@_03LEOLGMJP@Apr?$AA@  1001c9fc     libucrt:nlsdata.obj
 0002:00002a00       ??_C@_03CNMDKL@May?$AA@    1001ca00     libucrt:nlsdata.obj
 0002:00002a04       ??_C@_03IDFGHECI@Jun?$AA@  1001ca04     libucrt:nlsdata.obj
 0002:00002a08       ??_C@_03LBGABGKK@Jul?$AA@  1001ca08     libucrt:nlsdata.obj
 0002:00002a0c       ??_C@_03IFJFEIGA@Aug?$AA@  1001ca0c     libucrt:nlsdata.obj
 0002:00002a10       ??_C@_03GGCAPAJC@Sep?$AA@  1001ca10     libucrt:nlsdata.obj
 0002:00002a14       ??_C@_03BMAOKBAD@Oct?$AA@  1001ca14     libucrt:nlsdata.obj
 0002:00002a18       ??_C@_03JPJOFNIA@Nov?$AA@  1001ca18     libucrt:nlsdata.obj
 0002:00002a1c       ??_C@_03MKABNOCG@Dec?$AA@  1001ca1c     libucrt:nlsdata.obj
 0002:00002a20       ??_C@_07CGJPFGJA@January?$AA@ 1001ca20     libucrt:nlsdata.obj
 0002:00002a28       ??_C@_08GNJGEPFN@February?$AA@ 1001ca28     libucrt:nlsdata.obj
 0002:00002a34       ??_C@_05HPCKOFNC@March?$AA@ 1001ca34     libucrt:nlsdata.obj
 0002:00002a3c       ??_C@_05DMJDNLEJ@April?$AA@ 1001ca3c     libucrt:nlsdata.obj
 0002:00002a44       ??_C@_04CNLMGBGM@June?$AA@ 1001ca44     libucrt:nlsdata.obj
 0002:00002a4c       ??_C@_04MIEPOIFP@July?$AA@ 1001ca4c     libucrt:nlsdata.obj
 0002:00002a54       ??_C@_06LBBHFDDG@August?$AA@ 1001ca54     libucrt:nlsdata.obj
 0002:00002a5c       ??_C@_09BHHEALKD@September?$AA@ 1001ca5c     libucrt:nlsdata.obj
 0002:00002a68       ??_C@_07JJNFCEND@October?$AA@ 1001ca68     libucrt:nlsdata.obj
 0002:00002a70       ??_C@_08HCHEGEOA@November?$AA@ 1001ca70     libucrt:nlsdata.obj
 0002:00002a7c       ??_C@_08EDHMEBNP@December?$AA@ 1001ca7c     libucrt:nlsdata.obj
 0002:00002a88       ??_C@_02DEDBPAFC@AM?$AA@   1001ca88     libucrt:nlsdata.obj
 0002:00002a8c       ??_C@_02CJNFDJBF@PM?$AA@   1001ca8c     libucrt:nlsdata.obj
 0002:00002a90       ??_C@_08BPBNCDIB@MM?1dd?1yy?$AA@ 1001ca90     libucrt:nlsdata.obj
 0002:00002a9c       ??_C@_0BE@CKGJFCPC@dddd?0?5MMMM?5dd?0?5yyyy?$AA@ 1001ca9c     libucrt:nlsdata.obj
 0002:00002ab0       ??_C@_08JCCMCCIL@HH?3mm?3ss?$AA@ 1001cab0     libucrt:nlsdata.obj
 0002:00002abc       ??_C@_17MBGCMIPB@?$AAS?$AAu?$AAn?$AA?$AA@ 1001cabc     libucrt:nlsdata.obj
 0002:00002ac4       ??_C@_17KBOMKBF@?$AAM?$AAo?$AAn?$AA?$AA@ 1001cac4     libucrt:nlsdata.obj
 0002:00002acc       ??_C@_17BMKGEGOJ@?$AAT?$AAu?$AAe?$AA?$AA@ 1001cacc     libucrt:nlsdata.obj
 0002:00002ad4       ??_C@_17CJEDCEPE@?$AAW?$AAe?$AAd?$AA?$AA@ 1001cad4     libucrt:nlsdata.obj
 0002:00002adc       ??_C@_17PDPHAADD@?$AAT?$AAh?$AAu?$AA?$AA@ 1001cadc     libucrt:nlsdata.obj
 0002:00002ae4       ??_C@_17HFOLPPLP@?$AAF?$AAr?$AAi?$AA?$AA@ 1001cae4     libucrt:nlsdata.obj
 0002:00002aec       ??_C@_17GGIBDPIH@?$AAS?$AAa?$AAt?$AA?$AA@ 1001caec     libucrt:nlsdata.obj
 0002:00002af4       ??_C@_1O@IHNHDHPB@?$AAS?$AAu?$AAn?$AAd?$AAa?$AAy?$AA?$AA@ 1001caf4     libucrt:nlsdata.obj
 0002:00002b04       ??_C@_1O@MMNBFLIA@?$AAM?$AAo?$AAn?$AAd?$AAa?$AAy?$AA?$AA@ 1001cb04     libucrt:nlsdata.obj
 0002:00002b14       ??_C@_1BA@ENFBFFEK@?$AAT?$AAu?$AAe?$AAs?$AAd?$AAa?$AAy?$AA?$AA@ 1001cb14     libucrt:nlsdata.obj
 0002:00002b24       ??_C@_1BE@EBOGMDOH@?$AAW?$AAe?$AAd?$AAn?$AAe?$AAs?$AAd?$AAa?$AAy?$AA?$AA@ 1001cb24     libucrt:nlsdata.obj
 0002:00002b38       ??_C@_1BC@HHMNLIHE@?$AAT?$AAh?$AAu?$AAr?$AAs?$AAd?$AAa?$AAy?$AA?$AA@ 1001cb38     libucrt:nlsdata.obj
 0002:00002b4c       ??_C@_1O@PDICJHAG@?$AAF?$AAr?$AAi?$AAd?$AAa?$AAy?$AA?$AA@ 1001cb4c     libucrt:nlsdata.obj
 0002:00002b5c       ??_C@_1BC@ENMNNPAJ@?$AAS?$AAa?$AAt?$AAu?$AAr?$AAd?$AAa?$AAy?$AA?$AA@ 1001cb5c     libucrt:nlsdata.obj
 0002:00002b70       ??_C@_17DKNBKCHM@?$AAJ?$AAa?$AAn?$AA?$AA@ 1001cb70     libucrt:nlsdata.obj
 0002:00002b78       ??_C@_17LMDJEKJN@?$AAF?$AAe?$AAb?$AA?$AA@ 1001cb78     libucrt:nlsdata.obj
 0002:00002b80       ??_C@_17CKNLEDEC@?$AAM?$AAa?$AAr?$AA?$AA@ 1001cb80     libucrt:nlsdata.obj
 0002:00002b88       ??_C@_17LFPOIHDD@?$AAA?$AAp?$AAr?$AA?$AA@ 1001cb88     libucrt:nlsdata.obj
 0002:00002b90       ??_C@_17PNNKMEED@?$AAM?$AAa?$AAy?$AA?$AA@ 1001cb90     libucrt:nlsdata.obj
 0002:00002b98       ??_C@_17KCJGOCPB@?$AAJ?$AAu?$AAn?$AA?$AA@ 1001cb98     libucrt:nlsdata.obj
 0002:00002ba0       ??_C@_17IJPCKHK@?$AAJ?$AAu?$AAl?$AA?$AA@ 1001cba0     libucrt:nlsdata.obj
 0002:00002ba8       ??_C@_17ICPELBCN@?$AAA?$AAu?$AAg?$AA?$AA@ 1001cba8     libucrt:nlsdata.obj
 0002:00002bb0       ??_C@_17HCHCOKMG@?$AAS?$AAe?$AAp?$AA?$AA@ 1001cbb0     libucrt:nlsdata.obj
 0002:00002bb8       ??_C@_17FNLKOI@?$AAO?$AAc?$AAt?$AA?$AA@ 1001cbb8     libucrt:nlsdata.obj
 0002:00002bc0       ??_C@_17BBDMLCIG@?$AAN?$AAo?$AAv?$AA?$AA@ 1001cbc0     libucrt:nlsdata.obj
 0002:00002bc8       ??_C@_17EGKACKIF@?$AAD?$AAe?$AAc?$AA?$AA@ 1001cbc8     libucrt:nlsdata.obj
 0002:00002bd0       ??_C@_1BA@EFMEIEBA@?$AAJ?$AAa?$AAn?$AAu?$AAa?$AAr?$AAy?$AA?$AA@ 1001cbd0     libucrt:nlsdata.obj
 0002:00002be0       ??_C@_1BC@JGDDFFAM@?$AAF?$AAe?$AAb?$AAr?$AAu?$AAa?$AAr?$AAy?$AA?$AA@ 1001cbe0     libucrt:nlsdata.obj
 0002:00002bf4       ??_C@_1M@IKEENEDF@?$AAM?$AAa?$AAr?$AAc?$AAh?$AA?$AA@ 1001cbf4     libucrt:nlsdata.obj
 0002:00002c00       ??_C@_1M@GJNLMHFD@?$AAA?$AAp?$AAr?$AAi?$AAl?$AA?$AA@ 1001cc00     libucrt:nlsdata.obj
 0002:00002c0c       ??_C@_19EPFLPGAP@?$AAJ?$AAu?$AAn?$AAe?$AA?$AA@ 1001cc0c     libucrt:nlsdata.obj
 0002:00002c18       ??_C@_19BIFMLPCD@?$AAJ?$AAu?$AAl?$AAy?$AA?$AA@ 1001cc18     libucrt:nlsdata.obj
 0002:00002c24       ??_C@_1O@PAHLKOAC@?$AAA?$AAu?$AAg?$AAu?$AAs?$AAt?$AA?$AA@ 1001cc24     libucrt:nlsdata.obj
 0002:00002c34       ??_C@_1BE@DKAAMBJL@?$AAS?$AAe?$AAp?$AAt?$AAe?$AAm?$AAb?$AAe?$AAr?$AA?$AA@ 1001cc34     libucrt:nlsdata.obj
 0002:00002c48       ??_C@_1BA@EPANDLNG@?$AAO?$AAc?$AAt?$AAo?$AAb?$AAe?$AAr?$AA?$AA@ 1001cc48     libucrt:nlsdata.obj
 0002:00002c58       ??_C@_1BC@BGLIFPF@?$AAN?$AAo?$AAv?$AAe?$AAm?$AAb?$AAe?$AAr?$AA?$AA@ 1001cc58     libucrt:nlsdata.obj
 0002:00002c6c       ??_C@_1BC@FEMKIFH@?$AAD?$AAe?$AAc?$AAe?$AAm?$AAb?$AAe?$AAr?$AA?$AA@ 1001cc6c     libucrt:nlsdata.obj
 0002:00002c80       ??_C@_15ODEHAHHF@?$AAA?$AAM?$AA?$AA@ 1001cc80     libucrt:nlsdata.obj
 0002:00002c88       ??_C@_15CLMNNGEL@?$AAP?$AAM?$AA?$AA@ 1001cc88     libucrt:nlsdata.obj
 0002:00002c90       ??_C@_1BC@IEBCMHCM@?$AAM?$AAM?$AA?1?$AAd?$AAd?$AA?1?$AAy?$AAy?$AA?$AA@ 1001cc90     libucrt:nlsdata.obj
 0002:00002ca4       ??_C@_1CI@KNAKOEBC@?$AAd?$AAd?$AAd?$AAd?$AA?0?$AA?5?$AAM?$AAM?$AAM?$AAM?$AA?5?$AAd?$AAd?$AA?0?$AA?5?$AAy?$AAy?$AAy?$AAy?$AA?$AA@ 1001cca4     libucrt:nlsdata.obj
 0002:00002ccc       ??_C@_1BC@GDGBMEMK@?$AAH?$AAH?$AA?3?$AAm?$AAm?$AA?3?$AAs?$AAs?$AA?$AA@ 1001cccc     libucrt:nlsdata.obj
 0002:00002ce0       ??_C@_1M@BMHNFIME@?$AAe?$AAn?$AA?9?$AAU?$AAS?$AA?$AA@ 1001cce0     libucrt:nlsdata.obj
 0002:00002cf0       ___lc_time_c               1001ccf0     libucrt:nlsdata.obj
 0002:00002e54       ??_C@_03OEIAHPBN@INF?$AA@  1001ce54     libucrt:cvt.obj
 0002:00002e58       ??_C@_03OJHLLCGB@inf?$AA@  1001ce58     libucrt:cvt.obj
 0002:00002e5c       ??_C@_03LKNCIKJB@NAN?$AA@  1001ce5c     libucrt:cvt.obj
 0002:00002e60       ??_C@_03LHCJEHON@nan?$AA@  1001ce60     libucrt:cvt.obj
 0002:00002e64       ??_C@_09OFJJIMPC@NAN?$CISNAN?$CJ?$AA@ 1001ce64     libucrt:cvt.obj
 0002:00002e70       ??_C@_09IPFBKMDL@nan?$CIsnan?$CJ?$AA@ 1001ce70     libucrt:cvt.obj
 0002:00002e7c       ??_C@_08IKHNHAJ@NAN?$CIIND?$CJ?$AA@ 1001ce7c     libucrt:cvt.obj
 0002:00002e88       ??_C@_08OFCDMILK@nan?$CIind?$CJ?$AA@ 1001ce88     libucrt:cvt.obj
 0002:00002e94       ??_C@_05KLBDPFGC@e?$CL000?$AA@ 1001ce94     libucrt:cvt.obj
 0002:00002ef0       ??_C@_1EG@CNNIPFIM@?$AAa?$AAp?$AAi?$AA?9?$AAm?$AAs?$AA?9?$AAw?$AAi?$AAn?$AA?9?$AAa?$AAp?$AAp?$AAm?$AAo?$AAd?$AAe?$AAl?$AA?9?$AAr?$AAu?$AAn?$AAt?$AAi?$AAm?$AAe?$AA?9?$AAl?$AA1?$AA?9?$AA1@ 1001cef0     libucrt:winapi_thunks.obj
 0002:00002f38       ??_C@_1EA@JGEFHKEI@?$AAa?$AAp?$AAi?$AA?9?$AAm?$AAs?$AA?9?$AAw?$AAi?$AAn?$AA?9?$AAc?$AAo?$AAr?$AAe?$AA?9?$AAd?$AAa?$AAt?$AAe?$AAt?$AAi?$AAm?$AAe?$AA?9?$AAl?$AA1?$AA?9?$AA1?$AA?9?$AA1?$AA?$AA@ 1001cf38     libucrt:winapi_thunks.obj
 0002:00002f78       ??_C@_1DI@GCIAAENM@?$AAa?$AAp?$AAi?$AA?9?$AAm?$AAs?$AA?9?$AAw?$AAi?$AAn?$AA?9?$AAc?$AAo?$AAr?$AAe?$AA?9?$AAf?$AAi?$AAl?$AAe?$AA?9?$AAl?$AA2?$AA?9?$AA1?$AA?9?$AA1?$AA?$AA@ 1001cf78     libucrt:winapi_thunks.obj
 0002:00002fb0       ??_C@_1EI@MPIAOHOC@?$AAa?$AAp?$AAi?$AA?9?$AAm?$AAs?$AA?9?$AAw?$AAi?$AAn?$AA?9?$AAc?$AAo?$AAr?$AAe?$AA?9?$AAl?$AAo?$AAc?$AAa?$AAl?$AAi?$AAz?$AAa?$AAt?$AAi?$AAo?$AAn?$AA?9?$AAl?$AA1?$AA?9@ 1001cfb0     libucrt:winapi_thunks.obj
 0002:00002ff8       ??_C@_1FK@FPHCKFIE@?$AAa?$AAp?$AAi?$AA?9?$AAm?$AAs?$AA?9?$AAw?$AAi?$AAn?$AA?9?$AAc?$AAo?$AAr?$AAe?$AA?9?$AAl?$AAo?$AAc?$AAa?$AAl?$AAi?$AAz?$AAa?$AAt?$AAi?$AAo?$AAn?$AA?9?$AAo?$AAb?$AAs@ 1001cff8     libucrt:winapi_thunks.obj
 0002:00003058       ??_C@_1EM@DILCGIIO@?$AAa?$AAp?$AAi?$AA?9?$AAm?$AAs?$AA?9?$AAw?$AAi?$AAn?$AA?9?$AAc?$AAo?$AAr?$AAe?$AA?9?$AAp?$AAr?$AAo?$AAc?$AAe?$AAs?$AAs?$AAt?$AAh?$AAr?$AAe?$AAa?$AAd?$AAs?$AA?9?$AAl@ 1001d058     libucrt:winapi_thunks.obj
 0002:000030a4       ??_C@_1DM@LNCGDDPN@?$AAa?$AAp?$AAi?$AA?9?$AAm?$AAs?$AA?9?$AAw?$AAi?$AAn?$AA?9?$AAc?$AAo?$AAr?$AAe?$AA?9?$AAs?$AAt?$AAr?$AAi?$AAn?$AAg?$AA?9?$AAl?$AA1?$AA?9?$AA1?$AA?9?$AA0?$AA?$AA@ 1001d0a4     libucrt:winapi_thunks.obj
 0002:000030e0       ??_C@_1DO@FPAPJEMD@?$AAa?$AAp?$AAi?$AA?9?$AAm?$AAs?$AA?9?$AAw?$AAi?$AAn?$AA?9?$AAc?$AAo?$AAr?$AAe?$AA?9?$AAs?$AAy?$AAs?$AAi?$AAn?$AAf?$AAo?$AA?9?$AAl?$AA1?$AA?9?$AA2?$AA?9?$AA1?$AA?$AA@ 1001d0e0     libucrt:winapi_thunks.obj
 0002:00003120       ??_C@_1DK@NDHNAHIO@?$AAa?$AAp?$AAi?$AA?9?$AAm?$AAs?$AA?9?$AAw?$AAi?$AAn?$AA?9?$AAc?$AAo?$AAr?$AAe?$AA?9?$AAw?$AAi?$AAn?$AAr?$AAt?$AA?9?$AAl?$AA1?$AA?9?$AA1?$AA?9?$AA0?$AA?$AA@ 1001d120     libucrt:winapi_thunks.obj
 0002:0000315c       ??_C@_1DM@KGHDGBCM@?$AAa?$AAp?$AAi?$AA?9?$AAm?$AAs?$AA?9?$AAw?$AAi?$AAn?$AA?9?$AAc?$AAo?$AAr?$AAe?$AA?9?$AAx?$AAs?$AAt?$AAa?$AAt?$AAe?$AA?9?$AAl?$AA2?$AA?9?$AA1?$AA?9?$AA0?$AA?$AA@ 1001d15c     libucrt:winapi_thunks.obj
 0002:00003198       ??_C@_1EO@IJIOEFOH@?$AAa?$AAp?$AAi?$AA?9?$AAm?$AAs?$AA?9?$AAw?$AAi?$AAn?$AA?9?$AAr?$AAt?$AAc?$AAo?$AAr?$AAe?$AA?9?$AAn?$AAt?$AAu?$AAs?$AAe?$AAr?$AA?9?$AAw?$AAi?$AAn?$AAd?$AAo?$AAw?$AA?9@ 1001d198     libucrt:winapi_thunks.obj
 0002:000031e8       ??_C@_1FG@HHGEKANL@?$AAa?$AAp?$AAi?$AA?9?$AAm?$AAs?$AA?9?$AAw?$AAi?$AAn?$AA?9?$AAs?$AAe?$AAc?$AAu?$AAr?$AAi?$AAt?$AAy?$AA?9?$AAs?$AAy?$AAs?$AAt?$AAe?$AAm?$AAf?$AAu?$AAn?$AAc?$AAt?$AAi@ 1001d1e8     libucrt:winapi_thunks.obj
 0002:00003240       ??_C@_1FG@NCKKOLKO@?$AAe?$AAx?$AAt?$AA?9?$AAm?$AAs?$AA?9?$AAw?$AAi?$AAn?$AA?9?$AAk?$AAe?$AAr?$AAn?$AAe?$AAl?$AA3?$AA2?$AA?9?$AAp?$AAa?$AAc?$AAk?$AAa?$AAg?$AAe?$AA?9?$AAc?$AAu?$AAr?$AAr@ 1001d240     libucrt:winapi_thunks.obj
 0002:00003298       ??_C@_1EG@DBIOJECG@?$AAe?$AAx?$AAt?$AA?9?$AAm?$AAs?$AA?9?$AAw?$AAi?$AAn?$AA?9?$AAn?$AAt?$AAu?$AAs?$AAe?$AAr?$AA?9?$AAd?$AAi?$AAa?$AAl?$AAo?$AAg?$AAb?$AAo?$AAx?$AA?9?$AAl?$AA1?$AA?9?$AA1@ 1001d298     libucrt:winapi_thunks.obj
 0002:000032e0       ??_C@_1EO@FIHMJCLF@?$AAe?$AAx?$AAt?$AA?9?$AAm?$AAs?$AA?9?$AAw?$AAi?$AAn?$AA?9?$AAn?$AAt?$AAu?$AAs?$AAe?$AAr?$AA?9?$AAw?$AAi?$AAn?$AAd?$AAo?$AAw?$AAs?$AAt?$AAa?$AAt?$AAi?$AAo?$AAn?$AA?9@ 1001d2e0     libucrt:winapi_thunks.obj
 0002:00003330       ??_C@_1BC@DNHGCMLG@?$AAa?$AAd?$AAv?$AAa?$AAp?$AAi?$AA3?$AA2?$AA?$AA@ 1001d330     libucrt:winapi_thunks.obj
 0002:00003344       ??_C@_1O@BCCLBEOE@?$AAu?$AAs?$AAe?$AAr?$AA3?$AA2?$AA?$AA@ 1001d344     libucrt:winapi_thunks.obj
 0002:0000337c       ??_C@_0BE@JOGNEJCI@GetCurrentPackageId?$AA@ 1001d37c     libucrt:winapi_thunks.obj
 0002:000033a0       ??_C@_0O@KKBNKAPF@LCMapStringEx?$AA@ 1001d3a0     libucrt:winapi_thunks.obj
 0002:000033b8       ??_C@_0BB@HBDEELFH@LocaleNameToLCID?$AA@ 1001d3b8     libucrt:winapi_thunks.obj
 0002:000033dc       ??_C@_1M@HPNHIDJI@?$AAj?$AAa?$AA?9?$AAJ?$AAP?$AA?$AA@ 1001d3dc     libucrt:mbctype.obj
 0002:000033e8       ??_C@_1M@BIBDDEMK@?$AAz?$AAh?$AA?9?$AAC?$AAN?$AA?$AA@ 1001d3e8     libucrt:mbctype.obj
 0002:000033f4       ??_C@_1M@JLOOOEGK@?$AAk?$AAo?$AA?9?$AAK?$AAR?$AA?$AA@ 1001d3f4     libucrt:mbctype.obj
 0002:00003400       ??_C@_1M@CLNBBOPM@?$AAz?$AAh?$AA?9?$AAT?$AAW?$AA?$AA@ 1001d400     libucrt:mbctype.obj
 0002:0000340c       ??_C@_15PJPFLCCM@?$AAu?$AAk?$AA?$AA@ 1001d40c     libucrt:get_qualified_locale.obj
 0002:00003418       ?large_power_data@?1??multiply_by_power_of_ten@__crt_strtox@@YA_NAAUbig_integer@2@I@Z@4QBIB 1001d418     libucrt:cfout.obj
 0002:00003d20       ?large_power_indices@?1??multiply_by_power_of_ten@__crt_strtox@@YA_NAAUbig_integer@2@I@Z@4QBUunpack_index@?1??12@YA_N0I@Z@B 1001dd20     libucrt:cfout.obj
 0002:00003db8       ?small_powers_of_ten@?6??multiply_by_power_of_ten@__crt_strtox@@YA_NAAUbig_integer@2@I@Z@4QBIB 1001ddb8     libucrt:cfout.obj
 0002:00003ddc       ??_C@_01GBGANLPD@0?$AA@    1001dddc     libucrt:cfout.obj
 0002:00003de0       ??_C@_05DNEBIAHO@1?$CDINF?$AA@ 1001dde0     libucrt:cfout.obj
 0002:00003de8       ??_C@_06IMKFLFPG@1?$CDQNAN?$AA@ 1001dde8     libucrt:cfout.obj
 0002:00003df0       ??_C@_06PGGFOGJG@1?$CDSNAN?$AA@ 1001ddf0     libucrt:cfout.obj
 0002:00003df8       ??_C@_05PHHOCPM@1?$CDIND?$AA@ 1001ddf8     libucrt:cfout.obj
 0002:00004520       ??_C@_15EMKDOKLE@?$AAa?$AAr?$AA?$AA@ 1001e520     libucrt:lcidtoname_downlevel.obj
 0002:00004528       ??_C@_15KNPADPLH@?$AAb?$AAg?$AA?$AA@ 1001e528     libucrt:lcidtoname_downlevel.obj
 0002:00004530       ??_C@_15EDMHLDMO@?$AAc?$AAa?$AA?$AA@ 1001e530     libucrt:lcidtoname_downlevel.obj
 0002:00004538       ??_C@_1O@BPEAJADD@?$AAz?$AAh?$AA?9?$AAC?$AAH?$AAS?$AA?$AA@ 1001e538     libucrt:lcidtoname_downlevel.obj
 0002:00004548       ??_C@_15LJNHCMNK@?$AAc?$AAs?$AA?$AA@ 1001e548     libucrt:lcidtoname_downlevel.obj
 0002:00004550       ??_C@_15FOMCIDHG@?$AAd?$AAa?$AA?$AA@ 1001e550     libucrt:lcidtoname_downlevel.obj
 0002:00004558       ??_C@_15NBKABECB@?$AAd?$AAe?$AA?$AA@ 1001e558     libucrt:lcidtoname_downlevel.obj
 0002:00004560       ??_C@_15GHPEIIAO@?$AAe?$AAl?$AA?$AA@ 1001e560     libucrt:lcidtoname_downlevel.obj
 0002:00004568       ??_C@_15MNPNEAIF@?$AAe?$AAn?$AA?$AA@ 1001e568     libucrt:lcidtoname_downlevel.obj
 0002:00004570       ??_C@_15GPIOMPMH@?$AAe?$AAs?$AA?$AA@ 1001e570     libucrt:lcidtoname_downlevel.obj
 0002:00004578       ??_C@_15NGLOAKJC@?$AAf?$AAi?$AA?$AA@ 1001e578     libucrt:lcidtoname_downlevel.obj
 0002:00004580       ??_C@_15FBKGNKAM@?$AAf?$AAr?$AA?$AA@ 1001e580     libucrt:lcidtoname_downlevel.obj
 0002:00004588       ??_C@_15KGGCNEFK@?$AAh?$AAe?$AA?$AA@ 1001e588     libucrt:lcidtoname_downlevel.obj
 0002:00004590       ??_C@_15PGHLIDMF@?$AAh?$AAu?$AA?$AA@ 1001e590     libucrt:lcidtoname_downlevel.obj
 0002:00004598       ??_C@_15BIEMAPLM@?$AAi?$AAs?$AA?$AA@ 1001e598     libucrt:lcidtoname_downlevel.obj
 0002:000045a0       ??_C@_15IFJLDHAF@?$AAi?$AAt?$AA?$AA@ 1001e5a0     libucrt:lcidtoname_downlevel.obj
 0002:000045a8       ??_C@_15GEMIOCAG@?$AAj?$AAa?$AA?$AA@ 1001e5a8     libucrt:lcidtoname_downlevel.obj
 0002:000045b0       ??_C@_15EPELEGJA@?$AAk?$AAo?$AA?$AA@ 1001e5b0     libucrt:lcidtoname_downlevel.obj
 0002:000045b8       ??_C@_15NDDHIMN@?$AAn?$AAl?$AA?$AA@ 1001e5b8     libucrt:lcidtoname_downlevel.obj
 0002:000045c0       ??_C@_15BPIGNHCD@?$AAn?$AAo?$AA?$AA@ 1001e5c0     libucrt:lcidtoname_downlevel.obj
 0002:000045c8       ??_C@_15DEOPBLCG@?$AAp?$AAl?$AA?$AA@ 1001e5c8     libucrt:lcidtoname_downlevel.obj
 0002:000045d0       ??_C@_15KBECGEFG@?$AAp?$AAt?$AA?$AA@ 1001e5d0     libucrt:lcidtoname_downlevel.obj
 0002:000045d8       ??_C@_15GLJCBFMD@?$AAr?$AAo?$AA?$AA@ 1001e5d8     libucrt:lcidtoname_downlevel.obj
 0002:000045e0       ??_C@_15FEDGKCDI@?$AAr?$AAu?$AA?$AA@ 1001e5e0     libucrt:lcidtoname_downlevel.obj
 0002:000045e8       ??_C@_15GLKMLLHM@?$AAh?$AAr?$AA?$AA@ 1001e5e8     libucrt:lcidtoname_downlevel.obj
 0002:000045f0       ??_C@_15CPKMFBDB@?$AAs?$AAk?$AA?$AA@ 1001e5f0     libucrt:lcidtoname_downlevel.obj
 0002:000045f8       ??_C@_15BAAIOGMK@?$AAs?$AAq?$AA?$AA@ 1001e5f8     libucrt:lcidtoname_downlevel.obj
 0002:00004600       ??_C@_15INNPNOHD@?$AAs?$AAv?$AA?$AA@ 1001e600     libucrt:lcidtoname_downlevel.obj
 0002:00004608       ??_C@_15CABMMOGH@?$AAt?$AAh?$AA?$AA@ 1001e608     libucrt:lcidtoname_downlevel.obj
 0002:00004610       ??_C@_15BPLIHJJM@?$AAt?$AAr?$AA?$AA@ 1001e610     libucrt:lcidtoname_downlevel.obj
 0002:00004618       ??_C@_15NEOEKKDJ@?$AAu?$AAr?$AA?$AA@ 1001e618     libucrt:lcidtoname_downlevel.obj
 0002:00004620       ??_C@_15NFICGAJK@?$AAi?$AAd?$AA?$AA@ 1001e620     libucrt:lcidtoname_downlevel.obj
 0002:00004628       ??_C@_15HPJPHDM@?$AAb?$AAe?$AA?$AA@ 1001e628     libucrt:lcidtoname_downlevel.obj
 0002:00004630       ??_C@_15LCHLGJII@?$AAs?$AAl?$AA?$AA@ 1001e630     libucrt:lcidtoname_downlevel.obj
 0002:00004638       ??_C@_15PCFJPHHO@?$AAe?$AAt?$AA?$AA@ 1001e638     libucrt:lcidtoname_downlevel.obj
 0002:00004640       ??_C@_15HPFPGODN@?$AAl?$AAv?$AA?$AA@ 1001e640     libucrt:lcidtoname_downlevel.obj
 0002:00004648       ??_C@_15NFFGKGLG@?$AAl?$AAt?$AA?$AA@ 1001e648     libucrt:lcidtoname_downlevel.obj
 0002:00004650       ??_C@_15BDAKCCHN@?$AAf?$AAa?$AA?$AA@ 1001e650     libucrt:lcidtoname_downlevel.obj
 0002:00004658       ??_C@_15NFGIAIAJ@?$AAv?$AAi?$AA?$AA@ 1001e658     libucrt:lcidtoname_downlevel.obj
 0002:00004660       ??_C@_15LMKNDMHN@?$AAh?$AAy?$AA?$AA@ 1001e660     libucrt:lcidtoname_downlevel.obj
 0002:00004668       ??_C@_15IJBHMCFL@?$AAa?$AAz?$AA?$AA@ 1001e668     libucrt:lcidtoname_downlevel.obj
 0002:00004670       ??_C@_15EKOFJABL@?$AAe?$AAu?$AA?$AA@ 1001e670     libucrt:lcidtoname_downlevel.obj
 0002:00004678       ??_C@_15BGHADCNK@?$AAm?$AAk?$AA?$AA@ 1001e678     libucrt:lcidtoname_downlevel.obj
 0002:00004680       ??_C@_15JDNICKHM@?$AAa?$AAf?$AA?$AA@ 1001e680     libucrt:lcidtoname_downlevel.obj
 0002:00004688       ??_C@_15KPJEDBKD@?$AAk?$AAa?$AA?$AA@ 1001e688     libucrt:lcidtoname_downlevel.obj
 0002:00004690       ??_C@_15PDNFFFEO@?$AAf?$AAo?$AA?$AA@ 1001e690     libucrt:lcidtoname_downlevel.obj
 0002:00004698       ??_C@_15OMLEGLOC@?$AAh?$AAi?$AA?$AA@ 1001e698     libucrt:lcidtoname_downlevel.obj
 0002:000046a0       ??_C@_15IDNNENKK@?$AAm?$AAs?$AA?$AA@ 1001e6a0     libucrt:lcidtoname_downlevel.obj
 0002:000046a8       ??_C@_15MACJNBMH@?$AAk?$AAk?$AA?$AA@ 1001e6a8     libucrt:lcidtoname_downlevel.obj
 0002:000046b0       ??_C@_15DKDJEOND@?$AAk?$AAy?$AA?$AA@ 1001e6b0     libucrt:lcidtoname_downlevel.obj
 0002:000046b8       ??_C@_15DFGDLJBG@?$AAs?$AAw?$AA?$AA@ 1001e6b8     libucrt:lcidtoname_downlevel.obj
 0002:000046c0       ??_C@_15BBFAICNG@?$AAu?$AAz?$AA?$AA@ 1001e6c0     libucrt:lcidtoname_downlevel.obj
 0002:000046c8       ??_C@_15DKNDCGEA@?$AAt?$AAt?$AA?$AA@ 1001e6c8     libucrt:lcidtoname_downlevel.obj
 0002:000046d0       ??_C@_15MGIFMDPL@?$AAp?$AAa?$AA?$AA@ 1001e6d0     libucrt:lcidtoname_downlevel.obj
 0002:000046d8       ??_C@_15HCNDBBA@?$AAg?$AAu?$AA?$AA@ 1001e6d8     libucrt:lcidtoname_downlevel.obj
 0002:000046e0       ??_C@_15FNBEIBON@?$AAt?$AAa?$AA?$AA@ 1001e6e0     libucrt:lcidtoname_downlevel.obj
 0002:000046e8       ??_C@_15NCHGBGLK@?$AAt?$AAe?$AA?$AA@ 1001e6e8     libucrt:lcidtoname_downlevel.obj
 0002:000046f0       ??_C@_15PHPHCBPF@?$AAk?$AAn?$AA?$AA@ 1001e6f0     libucrt:lcidtoname_downlevel.obj
 0002:000046f8       ??_C@_15DLGBCKMP@?$AAm?$AAr?$AA?$AA@ 1001e6f8     libucrt:lcidtoname_downlevel.obj
 0002:00004700       ??_C@_15EABBLBFF@?$AAs?$AAa?$AA?$AA@ 1001e700     libucrt:lcidtoname_downlevel.obj
 0002:00004708       ??_C@_15CBKOMCOI@?$AAm?$AAn?$AA?$AA@ 1001e708     libucrt:lcidtoname_downlevel.obj
 0002:00004710       ??_C@_15CKDMCJAF@?$AAg?$AAl?$AA?$AA@ 1001e710     libucrt:lcidtoname_downlevel.obj
 0002:00004718       ??_C@_17CNJFBPG@?$AAk?$AAo?$AAk?$AA?$AA@ 1001e718     libucrt:lcidtoname_downlevel.obj
 0002:00004720       ??_C@_17FFBJICPL@?$AAs?$AAy?$AAr?$AA?$AA@ 1001e720     libucrt:lcidtoname_downlevel.obj
 0002:00004728       ??_C@_17KPNDCPAF@?$AAd?$AAi?$AAv?$AA?$AA@ 1001e728     libucrt:lcidtoname_downlevel.obj
 0002:00004730       ??_C@_1M@OKAHONE@?$AAa?$AAr?$AA?9?$AAS?$AAA?$AA?$AA@ 1001e730     libucrt:lcidtoname_downlevel.obj
 0002:0000473c       ??_C@_1M@FFFIGIGK@?$AAb?$AAg?$AA?9?$AAB?$AAG?$AA?$AA@ 1001e73c     libucrt:lcidtoname_downlevel.obj
 0002:00004748       ??_C@_1M@BJNKEDC@?$AAc?$AAa?$AA?9?$AAE?$AAS?$AA?$AA@ 1001e748     libucrt:lcidtoname_downlevel.obj
 0002:00004754       ??_C@_1M@IJJHFJHA@?$AAc?$AAs?$AA?9?$AAC?$AAZ?$AA?$AA@ 1001e754     libucrt:lcidtoname_downlevel.obj
 0002:00004760       ??_C@_1M@CLPEOBGI@?$AAd?$AAa?$AA?9?$AAD?$AAK?$AA?$AA@ 1001e760     libucrt:lcidtoname_downlevel.obj
 0002:0000476c       ??_C@_1M@MCMADGCB@?$AAd?$AAe?$AA?9?$AAD?$AAE?$AA?$AA@ 1001e76c     libucrt:lcidtoname_downlevel.obj
 0002:00004778       ??_C@_1M@OOCKEMAM@?$AAe?$AAl?$AA?9?$AAG?$AAR?$AA?$AA@ 1001e778     libucrt:lcidtoname_downlevel.obj
 0002:00004784       ??_C@_1M@DDNJFGID@?$AAf?$AAi?$AA?9?$AAF?$AAI?$AA?$AA@ 1001e784     libucrt:lcidtoname_downlevel.obj
 0002:00004790       ??_C@_1M@GLIPPMAC@?$AAf?$AAr?$AA?9?$AAF?$AAR?$AA?$AA@ 1001e790     libucrt:lcidtoname_downlevel.obj
 0002:0000479c       ??_C@_1M@GFMCHPE@?$AAh?$AAe?$AA?9?$AAI?$AAL?$AA?$AA@ 1001e79c     libucrt:lcidtoname_downlevel.obj
 0002:000047a8       ??_C@_1M@MHLPGNKM@?$AAh?$AAu?$AA?9?$AAH?$AAU?$AA?$AA@ 1001e7a8     libucrt:lcidtoname_downlevel.obj
 0002:000047b4       ??_C@_1M@LPDDNNPN@?$AAi?$AAs?$AA?9?$AAI?$AAS?$AA?$AA@ 1001e7b4     libucrt:lcidtoname_downlevel.obj
 0002:000047c0       ??_C@_1M@MADIPODN@?$AAi?$AAt?$AA?9?$AAI?$AAT?$AA?$AA@ 1001e7c0     libucrt:lcidtoname_downlevel.obj
 0002:000047cc       ??_C@_1M@IHBJJGG@?$AAn?$AAl?$AA?9?$AAN?$AAL?$AA?$AA@ 1001e7cc     libucrt:lcidtoname_downlevel.obj
 0002:000047d8       ??_C@_1M@EANAGDL@?$AAn?$AAb?$AA?9?$AAN?$AAO?$AA?$AA@ 1001e7d8     libucrt:lcidtoname_downlevel.obj
 0002:000047e4       ??_C@_1M@NEIEMEGP@?$AAp?$AAl?$AA?9?$AAP?$AAL?$AA?$AA@ 1001e7e4     libucrt:lcidtoname_downlevel.obj
 0002:000047f0       ??_C@_1M@BOCFIGEP@?$AAp?$AAt?$AA?9?$AAB?$AAR?$AA?$AA@ 1001e7f0     libucrt:lcidtoname_downlevel.obj
 0002:000047fc       ??_C@_1M@IMPFOPBG@?$AAr?$AAo?$AA?9?$AAR?$AAO?$AA?$AA@ 1001e7fc     libucrt:lcidtoname_downlevel.obj
 0002:00004808       ??_C@_1M@IDNNEJMM@?$AAr?$AAu?$AA?9?$AAR?$AAU?$AA?$AA@ 1001e808     libucrt:lcidtoname_downlevel.obj
 0002:00004814       ??_C@_1M@LILEEOGM@?$AAh?$AAr?$AA?9?$AAH?$AAR?$AA?$AA@ 1001e814     libucrt:lcidtoname_downlevel.obj
 0002:00004820       ??_C@_1M@FKIFEHPB@?$AAs?$AAk?$AA?9?$AAS?$AAK?$AA?$AA@ 1001e820     libucrt:lcidtoname_downlevel.obj
 0002:0000482c       ??_C@_1M@LJMAMNPJ@?$AAs?$AAq?$AA?9?$AAA?$AAL?$AA?$AA@ 1001e82c     libucrt:lcidtoname_downlevel.obj
 0002:00004838       ??_C@_1M@GIAKDKJK@?$AAs?$AAv?$AA?9?$AAS?$AAE?$AA?$AA@ 1001e838     libucrt:lcidtoname_downlevel.obj
 0002:00004844       ??_C@_1M@MKJKIKCL@?$AAt?$AAh?$AA?9?$AAT?$AAH?$AA?$AA@ 1001e844     libucrt:lcidtoname_downlevel.obj
 0002:00004850       ??_C@_1M@MFLCCMPB@?$AAt?$AAr?$AA?9?$AAT?$AAR?$AA?$AA@ 1001e850     libucrt:lcidtoname_downlevel.obj
 0002:0000485c       ??_C@_1M@OIJHDKJN@?$AAu?$AAr?$AA?9?$AAP?$AAK?$AA?$AA@ 1001e85c     libucrt:lcidtoname_downlevel.obj
 0002:00004868       ??_C@_1M@LHIPCIEK@?$AAi?$AAd?$AA?9?$AAI?$AAD?$AA?$AA@ 1001e868     libucrt:lcidtoname_downlevel.obj
 0002:00004874       ??_C@_1M@MFMOBGI@?$AAu?$AAk?$AA?9?$AAU?$AAA?$AA?$AA@ 1001e874     libucrt:lcidtoname_downlevel.obj
 0002:00004880       ??_C@_1M@OBGLJIPL@?$AAb?$AAe?$AA?9?$AAB?$AAY?$AA?$AA@ 1001e880     libucrt:lcidtoname_downlevel.obj
 0002:0000488c       ??_C@_1M@BCFAJEAD@?$AAs?$AAl?$AA?9?$AAS?$AAI?$AA?$AA@ 1001e88c     libucrt:lcidtoname_downlevel.obj
 0002:00004898       ??_C@_1M@FKFFEDDN@?$AAe?$AAt?$AA?9?$AAE?$AAE?$AA?$AA@ 1001e898     libucrt:lcidtoname_downlevel.obj
 0002:000048a4       ??_C@_1M@KGKKAACI@?$AAl?$AAv?$AA?9?$AAL?$AAV?$AA?$AA@ 1001e8a4     libucrt:lcidtoname_downlevel.obj
 0002:000048b0       ??_C@_1M@IFGBIJO@?$AAl?$AAt?$AA?9?$AAL?$AAT?$AA?$AA@ 1001e8b0     libucrt:lcidtoname_downlevel.obj
 0002:000048bc       ??_C@_1M@FGEAHEDM@?$AAf?$AAa?$AA?9?$AAI?$AAR?$AA?$AA@ 1001e8bc     libucrt:lcidtoname_downlevel.obj
 0002:000048c8       ??_C@_1M@KBMAIBFN@?$AAv?$AAi?$AA?9?$AAV?$AAN?$AA?$AA@ 1001e8c8     libucrt:lcidtoname_downlevel.obj
 0002:000048d4       ??_C@_1M@GPCBKDJK@?$AAh?$AAy?$AA?9?$AAA?$AAM?$AA?$AA@ 1001e8d4     libucrt:lcidtoname_downlevel.obj
 0002:000048e0       ??_C@_1BG@BECMDDJB@?$AAa?$AAz?$AA?9?$AAA?$AAZ?$AA?9?$AAL?$AAa?$AAt?$AAn?$AA?$AA@ 1001e8e0     libucrt:lcidtoname_downlevel.obj
 0002:000048f8       ??_C@_1M@MAOFCAEA@?$AAe?$AAu?$AA?9?$AAE?$AAS?$AA?$AA@ 1001e8f8     libucrt:lcidtoname_downlevel.obj
 0002:00004904       ??_C@_1M@IGHABKPI@?$AAm?$AAk?$AA?9?$AAM?$AAK?$AA?$AA@ 1001e904     libucrt:lcidtoname_downlevel.obj
 0002:00004910       ??_C@_1M@IAIGNEJG@?$AAt?$AAn?$AA?9?$AAZ?$AAA?$AA?$AA@ 1001e910     libucrt:lcidtoname_downlevel.obj
 0002:0000491c       ??_C@_1M@IIJCOJFA@?$AAx?$AAh?$AA?9?$AAZ?$AAA?$AA?$AA@ 1001e91c     libucrt:lcidtoname_downlevel.obj
 0002:00004928       ??_C@_1M@LGPJHNJH@?$AAz?$AAu?$AA?9?$AAZ?$AAA?$AA?$AA@ 1001e928     libucrt:lcidtoname_downlevel.obj
 0002:00004934       ??_C@_1M@HOKAOIO@?$AAa?$AAf?$AA?9?$AAZ?$AAA?$AA?$AA@ 1001e934     libucrt:lcidtoname_downlevel.obj
 0002:00004940       ??_C@_1M@DPCLHLIE@?$AAk?$AAa?$AA?9?$AAG?$AAE?$AA?$AA@ 1001e940     libucrt:lcidtoname_downlevel.obj
 0002:0000494c       ??_C@_1M@BLKMHJBI@?$AAf?$AAo?$AA?9?$AAF?$AAO?$AA?$AA@ 1001e94c     libucrt:lcidtoname_downlevel.obj
 0002:00004958       ??_C@_1M@LGGJAPPB@?$AAh?$AAi?$AA?9?$AAI?$AAN?$AA?$AA@ 1001e958     libucrt:lcidtoname_downlevel.obj
 0002:00004964       ??_C@_1M@FIKPIHFE@?$AAm?$AAt?$AA?9?$AAM?$AAT?$AA?$AA@ 1001e964     libucrt:lcidtoname_downlevel.obj
 0002:00004970       ??_C@_1M@HEGGPBFA@?$AAs?$AAe?$AA?9?$AAN?$AAO?$AA?$AA@ 1001e970     libucrt:lcidtoname_downlevel.obj
 0002:0000497c       ??_C@_1M@EIBJEEPA@?$AAm?$AAs?$AA?9?$AAM?$AAY?$AA?$AA@ 1001e97c     libucrt:lcidtoname_downlevel.obj
 0002:00004988       ??_C@_1M@FHLBGMPP@?$AAk?$AAk?$AA?9?$AAK?$AAZ?$AA?$AA@ 1001e988     libucrt:lcidtoname_downlevel.obj
 0002:00004994       ??_C@_1M@NGJJLCGI@?$AAk?$AAy?$AA?9?$AAK?$AAG?$AA?$AA@ 1001e994     libucrt:lcidtoname_downlevel.obj
 0002:000049a0       ??_C@_1M@GIENNBFC@?$AAs?$AAw?$AA?9?$AAK?$AAE?$AA?$AA@ 1001e9a0     libucrt:lcidtoname_downlevel.obj
 0002:000049ac       ??_C@_1BG@NDGMJIMJ@?$AAu?$AAz?$AA?9?$AAU?$AAZ?$AA?9?$AAL?$AAa?$AAt?$AAn?$AA?$AA@ 1001e9ac     libucrt:lcidtoname_downlevel.obj
 0002:000049c4       ??_C@_1M@IDCCIHBC@?$AAt?$AAt?$AA?9?$AAR?$AAU?$AA?$AA@ 1001e9c4     libucrt:lcidtoname_downlevel.obj
 0002:000049d0       ??_C@_1M@LOICPMOJ@?$AAb?$AAn?$AA?9?$AAI?$AAN?$AA?$AA@ 1001e9d0     libucrt:lcidtoname_downlevel.obj
 0002:000049dc       ??_C@_1M@KPKKNEAH@?$AAp?$AAa?$AA?9?$AAI?$AAN?$AA?$AA@ 1001e9dc     libucrt:lcidtoname_downlevel.obj
 0002:000049e8       ??_C@_1M@PJGPPBOG@?$AAg?$AAu?$AA?9?$AAI?$AAN?$AA?$AA@ 1001e9e8     libucrt:lcidtoname_downlevel.obj
 0002:000049f4       ??_C@_1M@KMKMOPHI@?$AAt?$AAa?$AA?9?$AAI?$AAN?$AA?$AA@ 1001e9f4     libucrt:lcidtoname_downlevel.obj
 0002:00004a00       ??_C@_1M@KFEHEPAC@?$AAt?$AAe?$AA?9?$AAI?$AAN?$AA?$AA@ 1001ea00     libucrt:lcidtoname_downlevel.obj
 0002:00004a0c       ??_C@_1M@CDCLMGHI@?$AAk?$AAn?$AA?9?$AAI?$AAN?$AA?$AA@ 1001ea0c     libucrt:lcidtoname_downlevel.obj
 0002:00004a18       ??_C@_1M@MIODLDKF@?$AAm?$AAl?$AA?9?$AAI?$AAN?$AA?$AA@ 1001ea18     libucrt:lcidtoname_downlevel.obj
 0002:00004a24       ??_C@_1M@PBIEACPO@?$AAm?$AAr?$AA?9?$AAI?$AAN?$AA?$AA@ 1001ea24     libucrt:lcidtoname_downlevel.obj
 0002:00004a30       ??_C@_1M@NIDEAGPH@?$AAs?$AAa?$AA?9?$AAI?$AAN?$AA?$AA@ 1001ea30     libucrt:lcidtoname_downlevel.obj
 0002:00004a3c       ??_C@_1M@FHIHCBIO@?$AAm?$AAn?$AA?9?$AAM?$AAN?$AA?$AA@ 1001ea3c     libucrt:lcidtoname_downlevel.obj
 0002:00004a48       ??_C@_1M@JAIJPENP@?$AAc?$AAy?$AA?9?$AAG?$AAB?$AA?$AA@ 1001ea48     libucrt:lcidtoname_downlevel.obj
 0002:00004a54       ??_C@_1M@PHGFBEPN@?$AAg?$AAl?$AA?9?$AAE?$AAS?$AA?$AA@ 1001ea54     libucrt:lcidtoname_downlevel.obj
 0002:00004a60       ??_C@_1O@KPIPDNCP@?$AAk?$AAo?$AAk?$AA?9?$AAI?$AAN?$AA?$AA@ 1001ea60     libucrt:lcidtoname_downlevel.obj
 0002:00004a70       ??_C@_1O@KNHJLDJA@?$AAs?$AAy?$AAr?$AA?9?$AAS?$AAY?$AA?$AA@ 1001ea70     libucrt:lcidtoname_downlevel.obj
 0002:00004a80       ??_C@_1O@MKEKBLAH@?$AAd?$AAi?$AAv?$AA?9?$AAM?$AAV?$AA?$AA@ 1001ea80     libucrt:lcidtoname_downlevel.obj
 0002:00004a90       ??_C@_1O@OHDCKDDF@?$AAq?$AAu?$AAz?$AA?9?$AAB?$AAO?$AA?$AA@ 1001ea90     libucrt:lcidtoname_downlevel.obj
 0002:00004aa0       ??_C@_1M@LEPJNLFD@?$AAn?$AAs?$AA?9?$AAZ?$AAA?$AA?$AA@ 1001eaa0     libucrt:lcidtoname_downlevel.obj
 0002:00004aac       ??_C@_1M@OMLEIIJB@?$AAm?$AAi?$AA?9?$AAN?$AAZ?$AA?$AA@ 1001eaac     libucrt:lcidtoname_downlevel.obj
 0002:00004ab8       ??_C@_1M@PMPEAILG@?$AAa?$AAr?$AA?9?$AAI?$AAQ?$AA?$AA@ 1001eab8     libucrt:lcidtoname_downlevel.obj
 0002:00004ac4       ??_C@_1M@CNKPNOEE@?$AAd?$AAe?$AA?9?$AAC?$AAH?$AA?$AA@ 1001eac4     libucrt:lcidtoname_downlevel.obj
 0002:00004ad0       ??_C@_1M@LKMGMLKO@?$AAe?$AAn?$AA?9?$AAG?$AAB?$AA?$AA@ 1001ead0     libucrt:lcidtoname_downlevel.obj
 0002:00004adc       ??_C@_1M@PGKJFFGL@?$AAe?$AAs?$AA?9?$AAM?$AAX?$AA?$AA@ 1001eadc     libucrt:lcidtoname_downlevel.obj
 0002:00004ae8       ??_C@_1M@DNNANBDC@?$AAf?$AAr?$AA?9?$AAB?$AAE?$AA?$AA@ 1001eae8     libucrt:lcidtoname_downlevel.obj
 0002:00004af4       ??_C@_1M@HLGMDFHM@?$AAi?$AAt?$AA?9?$AAC?$AAH?$AA?$AA@ 1001eaf4     libucrt:lcidtoname_downlevel.obj
 0002:00004b00       ??_C@_1M@CLLBGJH@?$AAn?$AAl?$AA?9?$AAB?$AAE?$AA?$AA@ 1001eb00     libucrt:lcidtoname_downlevel.obj
 0002:00004b0c       ??_C@_1M@BODBOGLF@?$AAn?$AAn?$AA?9?$AAN?$AAO?$AA?$AA@ 1001eb0c     libucrt:lcidtoname_downlevel.obj
 0002:00004b18       ??_C@_1M@HFFAHKAD@?$AAp?$AAt?$AA?9?$AAP?$AAT?$AA?$AA@ 1001eb18     libucrt:lcidtoname_downlevel.obj
 0002:00004b24       ??_C@_1BG@LNOAKHIE@?$AAs?$AAr?$AA?9?$AAS?$AAP?$AA?9?$AAL?$AAa?$AAt?$AAn?$AA?$AA@ 1001eb24     libucrt:lcidtoname_downlevel.obj
 0002:00004b3c       ??_C@_1M@HBMHBGAK@?$AAs?$AAv?$AA?9?$AAF?$AAI?$AA?$AA@ 1001eb3c     libucrt:lcidtoname_downlevel.obj
 0002:00004b48       ??_C@_1BG@DGCJGJBE@?$AAa?$AAz?$AA?9?$AAA?$AAZ?$AA?9?$AAC?$AAy?$AAr?$AAl?$AA?$AA@ 1001eb48     libucrt:lcidtoname_downlevel.obj
 0002:00004b60       ??_C@_1M@KEJDAAHB@?$AAs?$AAe?$AA?9?$AAS?$AAE?$AA?$AA@ 1001eb60     libucrt:lcidtoname_downlevel.obj
 0002:00004b6c       ??_C@_1M@HEIBJJAD@?$AAm?$AAs?$AA?9?$AAB?$AAN?$AA?$AA@ 1001eb6c     libucrt:lcidtoname_downlevel.obj
 0002:00004b78       ??_C@_1BG@PBGJMCEM@?$AAu?$AAz?$AA?9?$AAU?$AAZ?$AA?9?$AAC?$AAy?$AAr?$AAl?$AA?$AA@ 1001eb78     libucrt:lcidtoname_downlevel.obj
 0002:00004b90       ??_C@_1O@LAOBCMDF@?$AAq?$AAu?$AAz?$AA?9?$AAE?$AAC?$AA?$AA@ 1001eb90     libucrt:lcidtoname_downlevel.obj
 0002:00004ba0       ??_C@_1M@POEEMAIO@?$AAa?$AAr?$AA?9?$AAE?$AAG?$AA?$AA@ 1001eba0     libucrt:lcidtoname_downlevel.obj
 0002:00004bac       ??_C@_1M@EFAKDEDL@?$AAz?$AAh?$AA?9?$AAH?$AAK?$AA?$AA@ 1001ebac     libucrt:lcidtoname_downlevel.obj
 0002:00004bb8       ??_C@_1M@HKKIJHGI@?$AAd?$AAe?$AA?9?$AAA?$AAT?$AA?$AA@ 1001ebb8     libucrt:lcidtoname_downlevel.obj
 0002:00004bc4       ??_C@_1M@KBFBEHJF@?$AAe?$AAn?$AA?9?$AAA?$AAU?$AA?$AA@ 1001ebc4     libucrt:lcidtoname_downlevel.obj
 0002:00004bd0       ??_C@_1M@MNPLFAAH@?$AAe?$AAs?$AA?9?$AAE?$AAS?$AA?$AA@ 1001ebd0     libucrt:lcidtoname_downlevel.obj
 0002:00004bdc       ??_C@_1M@HJOOJFMA@?$AAf?$AAr?$AA?9?$AAC?$AAA?$AA?$AA@ 1001ebdc     libucrt:lcidtoname_downlevel.obj
 0002:00004be8       ??_C@_1BG@JPOFPNAB@?$AAs?$AAr?$AA?9?$AAS?$AAP?$AA?9?$AAC?$AAy?$AAr?$AAl?$AA?$AA@ 1001ebe8     libucrt:lcidtoname_downlevel.obj
 0002:00004c00       ??_C@_1M@LNFOCMOB@?$AAs?$AAe?$AA?9?$AAF?$AAI?$AA?$AA@ 1001ec00     libucrt:lcidtoname_downlevel.obj
 0002:00004c0c       ??_C@_1O@MGJBOAMB@?$AAq?$AAu?$AAz?$AA?9?$AAP?$AAE?$AA?$AA@ 1001ec0c     libucrt:lcidtoname_downlevel.obj
 0002:00004c1c       ??_C@_1M@GJINLBOK@?$AAa?$AAr?$AA?9?$AAL?$AAY?$AA?$AA@ 1001ec1c     libucrt:lcidtoname_downlevel.obj
 0002:00004c28       ??_C@_1M@GGMNHJNL@?$AAz?$AAh?$AA?9?$AAS?$AAG?$AA?$AA@ 1001ec28     libucrt:lcidtoname_downlevel.obj
 0002:00004c34       ??_C@_1M@HOIKODND@?$AAd?$AAe?$AA?9?$AAL?$AAU?$AA?$AA@ 1001ec34     libucrt:lcidtoname_downlevel.obj
 0002:00004c40       ??_C@_1M@DDOCCGFG@?$AAe?$AAn?$AA?9?$AAC?$AAA?$AA?$AA@ 1001ec40     libucrt:lcidtoname_downlevel.obj
 0002:00004c4c       ??_C@_1M@BNOEMJLF@?$AAe?$AAs?$AA?9?$AAG?$AAT?$AA?$AA@ 1001ec4c     libucrt:lcidtoname_downlevel.obj
 0002:00004c58       ??_C@_1M@EOGNKEK@?$AAf?$AAr?$AA?9?$AAC?$AAH?$AA?$AA@ 1001ec58     libucrt:lcidtoname_downlevel.obj
 0002:00004c64       ??_C@_1M@FLIDJFHL@?$AAh?$AAr?$AA?9?$AAB?$AAA?$AA?$AA@ 1001ec64     libucrt:lcidtoname_downlevel.obj
 0002:00004c70       ??_C@_1O@FMCELNAJ@?$AAs?$AAm?$AAj?$AA?9?$AAN?$AAO?$AA?$AA@ 1001ec70     libucrt:lcidtoname_downlevel.obj
 0002:00004c80       ??_C@_1M@JHGLJMGJ@?$AAa?$AAr?$AA?9?$AAD?$AAZ?$AA?$AA@ 1001ec80     libucrt:lcidtoname_downlevel.obj
 0002:00004c8c       ??_C@_1M@JKKFDCNP@?$AAz?$AAh?$AA?9?$AAM?$AAO?$AA?$AA@ 1001ec8c     libucrt:lcidtoname_downlevel.obj
 0002:00004c98       ??_C@_1M@GEEFALPE@?$AAd?$AAe?$AA?9?$AAL?$AAI?$AA?$AA@ 1001ec98     libucrt:lcidtoname_downlevel.obj
 0002:00004ca4       ??_C@_1M@IGEOFBG@?$AAe?$AAn?$AA?9?$AAN?$AAZ?$AA?$AA@ 1001eca4     libucrt:lcidtoname_downlevel.obj
 0002:00004cb0       ??_C@_1M@KDBONEHP@?$AAe?$AAs?$AA?9?$AAC?$AAR?$AA?$AA@ 1001ecb0     libucrt:lcidtoname_downlevel.obj
 0002:00004cbc       ??_C@_1M@FHMDOHNN@?$AAf?$AAr?$AA?9?$AAL?$AAU?$AA?$AA@ 1001ecbc     libucrt:lcidtoname_downlevel.obj
 0002:00004cc8       ??_C@_1BG@NFKKMAFG@?$AAb?$AAs?$AA?9?$AAB?$AAA?$AA?9?$AAL?$AAa?$AAt?$AAn?$AA?$AA@ 1001ecc8     libucrt:lcidtoname_downlevel.obj
 0002:00004ce0       ??_C@_1O@IMNBEMCI@?$AAs?$AAm?$AAj?$AA?9?$AAS?$AAE?$AA?$AA@ 1001ece0     libucrt:lcidtoname_downlevel.obj
 0002:00004cf0       ??_C@_1M@DHHMBNDP@?$AAa?$AAr?$AA?9?$AAM?$AAA?$AA?$AA@ 1001ecf0     libucrt:lcidtoname_downlevel.obj
 0002:00004cfc       ??_C@_1M@BNBLJCGH@?$AAe?$AAn?$AA?9?$AAI?$AAE?$AA?$AA@ 1001ecfc     libucrt:lcidtoname_downlevel.obj
 0002:00004d08       ??_C@_1M@GEPAFMDL@?$AAe?$AAs?$AA?9?$AAP?$AAA?$AA?$AA@ 1001ed08     libucrt:lcidtoname_downlevel.obj
 0002:00004d14       ??_C@_1M@OJONDMDL@?$AAf?$AAr?$AA?9?$AAM?$AAC?$AA?$AA@ 1001ed14     libucrt:lcidtoname_downlevel.obj
 0002:00004d20       ??_C@_1BG@OBCNFJB@?$AAs?$AAr?$AA?9?$AAB?$AAA?$AA?9?$AAL?$AAa?$AAt?$AAn?$AA?$AA@ 1001ed20     libucrt:lcidtoname_downlevel.obj
 0002:00004d38       ??_C@_1O@KEMEEGPO@?$AAs?$AAm?$AAa?$AA?9?$AAN?$AAO?$AA?$AA@ 1001ed38     libucrt:lcidtoname_downlevel.obj
 0002:00004d48       ??_C@_1M@ELMGFODK@?$AAa?$AAr?$AA?9?$AAT?$AAN?$AA?$AA@ 1001ed48     libucrt:lcidtoname_downlevel.obj
 0002:00004d54       ??_C@_1M@BHDLHFAF@?$AAe?$AAn?$AA?9?$AAZ?$AAA?$AA?$AA@ 1001ed54     libucrt:lcidtoname_downlevel.obj
 0002:00004d60       ??_C@_1M@BMGIGLIF@?$AAe?$AAs?$AA?9?$AAD?$AAO?$AA?$AA@ 1001ed60     libucrt:lcidtoname_downlevel.obj
 0002:00004d6c       ??_C@_1BG@CMBHIPBE@?$AAs?$AAr?$AA?9?$AAB?$AAA?$AA?9?$AAC?$AAy?$AAr?$AAl?$AA?$AA@ 1001ed6c     libucrt:lcidtoname_downlevel.obj
 0002:00004d84       ??_C@_1O@HEDBLHNP@?$AAs?$AAm?$AAa?$AA?9?$AAS?$AAE?$AA?$AA@ 1001ed84     libucrt:lcidtoname_downlevel.obj
 0002:00004d94       ??_C@_1M@DAGCADIM@?$AAa?$AAr?$AA?9?$AAO?$AAM?$AA?$AA@ 1001ed94     libucrt:lcidtoname_downlevel.obj
 0002:00004da0       ??_C@_1M@FODLMICG@?$AAe?$AAn?$AA?9?$AAJ?$AAM?$AA?$AA@ 1001eda0     libucrt:lcidtoname_downlevel.obj
 0002:00004dac       ??_C@_1M@DNMLCIHB@?$AAe?$AAs?$AA?9?$AAV?$AAE?$AA?$AA@ 1001edac     libucrt:lcidtoname_downlevel.obj
 0002:00004db8       ??_C@_1O@EOKHMKJK@?$AAs?$AAm?$AAs?$AA?9?$AAF?$AAI?$AA?$AA@ 1001edb8     libucrt:lcidtoname_downlevel.obj
 0002:00004dc8       ??_C@_1M@CAFJMKOF@?$AAa?$AAr?$AA?9?$AAY?$AAE?$AA?$AA@ 1001edc8     libucrt:lcidtoname_downlevel.obj
 0002:00004dd4       ??_C@_1M@CBFHIJLI@?$AAe?$AAn?$AA?9?$AAC?$AAB?$AA?$AA@ 1001edd4     libucrt:lcidtoname_downlevel.obj
 0002:00004de0       ??_C@_1M@BGNFLDN@?$AAe?$AAs?$AA?9?$AAC?$AAO?$AA?$AA@ 1001ede0     libucrt:lcidtoname_downlevel.obj
 0002:00004dec       ??_C@_1O@JMPHMAMC@?$AAs?$AAm?$AAn?$AA?9?$AAF?$AAI?$AA?$AA@ 1001edec     libucrt:lcidtoname_downlevel.obj
 0002:00004dfc       ??_C@_1M@JLANABKE@?$AAa?$AAr?$AA?9?$AAS?$AAY?$AA?$AA@ 1001edfc     libucrt:lcidtoname_downlevel.obj
 0002:00004e08       ??_C@_1M@HPKGCFGN@?$AAe?$AAn?$AA?9?$AAB?$AAZ?$AA?$AA@ 1001ee08     libucrt:lcidtoname_downlevel.obj
 0002:00004e14       ??_C@_1M@OLJCMLGM@?$AAe?$AAs?$AA?9?$AAP?$AAE?$AA?$AA@ 1001ee14     libucrt:lcidtoname_downlevel.obj
 0002:00004e20       ??_C@_1M@MKKGFKLE@?$AAa?$AAr?$AA?9?$AAJ?$AAO?$AA?$AA@ 1001ee20     libucrt:lcidtoname_downlevel.obj
 0002:00004e2c       ??_C@_1M@EKPGLDNI@?$AAe?$AAn?$AA?9?$AAT?$AAT?$AA?$AA@ 1001ee2c     libucrt:lcidtoname_downlevel.obj
 0002:00004e38       ??_C@_1M@OONGHFHE@?$AAe?$AAs?$AA?9?$AAA?$AAR?$AA?$AA@ 1001ee38     libucrt:lcidtoname_downlevel.obj
 0002:00004e44       ??_C@_1M@OOJFGBHE@?$AAa?$AAr?$AA?9?$AAL?$AAB?$AA?$AA@ 1001ee44     libucrt:lcidtoname_downlevel.obj
 0002:00004e50       ??_C@_1M@GCEJHNEG@?$AAe?$AAn?$AA?9?$AAZ?$AAW?$AA?$AA@ 1001ee50     libucrt:lcidtoname_downlevel.obj
 0002:00004e5c       ??_C@_1M@JNOCAHJI@?$AAe?$AAs?$AA?9?$AAE?$AAC?$AA?$AA@ 1001ee5c     libucrt:lcidtoname_downlevel.obj
 0002:00004e68       ??_C@_1M@JEFHPGGB@?$AAa?$AAr?$AA?9?$AAK?$AAW?$AA?$AA@ 1001ee68     libucrt:lcidtoname_downlevel.obj
 0002:00004e74       ??_C@_1M@MLKIBJOJ@?$AAe?$AAn?$AA?9?$AAP?$AAH?$AA?$AA@ 1001ee74     libucrt:lcidtoname_downlevel.obj
 0002:00004e80       ??_C@_1M@BDNIPEND@?$AAe?$AAs?$AA?9?$AAC?$AAL?$AA?$AA@ 1001ee80     libucrt:lcidtoname_downlevel.obj
 0002:00004e8c       ??_C@_1M@MPNMEKBD@?$AAa?$AAr?$AA?9?$AAA?$AAE?$AA?$AA@ 1001ee8c     libucrt:lcidtoname_downlevel.obj
 0002:00004e98       ??_C@_1M@KBJALCPI@?$AAe?$AAs?$AA?9?$AAU?$AAY?$AA?$AA@ 1001ee98     libucrt:lcidtoname_downlevel.obj
 0002:00004ea4       ??_C@_1M@LLCCOAGA@?$AAa?$AAr?$AA?9?$AAB?$AAH?$AA?$AA@ 1001eea4     libucrt:lcidtoname_downlevel.obj
 0002:00004eb0       ??_C@_1M@PBFNCDEL@?$AAe?$AAs?$AA?9?$AAP?$AAY?$AA?$AA@ 1001eeb0     libucrt:lcidtoname_downlevel.obj
 0002:00004ebc       ??_C@_1M@EDGINPNP@?$AAa?$AAr?$AA?9?$AAQ?$AAA?$AA?$AA@ 1001eebc     libucrt:lcidtoname_downlevel.obj
 0002:00004ec8       ??_C@_1M@MKDBIIJI@?$AAe?$AAs?$AA?9?$AAB?$AAO?$AA?$AA@ 1001eec8     libucrt:lcidtoname_downlevel.obj
 0002:00004ed4       ??_C@_1M@CPKKEBLD@?$AAe?$AAs?$AA?9?$AAS?$AAV?$AA?$AA@ 1001eed4     libucrt:lcidtoname_downlevel.obj
 0002:00004ee0       ??_C@_1M@NDBGMMJL@?$AAe?$AAs?$AA?9?$AAH?$AAN?$AA?$AA@ 1001eee0     libucrt:lcidtoname_downlevel.obj
 0002:00004eec       ??_C@_1M@JIJIBHDP@?$AAe?$AAs?$AA?9?$AAN?$AAI?$AA?$AA@ 1001eeec     libucrt:lcidtoname_downlevel.obj
 0002:00004ef8       ??_C@_1M@CGFMKEEK@?$AAe?$AAs?$AA?9?$AAP?$AAR?$AA?$AA@ 1001eef8     libucrt:lcidtoname_downlevel.obj
 0002:00004f04       ??_C@_1O@ICJHKIIK@?$AAz?$AAh?$AA?9?$AAC?$AAH?$AAT?$AA?$AA@ 1001ef04     libucrt:lcidtoname_downlevel.obj
 0002:00004f14       ??_C@_15CLNEJCE@?$AAs?$AAr?$AA?$AA@ 1001ef14     libucrt:lcidtoname_downlevel.obj
 0002:00005640       ??_C@_1M@KAHEKEIG@?$AAa?$AAf?$AA?9?$AAz?$AAa?$AA?$AA@ 1001f640     libucrt:lcidtoname_downlevel.obj
 0002:0000564c       ??_C@_1M@GIECOABL@?$AAa?$AAr?$AA?9?$AAa?$AAe?$AA?$AA@ 1001f64c     libucrt:lcidtoname_downlevel.obj
 0002:00005658       ??_C@_1M@BMLMEKGI@?$AAa?$AAr?$AA?9?$AAb?$AAh?$AA?$AA@ 1001f658     libucrt:lcidtoname_downlevel.obj
 0002:00005664       ??_C@_1M@DAPFDGGB@?$AAa?$AAr?$AA?9?$AAd?$AAz?$AA?$AA@ 1001f664     libucrt:lcidtoname_downlevel.obj
 0002:00005670       ??_C@_1M@FJNKGKIG@?$AAa?$AAr?$AA?9?$AAe?$AAg?$AA?$AA@ 1001f670     libucrt:lcidtoname_downlevel.obj
 0002:0000567c       ??_C@_1M@FLGKKCLO@?$AAa?$AAr?$AA?9?$AAi?$AAq?$AA?$AA@ 1001f67c     libucrt:lcidtoname_downlevel.obj
 0002:00005688       ??_C@_1M@GNDIPALM@?$AAa?$AAr?$AA?9?$AAj?$AAo?$AA?$AA@ 1001f688     libucrt:lcidtoname_downlevel.obj
 0002:00005694       ??_C@_1M@DDMJFMGJ@?$AAa?$AAr?$AA?9?$AAk?$AAw?$AA?$AA@ 1001f694     libucrt:lcidtoname_downlevel.obj
 0002:000056a0       ??_C@_1M@EJALMLHM@?$AAa?$AAr?$AA?9?$AAl?$AAb?$AA?$AA@ 1001f6a0     libucrt:lcidtoname_downlevel.obj
 0002:000056ac       ??_C@_1M@MOBDBLOC@?$AAa?$AAr?$AA?9?$AAl?$AAy?$AA?$AA@ 1001f6ac     libucrt:lcidtoname_downlevel.obj
 0002:000056b8       ??_C@_1M@JAOCLHDH@?$AAa?$AAr?$AA?9?$AAm?$AAa?$AA?$AA@ 1001f6b8     libucrt:lcidtoname_downlevel.obj
 0002:000056c4       ??_C@_1M@JHPMKJIE@?$AAa?$AAr?$AA?9?$AAo?$AAm?$AA?$AA@ 1001f6c4     libucrt:lcidtoname_downlevel.obj
 0002:000056d0       ??_C@_1M@OEPGHFNH@?$AAa?$AAr?$AA?9?$AAq?$AAa?$AA?$AA@ 1001f6d0     libucrt:lcidtoname_downlevel.obj
 0002:000056dc       ??_C@_1M@KJDONENM@?$AAa?$AAr?$AA?9?$AAs?$AAa?$AA?$AA@ 1001f6dc     libucrt:lcidtoname_downlevel.obj
 0002:000056e8       ??_C@_1M@DMJDKLKM@?$AAa?$AAr?$AA?9?$AAs?$AAy?$AA?$AA@ 1001f6e8     libucrt:lcidtoname_downlevel.obj
 0002:000056f4       ??_C@_1M@OMFIPEDC@?$AAa?$AAr?$AA?9?$AAt?$AAn?$AA?$AA@ 1001f6f4     libucrt:lcidtoname_downlevel.obj
 0002:00005700       ??_C@_1M@IHMHGAON@?$AAa?$AAr?$AA?9?$AAy?$AAe?$AA?$AA@ 1001f700     libucrt:lcidtoname_downlevel.obj
 0002:0000570c       ??_C@_1BG@KDCPGJGB@?$AAa?$AAz?$AA?9?$AAa?$AAz?$AA?9?$AAc?$AAy?$AAr?$AAl?$AA?$AA@ 1001f70c     libucrt:lcidtoname_downlevel.obj
 0002:00005724       ??_C@_1BG@IBCKDDOE@?$AAa?$AAz?$AA?9?$AAa?$AAz?$AA?9?$AAl?$AAa?$AAt?$AAn?$AA?$AA@ 1001f724     libucrt:lcidtoname_downlevel.obj
 0002:0000573c       ??_C@_1M@EGPFDCPD@?$AAb?$AAe?$AA?9?$AAb?$AAy?$AA?$AA@ 1001f73c     libucrt:lcidtoname_downlevel.obj
 0002:00005748       ??_C@_1M@PCMGMCGC@?$AAb?$AAg?$AA?9?$AAb?$AAg?$AA?$AA@ 1001f748     libucrt:lcidtoname_downlevel.obj
 0002:00005754       ??_C@_1M@BJBMFGOB@?$AAb?$AAn?$AA?9?$AAi?$AAn?$AA?$AA@ 1001f754     libucrt:lcidtoname_downlevel.obj
 0002:00005760       ??_C@_1BG@EAKMMACD@?$AAb?$AAs?$AA?9?$AAb?$AAa?$AA?9?$AAl?$AAa?$AAt?$AAn?$AA?$AA@ 1001f760     libucrt:lcidtoname_downlevel.obj
 0002:00005778       ??_C@_1M@KGADAODK@?$AAc?$AAa?$AA?9?$AAe?$AAs?$AA?$AA@ 1001f778     libucrt:lcidtoname_downlevel.obj
 0002:00005784       ??_C@_1M@COAJPDHI@?$AAc?$AAs?$AA?9?$AAc?$AAz?$AA?$AA@ 1001f784     libucrt:lcidtoname_downlevel.obj
 0002:00005790       ??_C@_1M@DHBHFONH@?$AAc?$AAy?$AA?9?$AAg?$AAb?$AA?$AA@ 1001f790     libucrt:lcidtoname_downlevel.obj
 0002:0000579c       ??_C@_1M@IMGKELGA@?$AAd?$AAa?$AA?9?$AAd?$AAk?$AA?$AA@ 1001f79c     libucrt:lcidtoname_downlevel.obj
 0002:000057a8       ??_C@_1M@NNDGDNGA@?$AAd?$AAe?$AA?9?$AAa?$AAt?$AA?$AA@ 1001f7a8     libucrt:lcidtoname_downlevel.obj
 0002:000057b4       ??_C@_1M@IKDBHEEM@?$AAd?$AAe?$AA?9?$AAc?$AAh?$AA?$AA@ 1001f7b4     libucrt:lcidtoname_downlevel.obj
 0002:000057c0       ??_C@_1M@GFFOJMCJ@?$AAd?$AAe?$AA?9?$AAd?$AAe?$AA?$AA@ 1001f7c0     libucrt:lcidtoname_downlevel.obj
 0002:000057cc       ??_C@_1M@MDNLKBPM@?$AAd?$AAe?$AA?9?$AAl?$AAi?$AA?$AA@ 1001f7cc     libucrt:lcidtoname_downlevel.obj
 0002:000057d8       ??_C@_1M@NJBEEJNL@?$AAd?$AAe?$AA?9?$AAl?$AAu?$AA?$AA@ 1001f7d8     libucrt:lcidtoname_downlevel.obj
 0002:000057e4       ??_C@_1O@GNNELBAP@?$AAd?$AAi?$AAv?$AA?9?$AAm?$AAv?$AA?$AA@ 1001f7e4     libucrt:lcidtoname_downlevel.obj
 0002:000057f4       ??_C@_1M@EJLEOGAE@?$AAe?$AAl?$AA?9?$AAg?$AAr?$AA?$AA@ 1001f7f4     libucrt:lcidtoname_downlevel.obj
 0002:00005800       ??_C@_1M@GMPONJN@?$AAe?$AAn?$AA?9?$AAa?$AAu?$AA?$AA@ 1001f800     libucrt:lcidtoname_downlevel.obj
 0002:0000580c       ??_C@_1M@NIDIIPGF@?$AAe?$AAn?$AA?9?$AAb?$AAz?$AA?$AA@ 1001f80c     libucrt:lcidtoname_downlevel.obj
 0002:00005818       ??_C@_1M@JEHMIMFO@?$AAe?$AAn?$AA?9?$AAc?$AAa?$AA?$AA@ 1001f818     libucrt:lcidtoname_downlevel.obj
 0002:00005824       ??_C@_1M@IGMJCDLA@?$AAe?$AAn?$AA?9?$AAc?$AAb?$AA?$AA@ 1001f824     libucrt:lcidtoname_downlevel.obj
 0002:00005830       ??_C@_1M@BNFIGBKG@?$AAe?$AAn?$AA?9?$AAg?$AAb?$AA?$AA@ 1001f830     libucrt:lcidtoname_downlevel.obj
 0002:0000583c       ??_C@_1M@LKIFDIGP@?$AAe?$AAn?$AA?9?$AAi?$AAe?$AA?$AA@ 1001f83c     libucrt:lcidtoname_downlevel.obj
 0002:00005848       ??_C@_1M@PJKFGCCO@?$AAe?$AAn?$AA?9?$AAj?$AAm?$AA?$AA@ 1001f848     libucrt:lcidtoname_downlevel.obj
 0002:00005854       ??_C@_1M@KPPKEPBO@?$AAe?$AAn?$AA?9?$AAn?$AAz?$AA?$AA@ 1001f854     libucrt:lcidtoname_downlevel.obj
 0002:00005860       ??_C@_1M@GMDGLDOB@?$AAe?$AAn?$AA?9?$AAp?$AAh?$AA?$AA@ 1001f860     libucrt:lcidtoname_downlevel.obj
 0002:0000586c       ??_C@_1M@ONGIBJNA@?$AAe?$AAn?$AA?9?$AAt?$AAt?$AA?$AA@ 1001f86c     libucrt:lcidtoname_downlevel.obj
 0002:00005878       ??_C@_1M@LLODPCMM@?$AAe?$AAn?$AA?9?$AAu?$AAs?$AA?$AA@ 1001f878     libucrt:lcidtoname_downlevel.obj
 0002:00005884       ??_C@_1M@LAKFNPAN@?$AAe?$AAn?$AA?9?$AAz?$AAa?$AA?$AA@ 1001f884     libucrt:lcidtoname_downlevel.obj
 0002:00005890       ??_C@_1M@MFNHNHEO@?$AAe?$AAn?$AA?9?$AAz?$AAw?$AA?$AA@ 1001f890     libucrt:lcidtoname_downlevel.obj
 0002:0000589c       ??_C@_1M@EJEINPHM@?$AAe?$AAs?$AA?9?$AAa?$AAr?$AA?$AA@ 1001f89c     libucrt:lcidtoname_downlevel.obj
 0002:000058a8       ??_C@_1M@GNKPCCJA@?$AAe?$AAs?$AA?9?$AAb?$AAo?$AA?$AA@ 1001f8a8     libucrt:lcidtoname_downlevel.obj
 0002:000058b4       ??_C@_1M@LEEGFONL@?$AAe?$AAs?$AA?9?$AAc?$AAl?$AA?$AA@ 1001f8b4     libucrt:lcidtoname_downlevel.obj
 0002:000058c0       ??_C@_1M@KGPDPBDF@?$AAe?$AAs?$AA?9?$AAc?$AAo?$AA?$AA@ 1001f8c0     libucrt:lcidtoname_downlevel.obj
 0002:000058cc       ??_C@_1M@EIAHOHH@?$AAe?$AAs?$AA?9?$AAc?$AAr?$AA?$AA@ 1001f8cc     libucrt:lcidtoname_downlevel.obj
 0002:000058d8       ??_C@_1M@LLPGMBIN@?$AAe?$AAs?$AA?9?$AAd?$AAo?$AA?$AA@ 1001f8d8     libucrt:lcidtoname_downlevel.obj
 0002:000058e4       ??_C@_1M@DKHMKNJA@?$AAe?$AAs?$AA?9?$AAe?$AAc?$AA?$AA@ 1001f8e4     libucrt:lcidtoname_downlevel.obj
 0002:000058f0       ??_C@_1M@GKGFPKAP@?$AAe?$AAs?$AA?9?$AAe?$AAs?$AA?$AA@ 1001f8f0     libucrt:lcidtoname_downlevel.obj
 0002:000058fc       ??_C@_1M@LKHKGDLN@?$AAe?$AAs?$AA?9?$AAg?$AAt?$AA?$AA@ 1001f8fc     libucrt:lcidtoname_downlevel.obj
 0002:00005908       ??_C@_1M@HEIIGGJD@?$AAe?$AAs?$AA?9?$AAh?$AAn?$AA?$AA@ 1001f908     libucrt:lcidtoname_downlevel.obj
 0002:00005914       ??_C@_1M@FBDHPPGD@?$AAe?$AAs?$AA?9?$AAm?$AAx?$AA?$AA@ 1001f914     libucrt:lcidtoname_downlevel.obj
 0002:00005920       ??_C@_1M@DPAGLNDH@?$AAe?$AAs?$AA?9?$AAn?$AAi?$AA?$AA@ 1001f920     libucrt:lcidtoname_downlevel.obj
 0002:0000592c       ??_C@_1M@MDGOPGDD@?$AAe?$AAs?$AA?9?$AAp?$AAa?$AA?$AA@ 1001f92c     libucrt:lcidtoname_downlevel.obj
 0002:00005938       ??_C@_1M@EMAMGBGE@?$AAe?$AAs?$AA?9?$AAp?$AAe?$AA?$AA@ 1001f938     libucrt:lcidtoname_downlevel.obj
 0002:00005944       ??_C@_1M@IBMCAOEC@?$AAe?$AAs?$AA?9?$AAp?$AAr?$AA?$AA@ 1001f944     libucrt:lcidtoname_downlevel.obj
 0002:00005950       ??_C@_1M@FGMDIJED@?$AAe?$AAs?$AA?9?$AAp?$AAy?$AA?$AA@ 1001f950     libucrt:lcidtoname_downlevel.obj
 0002:0000595c       ??_C@_1M@IIDEOLLL@?$AAe?$AAs?$AA?9?$AAs?$AAv?$AA?$AA@ 1001f95c     libucrt:lcidtoname_downlevel.obj
 0002:00005968       ??_C@_1M@GAOBIPA@?$AAe?$AAs?$AA?9?$AAu?$AAy?$AA?$AA@ 1001f968     libucrt:lcidtoname_downlevel.obj
 0002:00005974       ??_C@_1M@JKFFICHJ@?$AAe?$AAs?$AA?9?$AAv?$AAe?$AA?$AA@ 1001f974     libucrt:lcidtoname_downlevel.obj
 0002:00005980       ??_C@_1M@PNMLOJDF@?$AAe?$AAt?$AA?9?$AAe?$AAe?$AA?$AA@ 1001f980     libucrt:lcidtoname_downlevel.obj
 0002:0000598c       ??_C@_1M@GHHLIKEI@?$AAe?$AAu?$AA?9?$AAe?$AAs?$AA?$AA@ 1001f98c     libucrt:lcidtoname_downlevel.obj
 0002:00005998       ??_C@_1M@PBNONODE@?$AAf?$AAa?$AA?9?$AAi?$AAr?$AA?$AA@ 1001f998     libucrt:lcidtoname_downlevel.obj
 0002:000059a4       ??_C@_1M@JEEHPMIL@?$AAf?$AAi?$AA?9?$AAf?$AAi?$AA?$AA@ 1001f9a4     libucrt:lcidtoname_downlevel.obj
 0002:000059b0       ??_C@_1M@LMDCNDBA@?$AAf?$AAo?$AA?9?$AAf?$AAo?$AA?$AA@ 1001f9b0     libucrt:lcidtoname_downlevel.obj
 0002:000059bc       ??_C@_1M@JKEOHLDK@?$AAf?$AAr?$AA?9?$AAb?$AAe?$AA?$AA@ 1001f9bc     libucrt:lcidtoname_downlevel.obj
 0002:000059c8       ??_C@_1M@NOHADPMI@?$AAf?$AAr?$AA?9?$AAc?$AAa?$AA?$AA@ 1001f9c8     libucrt:lcidtoname_downlevel.obj
 0002:000059d4       ??_C@_1M@KDHIHAEC@?$AAf?$AAr?$AA?9?$AAc?$AAh?$AA?$AA@ 1001f9d4     libucrt:lcidtoname_downlevel.obj
 0002:000059e0       ??_C@_1M@MMBBFGAK@?$AAf?$AAr?$AA?9?$AAf?$AAr?$AA?$AA@ 1001f9e0     libucrt:lcidtoname_downlevel.obj
 0002:000059ec       ??_C@_1M@PAFNENNF@?$AAf?$AAr?$AA?9?$AAl?$AAu?$AA?$AA@ 1001f9ec     libucrt:lcidtoname_downlevel.obj
 0002:000059f8       ??_C@_1M@EOHDJGDD@?$AAf?$AAr?$AA?9?$AAm?$AAc?$AA?$AA@ 1001f9f8     libucrt:lcidtoname_downlevel.obj
 0002:00005a04       ??_C@_1M@FAPLLOPF@?$AAg?$AAl?$AA?9?$AAe?$AAs?$AA?$AA@ 1001fa04     libucrt:lcidtoname_downlevel.obj
 0002:00005a10       ??_C@_1M@FOPBFLOO@?$AAg?$AAu?$AA?9?$AAi?$AAn?$AA?$AA@ 1001fa10     libucrt:lcidtoname_downlevel.obj
 0002:00005a1c       ??_C@_1M@KBMCINPM@?$AAh?$AAe?$AA?9?$AAi?$AAl?$AA?$AA@ 1001fa1c     libucrt:lcidtoname_downlevel.obj
 0002:00005a28       ??_C@_1M@BBPHKFPJ@?$AAh?$AAi?$AA?9?$AAi?$AAn?$AA?$AA@ 1001fa28     libucrt:lcidtoname_downlevel.obj
 0002:00005a34       ??_C@_1M@PMBNDPHD@?$AAh?$AAr?$AA?9?$AAb?$AAa?$AA?$AA@ 1001fa34     libucrt:lcidtoname_downlevel.obj
 0002:00005a40       ??_C@_1M@BPCKOEGE@?$AAh?$AAr?$AA?9?$AAh?$AAr?$AA?$AA@ 1001fa40     libucrt:lcidtoname_downlevel.obj
 0002:00005a4c       ??_C@_1M@GACBMHKE@?$AAh?$AAu?$AA?9?$AAh?$AAu?$AA?$AA@ 1001fa4c     libucrt:lcidtoname_downlevel.obj
 0002:00005a58       ??_C@_1M@MILPAJJC@?$AAh?$AAy?$AA?9?$AAa?$AAm?$AA?$AA@ 1001fa58     libucrt:lcidtoname_downlevel.obj
 0002:00005a64       ??_C@_1M@BABBICEC@?$AAi?$AAd?$AA?9?$AAi?$AAd?$AA?$AA@ 1001fa64     libucrt:lcidtoname_downlevel.obj
 0002:00005a70       ??_C@_1M@BIKNHHPF@?$AAi?$AAs?$AA?9?$AAi?$AAs?$AA?$AA@ 1001fa70     libucrt:lcidtoname_downlevel.obj
 0002:00005a7c       ??_C@_1M@NMPCJPHE@?$AAi?$AAt?$AA?9?$AAc?$AAh?$AA?$AA@ 1001fa7c     libucrt:lcidtoname_downlevel.obj
 0002:00005a88       ??_C@_1M@GHKGFEDF@?$AAi?$AAt?$AA?9?$AAi?$AAt?$AA?$AA@ 1001fa88     libucrt:lcidtoname_downlevel.obj
 0002:00005a94       ??_C@_1M@NIEJCJJA@?$AAj?$AAa?$AA?9?$AAj?$AAp?$AA?$AA@ 1001fa94     libucrt:lcidtoname_downlevel.obj
 0002:00005aa0       ??_C@_1M@JILFNBIM@?$AAk?$AAa?$AA?9?$AAg?$AAe?$AA?$AA@ 1001faa0     libucrt:lcidtoname_downlevel.obj
 0002:00005aac       ??_C@_1M@PACPMGPH@?$AAk?$AAk?$AA?9?$AAk?$AAz?$AA?$AA@ 1001faac     libucrt:lcidtoname_downlevel.obj
 0002:00005ab8       ??_C@_1M@IELFGMHA@?$AAk?$AAn?$AA?9?$AAi?$AAn?$AA?$AA@ 1001fab8     libucrt:lcidtoname_downlevel.obj
 0002:00005ac4       ??_C@_1O@IBBJHCH@?$AAk?$AAo?$AAk?$AA?9?$AAi?$AAn?$AA?$AA@ 1001fac4     libucrt:lcidtoname_downlevel.obj
 0002:00005ad4       ??_C@_1M@DMHAEOGC@?$AAk?$AAo?$AA?9?$AAk?$AAr?$AA?$AA@ 1001fad4     libucrt:lcidtoname_downlevel.obj
 0002:00005ae0       ??_C@_1M@HBAHBIGA@?$AAk?$AAy?$AA?9?$AAk?$AAg?$AA?$AA@ 1001fae0     libucrt:lcidtoname_downlevel.obj
 0002:00005aec       ??_C@_1M@KPMILCJG@?$AAl?$AAt?$AA?9?$AAl?$AAt?$AA?$AA@ 1001faec     libucrt:lcidtoname_downlevel.obj
 0002:00005af8       ??_C@_1M@BDEKKCA@?$AAl?$AAv?$AA?9?$AAl?$AAv?$AA?$AA@ 1001faf8     libucrt:lcidtoname_downlevel.obj
 0002:00005b04       ??_C@_1M@ELCKCCJJ@?$AAm?$AAi?$AA?9?$AAn?$AAz?$AA?$AA@ 1001fb04     libucrt:lcidtoname_downlevel.obj
 0002:00005b10       ??_C@_1M@CBOOLAPA@?$AAm?$AAk?$AA?9?$AAm?$AAk?$AA?$AA@ 1001fb10     libucrt:lcidtoname_downlevel.obj
 0002:00005b1c       ??_C@_1M@GPHNBJKN@?$AAm?$AAl?$AA?9?$AAi?$AAn?$AA?$AA@ 1001fb1c     libucrt:lcidtoname_downlevel.obj
 0002:00005b28       ??_C@_1M@PABJILIG@?$AAm?$AAn?$AA?9?$AAm?$AAn?$AA?$AA@ 1001fb28     libucrt:lcidtoname_downlevel.obj
 0002:00005b34       ??_C@_1M@FGBKKIPG@?$AAm?$AAr?$AA?9?$AAi?$AAn?$AA?$AA@ 1001fb34     libucrt:lcidtoname_downlevel.obj
 0002:00005b40       ??_C@_1M@NDBPDDAL@?$AAm?$AAs?$AA?9?$AAb?$AAn?$AA?$AA@ 1001fb40     libucrt:lcidtoname_downlevel.obj
 0002:00005b4c       ??_C@_1M@OPIHOOPI@?$AAm?$AAs?$AA?9?$AAm?$AAy?$AA?$AA@ 1001fb4c     libucrt:lcidtoname_downlevel.obj
 0002:00005b58       ??_C@_1M@PPDBCNFM@?$AAm?$AAt?$AA?9?$AAm?$AAt?$AA?$AA@ 1001fb58     libucrt:lcidtoname_downlevel.obj
 0002:00005b64       ??_C@_1M@KDJDKMDD@?$AAn?$AAb?$AA?9?$AAn?$AAo?$AA?$AA@ 1001fb64     libucrt:lcidtoname_downlevel.obj
 0002:00005b70       ??_C@_1M@KFCFLMJP@?$AAn?$AAl?$AA?9?$AAb?$AAe?$AA?$AA@ 1001fb70     libucrt:lcidtoname_downlevel.obj
 0002:00005b7c       ??_C@_1M@KPOPDDGO@?$AAn?$AAl?$AA?9?$AAn?$AAl?$AA?$AA@ 1001fb7c     libucrt:lcidtoname_downlevel.obj
 0002:00005b88       ??_C@_1M@LJKPEMLN@?$AAn?$AAn?$AA?9?$AAn?$AAo?$AA?$AA@ 1001fb88     libucrt:lcidtoname_downlevel.obj
 0002:00005b94       ??_C@_1M@BDGHHBFL@?$AAn?$AAs?$AA?9?$AAz?$AAa?$AA?$AA@ 1001fb94     libucrt:lcidtoname_downlevel.obj
 0002:00005ba0       ??_C@_1M@IDEHOAP@?$AAp?$AAa?$AA?9?$AAi?$AAn?$AA?$AA@ 1001fba0     libucrt:lcidtoname_downlevel.obj
 0002:00005bac       ??_C@_1M@HDBKGOGH@?$AAp?$AAl?$AA?9?$AAp?$AAl?$AA?$AA@ 1001fbac     libucrt:lcidtoname_downlevel.obj
 0002:00005bb8       ??_C@_1M@LJLLCMEH@?$AAp?$AAt?$AA?9?$AAb?$AAr?$AA?$AA@ 1001fbb8     libucrt:lcidtoname_downlevel.obj
 0002:00005bc4       ??_C@_1M@NCMONAAL@?$AAp?$AAt?$AA?9?$AAp?$AAt?$AA?$AA@ 1001fbc4     libucrt:lcidtoname_downlevel.obj
 0002:00005bd0       ??_C@_1O@EAKMAJDN@?$AAq?$AAu?$AAz?$AA?9?$AAb?$AAo?$AA?$AA@ 1001fbd0     libucrt:lcidtoname_downlevel.obj
 0002:00005be0       ??_C@_1O@BHHPIGDN@?$AAq?$AAu?$AAz?$AA?9?$AAe?$AAc?$AA?$AA@ 1001fbe0     libucrt:lcidtoname_downlevel.obj
 0002:00005bf0       ??_C@_1O@GBAPEKMJ@?$AAq?$AAu?$AAz?$AA?9?$AAp?$AAe?$AA?$AA@ 1001fbf0     libucrt:lcidtoname_downlevel.obj
 0002:00005c00       ??_C@_1M@CLGLEFBO@?$AAr?$AAo?$AA?9?$AAr?$AAo?$AA?$AA@ 1001fc00     libucrt:lcidtoname_downlevel.obj
 0002:00005c0c       ??_C@_1M@CEEDODME@?$AAr?$AAu?$AA?9?$AAr?$AAu?$AA?$AA@ 1001fc0c     libucrt:lcidtoname_downlevel.obj
 0002:00005c18       ??_C@_1M@HPKKKMPP@?$AAs?$AAa?$AA?9?$AAi?$AAn?$AA?$AA@ 1001fc18     libucrt:lcidtoname_downlevel.obj
 0002:00005c24       ??_C@_1M@BKMAIGOJ@?$AAs?$AAe?$AA?9?$AAf?$AAi?$AA?$AA@ 1001fc24     libucrt:lcidtoname_downlevel.obj
 0002:00005c30       ??_C@_1M@NDPIFLFI@?$AAs?$AAe?$AA?9?$AAn?$AAo?$AA?$AA@ 1001fc30     libucrt:lcidtoname_downlevel.obj
 0002:00005c3c       ??_C@_1M@DANKKHJ@?$AAs?$AAe?$AA?9?$AAs?$AAe?$AA?$AA@ 1001fc3c     libucrt:lcidtoname_downlevel.obj
 0002:00005c48       ??_C@_1M@PNBLONPJ@?$AAs?$AAk?$AA?9?$AAs?$AAk?$AA?$AA@ 1001fc48     libucrt:lcidtoname_downlevel.obj
 0002:00005c54       ??_C@_1M@LFMODOAL@?$AAs?$AAl?$AA?9?$AAs?$AAi?$AA?$AA@ 1001fc54     libucrt:lcidtoname_downlevel.obj
 0002:00005c60       ??_C@_1O@DFKOMPG@?$AAs?$AAm?$AAa?$AA?9?$AAn?$AAo?$AA?$AA@ 1001fc60     libucrt:lcidtoname_downlevel.obj
 0002:00005c70       ??_C@_1O@NDKPBNNH@?$AAs?$AAm?$AAa?$AA?9?$AAs?$AAe?$AA?$AA@ 1001fc70     libucrt:lcidtoname_downlevel.obj
 0002:00005c80       ??_C@_1O@PLLKBHAB@?$AAs?$AAm?$AAj?$AA?9?$AAn?$AAo?$AA?$AA@ 1001fc80     libucrt:lcidtoname_downlevel.obj
 0002:00005c90       ??_C@_1O@CLEPOGCA@?$AAs?$AAm?$AAj?$AA?9?$AAs?$AAe?$AA?$AA@ 1001fc90     libucrt:lcidtoname_downlevel.obj
 0002:00005ca0       ??_C@_1O@DLGJGKMK@?$AAs?$AAm?$AAn?$AA?9?$AAf?$AAi?$AA?$AA@ 1001fca0     libucrt:lcidtoname_downlevel.obj
 0002:00005cb0       ??_C@_1O@OJDJGAJC@?$AAs?$AAm?$AAs?$AA?9?$AAf?$AAi?$AA?$AA@ 1001fcb0     libucrt:lcidtoname_downlevel.obj
 0002:00005cc0       ??_C@_1M@BOFOGHPB@?$AAs?$AAq?$AA?9?$AAa?$AAl?$AA?$AA@ 1001fcc0     libucrt:lcidtoname_downlevel.obj
 0002:00005ccc       ??_C@_1BG@LJBBIPGB@?$AAs?$AAr?$AA?9?$AAb?$AAa?$AA?9?$AAc?$AAy?$AAr?$AAl?$AA?$AA@ 1001fccc     libucrt:lcidtoname_downlevel.obj
 0002:00005ce4       ??_C@_1BG@JLBENFOE@?$AAs?$AAr?$AA?9?$AAb?$AAa?$AA?9?$AAl?$AAa?$AAt?$AAn?$AA?$AA@ 1001fce4     libucrt:lcidtoname_downlevel.obj
 0002:00005cfc       ??_C@_1BG@KODPNHE@?$AAs?$AAr?$AA?9?$AAs?$AAp?$AA?9?$AAc?$AAy?$AAr?$AAl?$AA?$AA@ 1001fcfc     libucrt:lcidtoname_downlevel.obj
 0002:00005d14       ??_C@_1BG@CIOGKHPB@?$AAs?$AAr?$AA?9?$AAs?$AAp?$AA?9?$AAl?$AAa?$AAt?$AAn?$AA?$AA@ 1001fd14     libucrt:lcidtoname_downlevel.obj
 0002:00005d2c       ??_C@_1M@NGFJLMAC@?$AAs?$AAv?$AA?9?$AAf?$AAi?$AA?$AA@ 1001fd2c     libucrt:lcidtoname_downlevel.obj
 0002:00005d38       ??_C@_1M@MPJEJAJC@?$AAs?$AAv?$AA?9?$AAs?$AAe?$AA?$AA@ 1001fd38     libucrt:lcidtoname_downlevel.obj
 0002:00005d44       ??_C@_1M@MPNDHLFK@?$AAs?$AAw?$AA?9?$AAk?$AAe?$AA?$AA@ 1001fd44     libucrt:lcidtoname_downlevel.obj
 0002:00005d50       ??_C@_1O@KOHBJJI@?$AAs?$AAy?$AAr?$AA?9?$AAs?$AAy?$AA?$AA@ 1001fd50     libucrt:lcidtoname_downlevel.obj
 0002:00005d60       ??_C@_1M@LDCEFHA@?$AAt?$AAa?$AA?9?$AAi?$AAn?$AA?$AA@ 1001fd60     libucrt:lcidtoname_downlevel.obj
 0002:00005d6c       ??_C@_1M@CNJOFAK@?$AAt?$AAe?$AA?9?$AAi?$AAn?$AA?$AA@ 1001fd6c     libucrt:lcidtoname_downlevel.obj
 0002:00005d78       ??_C@_1M@GNAECACD@?$AAt?$AAh?$AA?9?$AAt?$AAh?$AA?$AA@ 1001fd78     libucrt:lcidtoname_downlevel.obj
 0002:00005d84       ??_C@_1M@CHBIHOJO@?$AAt?$AAn?$AA?9?$AAz?$AAa?$AA?$AA@ 1001fd84     libucrt:lcidtoname_downlevel.obj
 0002:00005d90       ??_C@_1M@GCCMIGPJ@?$AAt?$AAr?$AA?9?$AAt?$AAr?$AA?$AA@ 1001fd90     libucrt:lcidtoname_downlevel.obj
 0002:00005d9c       ??_C@_1M@CELMCNBK@?$AAt?$AAt?$AA?9?$AAr?$AAu?$AA?$AA@ 1001fd9c     libucrt:lcidtoname_downlevel.obj
 0002:00005da8       ??_C@_1M@KLMCELGA@?$AAu?$AAk?$AA?9?$AAu?$AAa?$AA?$AA@ 1001fda8     libucrt:lcidtoname_downlevel.obj
 0002:00005db4       ??_C@_1M@EPAJJAJF@?$AAu?$AAr?$AA?9?$AAp?$AAk?$AA?$AA@ 1001fdb4     libucrt:lcidtoname_downlevel.obj
 0002:00005dc0       ??_C@_1BG@GEGPMCDJ@?$AAu?$AAz?$AA?9?$AAu?$AAz?$AA?9?$AAc?$AAy?$AAr?$AAl?$AA?$AA@ 1001fdc0     libucrt:lcidtoname_downlevel.obj
 0002:00005dd8       ??_C@_1BG@EGGKJILM@?$AAu?$AAz?$AA?9?$AAu?$AAz?$AA?9?$AAl?$AAa?$AAt?$AAn?$AA?$AA@ 1001fdd8     libucrt:lcidtoname_downlevel.obj
 0002:00005df0       ??_C@_1M@GFOCLFF@?$AAv?$AAi?$AA?9?$AAv?$AAn?$AA?$AA@ 1001fdf0     libucrt:lcidtoname_downlevel.obj
 0002:00005dfc       ??_C@_1M@CPAMEDFI@?$AAx?$AAh?$AA?9?$AAz?$AAa?$AA?$AA@ 1001fdfc     libucrt:lcidtoname_downlevel.obj
 0002:00005e08       ??_C@_1O@EBKIFIGN@?$AAz?$AAh?$AA?9?$AAc?$AAh?$AAs?$AA?$AA@ 1001fe08     libucrt:lcidtoname_downlevel.obj
 0002:00005e18       ??_C@_1O@NMHPGANE@?$AAz?$AAh?$AA?9?$AAc?$AAh?$AAt?$AA?$AA@ 1001fe18     libucrt:lcidtoname_downlevel.obj
 0002:00005e28       ??_C@_1M@LPINJOMC@?$AAz?$AAh?$AA?9?$AAc?$AAn?$AA?$AA@ 1001fe28     libucrt:lcidtoname_downlevel.obj
 0002:00005e34       ??_C@_1M@OCJEJODD@?$AAz?$AAh?$AA?9?$AAh?$AAk?$AA?$AA@ 1001fe34     libucrt:lcidtoname_downlevel.obj
 0002:00005e40       ??_C@_1M@DNDLJINH@?$AAz?$AAh?$AA?9?$AAm?$AAo?$AA?$AA@ 1001fe40     libucrt:lcidtoname_downlevel.obj
 0002:00005e4c       ??_C@_1M@MBFDNDND@?$AAz?$AAh?$AA?9?$AAs?$AAg?$AA?$AA@ 1001fe4c     libucrt:lcidtoname_downlevel.obj
 0002:00005e58       ??_C@_1M@IMEPLEPE@?$AAz?$AAh?$AA?9?$AAt?$AAw?$AA?$AA@ 1001fe58     libucrt:lcidtoname_downlevel.obj
 0002:00005e64       ??_C@_1M@BBGHNHJP@?$AAz?$AAu?$AA?9?$AAz?$AAa?$AA?$AA@ 1001fe64     libucrt:lcidtoname_downlevel.obj
 0002:00005fd0       __infinity                 1001ffd0     libucrt:87tran.obj
 0002:00005fda       __minfinity                1001ffda     libucrt:87tran.obj
 0002:00005fe4       __logemax                  1001ffe4     libucrt:87tran.obj
 0002:0000600a       __OP_EXPjmptab             1002000a     libucrt:87tran.obj
 0002:00006030       __indefinite               10020030     libucrt:87disp.obj
 0002:0000603a       __piby2                    1002003a     libucrt:87disp.obj
 0002:00006044       __piby4                    10020044     libucrt:87disp.obj
 0002:00006078       __DEFAULT_CW_in_mem        10020078     libucrt:common.obj
 0002:0000607a       __pi_by_2_to_61            1002007a     libucrt:common.obj
 0002:000060b4       ??_C@_03MGHMBJCF@log?$AA@  100200b4     libucrt:libm_error.obj
 0002:000060b8       ??_C@_05HGHHAHAP@log10?$AA@ 100200b8     libucrt:libm_error.obj
 0002:000060c0       ??_C@_03KHJOGHMM@exp?$AA@  100200c0     libucrt:libm_error.obj
 0002:000060c4       ??_C@_03JGHBODFD@pow?$AA@  100200c4     libucrt:libm_error.obj
 0002:000060c8       ??_C@_04FIHNOPOL@asin?$AA@ 100200c8     libucrt:libm_error.obj
 0002:000060d0       ??_C@_04PDIFKINK@acos?$AA@ 100200d0     libucrt:libm_error.obj
 0002:000060d8       ??_C@_04EIAKFFMI@sqrt?$AA@ 100200d8     libucrt:libm_error.obj
 0002:000060e0       __real@3ff0000000000000    100200e0     libucrt:libm_error.obj
 0002:00006100       ___acrt_log10_table_t      10020100     libucrt:log10_tables.obj
 0002:00006510       ___acrt_log10_table_cb     10020510     libucrt:log10_tables.obj
 0002:00006920       __real@3fe0000000000000    10020920     libucrt:powhlp.obj
 0002:00006928       ??_C@_04FJHINJAO@tanh?$AA@ 10020928     libucrt:fpexcept.obj
 0002:00006930       ??_C@_04MLLJIGOK@atan?$AA@ 10020930     libucrt:fpexcept.obj
 0002:00006938       ??_C@_05KNGEOGJB@atan2?$AA@ 10020938     libucrt:fpexcept.obj
 0002:00006940       ??_C@_03BLEJJJBH@sin?$AA@  10020940     libucrt:fpexcept.obj
 0002:00006944       ??_C@_03LALBNOCG@cos?$AA@  10020944     libucrt:fpexcept.obj
 0002:00006948       ??_C@_03IIINPABG@tan?$AA@  10020948     libucrt:fpexcept.obj
 0002:0000694c       ??_C@_04GFPJNGEK@ceil?$AA@ 1002094c     libucrt:fpexcept.obj
 0002:00006954       ??_C@_05PBJFFIGL@floor?$AA@ 10020954     libucrt:fpexcept.obj
 0002:0000695c       ??_C@_04ODHECPBC@fabs?$AA@ 1002095c     libucrt:fpexcept.obj
 0002:00006964       ??_C@_04EHEDPDJG@modf?$AA@ 10020964     libucrt:fpexcept.obj
 0002:0000696c       ??_C@_05CEJMAHNP@ldexp?$AA@ 1002096c     libucrt:fpexcept.obj
 0002:00006974       ??_C@_05KBKMEMPO@_cabs?$AA@ 10020974     libucrt:fpexcept.obj
 0002:0000697c       ??_C@_06MEIMCGCF@_hypot?$AA@ 1002097c     libucrt:fpexcept.obj
 0002:00006984       ??_C@_04KEPJIHGP@fmod?$AA@ 10020984     libucrt:fpexcept.obj
 0002:0000698c       ??_C@_05GKKHEGJL@frexp?$AA@ 1002098c     libucrt:fpexcept.obj
 0002:00006994       ??_C@_03MJLDFKDL@_y0?$AA@  10020994     libucrt:fpexcept.obj
 0002:00006998       ??_C@_03NAKIGLHK@_y1?$AA@  10020998     libucrt:fpexcept.obj
 0002:0000699c       ??_C@_03ONILCKOB@_yn?$AA@  1002099c     libucrt:fpexcept.obj
 0002:000069a0       ??_C@_05JGDBENOH@_logb?$AA@ 100209a0     libucrt:fpexcept.obj
 0002:000069a8       ??_C@_0L@KDOEJCKC@_nextafter?$AA@ 100209a8     libucrt:fpexcept.obj
 0002:00006aa0       ??_C@_04COOMCNPB@sinh?$AA@ 10020aa0     libucrt:fpexcept.obj
 0002:00006aa8       ??_C@_04HPJJNFIM@cosh?$AA@ 10020aa8     libucrt:fpexcept.obj
 0002:00006ab0       __d_inf                    10020ab0     libucrt:util.obj
 0002:00006ab8       __d_max                    10020ab8     libucrt:util.obj
 0002:00006ac0       __d_mzero                  10020ac0     libucrt:util.obj
 0002:00006ac8       ??_C@_1BA@BALFACEM@?$AAC?$AAO?$AAN?$AAO?$AAU?$AAT?$AA$?$AA?$AA@ 10020ac8     libucrt:initcon.obj
 0002:00006b38       __load_config_used         10020b38     LIBCMT:loadcfg.obj
 0002:00006bd8       __tls_used                 10020bd8     LIBCMT:tlssup.obj
 0002:00006bf0       ??_R3IUnknown@@8           10020bf0     ConEmuBg.obj
 0002:00006c00       ??_R2IUnknown@@8           10020c00     ConEmuBg.obj
 0002:00006c08       ??_R1A@?0A@EA@IUnknown@@8  10020c08     ConEmuBg.obj
 0002:00006c24       ??_R3ISequentialStream@@8  10020c24     ConEmuBg.obj
 0002:00006c34       ??_R2ISequentialStream@@8  10020c34     ConEmuBg.obj
 0002:00006c40       ??_R1A@?0A@EA@ISequentialStream@@8 10020c40     ConEmuBg.obj
 0002:00006c5c       ??_R3IStream@@8            10020c5c     ConEmuBg.obj
 0002:00006c6c       ??_R2IStream@@8            10020c6c     ConEmuBg.obj
 0002:00006c7c       ??_R1A@?0A@EA@IStream@@8   10020c7c     ConEmuBg.obj
 0002:00006c98       ??_R4MStream@@6B@          10020c98     ConEmuBg.obj
 0002:00006cac       ??_R3MStream@@8            10020cac     ConEmuBg.obj
 0002:00006cbc       ??_R2MStream@@8            10020cbc     ConEmuBg.obj
 0002:00006cd0       ??_R1A@?0A@EA@MStream@@8   10020cd0     ConEmuBg.obj
 0002:00006cec       ??_R4type_info@@6B@        10020cec     LIBCMT:std_type_info_static.obj
 0002:00006d00       ??_R3type_info@@8          10020d00     LIBCMT:std_type_info_static.obj
 0002:00006d10       ??_R2type_info@@8          10020d10     LIBCMT:std_type_info_static.obj
 0002:00006d18       ??_R1A@?0A@EA@type_info@@8 10020d18     LIBCMT:std_type_info_static.obj
 0002:00006d34       ??_R4exception@std@@6B@    10020d34     libvcruntime:frame.obj
 0002:00006d48       ??_R3exception@std@@8      10020d48     libvcruntime:frame.obj
 0002:00006d58       ??_R2exception@std@@8      10020d58     libvcruntime:frame.obj
 0002:00006d60       ??_R1A@?0A@EA@exception@std@@8 10020d60     libvcruntime:frame.obj
 0002:00006d7c       ??_R4bad_exception@std@@6B@ 10020d7c     libvcruntime:frame.obj
 0002:00006d90       ??_R3bad_exception@std@@8  10020d90     libvcruntime:frame.obj
 0002:00006da0       ??_R2bad_exception@std@@8  10020da0     libvcruntime:frame.obj
 0002:00006dac       ??_R1A@?0A@EA@bad_exception@std@@8 10020dac     libvcruntime:frame.obj
 0002:00006dd0       ___safe_se_handler_table   10020dd0     <linker-defined>
 0002:0000717c       ___rtc_iaa                 1002117c     LIBCMT:_initsect_.obj
 0002:00007180       ___rtc_izz                 10021180     LIBCMT:_initsect_.obj
 0002:00007184       ___rtc_taa                 10021184     LIBCMT:_initsect_.obj
 0002:00007188       ___rtc_tzz                 10021188     LIBCMT:_initsect_.obj
 0002:0000718c       __tls_start                1002118c     LIBCMT:tlssup.obj
 0002:00007190       __Init_thread_epoch        10021190     LIBCMT:thread_safe_statics.obj
 0002:00007194       __tls_end                  10021194     LIBCMT:tlssup.obj
 0002:000073f4       __TI2?AVbad_exception@std@@ 100213f4     libvcruntime:frame.obj
 0002:00007404       __CTA2?AVbad_exception@std@@ 10021404     libvcruntime:frame.obj
 0002:00007410       __CT??_R0?AVbad_exception@std@@@8??0bad_exception@std@@QAE@ABV01@@Z12 10021410     libvcruntime:frame.obj
 0002:0000742c       __CT??_R0?AVexception@std@@@8??0exception@std@@QAE@ABV01@@Z12 1002142c     libvcruntime:frame.obj
 0002:0000790c       __IMPORT_DESCRIPTOR_VERSION 1002190c     version:VERSION.dll
 0002:00007920       __IMPORT_DESCRIPTOR_KERNEL32 10021920     kernel32:KERNEL32.dll
 0002:00007934       __IMPORT_DESCRIPTOR_USER32 10021934     user32:USER32.dll
 0002:00007948       __IMPORT_DESCRIPTOR_GDI32  10021948     gdi32:GDI32.dll
 0002:0000795c       __IMPORT_DESCRIPTOR_ADVAPI32 1002195c     advapi32:ADVAPI32.dll
 0002:00007970       __IMPORT_DESCRIPTOR_ole32  10021970     ole32:ole32.dll
 0002:00007984       __NULL_IMPORT_DESCRIPTOR   10021984     version:VERSION.dll
 0003:00000000       ?szDefaultXmlName@@3PB_WB  10023000     ConEmuBg.obj
 0003:00000004       ?gSettings@@3PAUConEmuBgSettings@@A 10023004     ConEmuBg.obj
 0003:00000034       ?Far3Func@@3PAUExportFunc@@A 10023034     ConEmuBg.obj
 0003:00000218       ?guid_ConEmuBg@@3U_GUID@@A 10023218     ConEmuBg2800.obj
 0003:00000228       ?guid_ConEmuBgCfgDlg@@3U_GUID@@A 10023228     ConEmuBg2800.obj
 0003:00000238       ?guid_ConEmuBgPluginMenu@@3U_GUID@@A 10023238     ConEmuBg2800.obj
 0003:00000248       ?guid_ConEmuBgPluginConfig@@3U_GUID@@A 10023248     ConEmuBg2800.obj
 0003:000016d8       ?g_TerminatedThreadIdx@@3JA 100246d8     common-kernel32:WThreads.obj
 0003:000016e0       ___security_cookie         100246e0     LIBCMT:gs_cookie.obj
 0003:000016e4       ___security_cookie_complement 100246e4     LIBCMT:gs_cookie.obj
 0003:000016e8       __Init_global_epoch        100246e8     LIBCMT:thread_safe_statics.obj
 0003:000016f0       ___scrt_native_dllmain_reason 100246f0     LIBCMT:utility.obj
 0003:000016f4       ___isa_enabled             100246f4     LIBCMT:_cpu_disp_.obj
 0003:00001710       __NLG_Destination          10024710     libvcruntime:_exsup_.obj
 0003:00001720       ___abort_behavior          10024720     libucrt:abort.obj
 0003:00001738       __pwctype                  10024738     libucrt:ctype.obj
 0003:00001740       ___acrt_initial_locale_data 10024740     libucrt:nlsdata.obj
 0003:000017f8       ___acrt_initial_locale_pointers 100247f8     libucrt:nlsdata.obj
 0003:00001800       ___acrt_wide_c_locale_string 10024800     libucrt:nlsdata.obj
 0003:00001808       __iob                      10024808     libucrt:_file.obj
 0003:000019a8       __mbctype                  100249a8     libucrt:mbctype.obj
 0003:00001ab0       __mbcasemap                10024ab0     libucrt:mbctype.obj
 0003:00001bb0       ___acrt_initial_multibyte_data 10024bb0     libucrt:mbctype.obj
 0003:00001dd0       ___acrt_current_multibyte_data 10024dd0     libucrt:mbctype.obj
 0003:00001dd4       ___globallocalestatus      10024dd4     libucrt:glstatus.obj
 0003:00001dd8       ___acrt_lconv_static_decimal 10024dd8     libucrt:localeconv.obj
 0003:00001ddc       ___acrt_lconv_static_W_decimal 10024ddc     libucrt:localeconv.obj
 0003:00001de0       ___acrt_lconv_c            10024de0     libucrt:localeconv.obj
 0003:00001e30       ___dcrt_lowio_console_output_handle 10024e30     libucrt:initcon.obj
 0003:00001e40       __fltused                  10024e40     LIBCMT:fltused.obj
 0003:00001e50       ??_R0?AUIUnknown@@@8       10024e50     ConEmuBg.obj
 0003:00001e68       ??_R0?AUISequentialStream@@@8 10024e68     ConEmuBg.obj
 0003:00001e88       ??_R0?AUIStream@@@8        10024e88     ConEmuBg.obj
 0003:00001ea0       ??_R0?AVMStream@@@8        10024ea0     ConEmuBg.obj
 0003:00001eb8       ??_R0?AVtype_info@@@8      10024eb8     LIBCMT:std_type_info_static.obj
 0003:00001ed0       ??_R0?AVbad_exception@std@@@8 10024ed0     libvcruntime:frame.obj
 0003:00001ef0       ??_R0?AVexception@std@@@8  10024ef0     libvcruntime:frame.obj
 0003:00001f10       ?gbGdiPlusInitialized@@3_NA 10024f10     ConEmuBg.obj
 0003:00001f11       ?gbInStartPlugin@@3_NA     10024f11     ConEmuBg.obj
 0003:00001f12       ?gbSetStartupInfoOk@@3_NA  10024f12     ConEmuBg.obj
 0003:00001f14       ?gfCreateXmlReader@@3P6GJABU_GUID@@PAPAXPAX@ZA 10024f14     ConEmuBg.obj
 0003:00001f18       ?ghXmlLite@@3PAUHINSTANCE__@@A 10024f18     ConEmuBg.obj
 0003:00001f1c       ?XmlFile@@3UXmlConfigFile@@A 10024f1c     ConEmuBg.obj
 0003:00001f30       ?gpszXmlFile@@3PA_WA       10024f30     ConEmuBg.obj
 0003:00001f34       ?gpszXmlFolder@@3PA_WA     10024f34     ConEmuBg.obj
 0003:00001f38       ?ghXmlNotification@@3PAXA  10024f38     ConEmuBg.obj
 0003:00001f3c       ?gpDecoder@@3PAUGDIPlusDecoder@@A 10024f3c     ConEmuBg.obj
 0003:00001f40       ?ghPluginModule@@3PAUHINSTANCE__@@A 10024f40     ConEmuBg.obj
 0003:00001f44       ?gFarVersion@@3UFarVersion@@A 10024f44     ConEmuBg.obj
 0003:00001f50       ?gbBackgroundEnabled@@3HA  10024f50     ConEmuBg.obj
 0003:00001f54       ?gbMonitorFileChange@@3HA  10024f54     ConEmuBg.obj
 0003:00001f58       ?gsXmlConfigFile@@3PA_WA   10024f58     ConEmuBg.obj
 0003:00002160       ?gbInfoW_OK@@3HA           10025160     ConEmuBg.obj
 0003:00002168       ?_OptionsStorage@?1??__local_stdio_printf_options@@9@4_KA 10025168     ConEmuBg.obj
 0003:00002174       ?InfoW1900@@3PAUPluginStartupInfo@@A 10025174     ConEmuBg1900.obj
 0003:00002178       ?FSFW1900@@3PAUFarStandardFunctions@@A 10025178     ConEmuBg1900.obj
 0003:00002384       ?InfoW2800@@3PAUPluginStartupInfo@@A 10025384     ConEmuBg2800.obj
 0003:00002388       ?FSFW2800@@3PAUFarStandardFunctions@@A 10025388     ConEmuBg2800.obj
 0003:00002594       ?InfoW995@@3PAUPluginStartupInfo@@A 10025594     ConEmuBg995.obj
 0003:00002598       ?FSFW995@@3PAUFarStandardFunctions@@A 10025598     ConEmuBg995.obj
 0003:000027ac       ?InfoA@@3PAUPluginStartupInfo@@A 100257ac     ConEmuBgA.obj
 0003:000027b0       ?FSFA@@3PAUFarStandardFunctions@@A 100257b0     ConEmuBgA.obj
 0003:000028c4       ?ghHeap@@3PAXA             100258c4     common-kernel32:Memory.obj
 0003:000028c8       ?g_LastDeletePtr@@3PAXA    100258c8     common-kernel32:Memory.obj
 0003:000028d0       ?g_ThreadsIdx@@3JA         100258d0     common-kernel32:WThreads.obj
 0003:0000a41c       __tls_index                1002d41c     LIBCMT:tlssup.obj
 0003:0000a440       ___scrt_current_native_startup_state 1002d440     LIBCMT:utility.obj
 0003:0000a444       ___scrt_native_startup_lock 1002d444     LIBCMT:utility.obj
 0003:0000a44c       ___scrt_debugger_hook_flag 1002d44c     LIBCMT:utility_desktop.obj
 0003:0000a450       ?__type_info_root_node@@3U__type_info_node@@A 1002d450     LIBCMT:tncleanup.obj
 0003:0000a458       ?_OptionsStorage@?1??__local_stdio_scanf_options@@9@4_KA 1002d458     LIBCMT:default_local_stdio_options.obj
 0003:0000a460       ___isa_available           1002d460     LIBCMT:_cpu_disp_.obj
 0003:0000a464       ___favor                   1002d464     LIBCMT:_cpu_disp_.obj
 0003:0000a4cc       ___pPurecall               1002d4cc     libvcruntime:purevirt_data.obj
 0003:0000a4d0       ?pArgList@UnDecorator@@0PAVReplicator@@A 1002d4d0     libvcruntime:undname.obj
 0003:0000a4d4       ?pZNameList@UnDecorator@@0PAVReplicator@@A 1002d4d4     libvcruntime:undname.obj
 0003:0000a4d8       ?pTemplateArgList@UnDecorator@@0PAVReplicator@@A 1002d4d8     libvcruntime:undname.obj
 0003:0000a4dc       ?gName@UnDecorator@@0PBDB  1002d4dc     libvcruntime:undname.obj
 0003:0000a4e0       ?name@UnDecorator@@0PBDB   1002d4e0     libvcruntime:undname.obj
 0003:0000a4e4       ?disableFlags@UnDecorator@@0KA 1002d4e4     libvcruntime:undname.obj
 0003:0000a4e8       ?fExplicitTemplateParams@UnDecorator@@0_NA 1002d4e8     libvcruntime:undname.obj
 0003:0000a4e9       ?fGetTemplateArgumentList@UnDecorator@@0_NA 1002d4e9     libvcruntime:undname.obj
 0003:0000a4ec       ?m_pGetParameter@UnDecorator@@0P6APADJ@ZA 1002d4ec     libvcruntime:undname.obj
 0003:0000a4f0       ?m_CHPENameOffset@UnDecorator@@0KA 1002d4f0     libvcruntime:undname.obj
 0003:0000a4f4       ?m_recursionLevel@UnDecorator@@0KA 1002d4f4     libvcruntime:undname.obj
 0003:0000a50c       ?__WinRTOutOfMemoryExceptionCallback@@3P6GPAXXZA 1002d50c     libvcruntime:ehhelpers.obj
 0003:0000a628       __environ_table            1002d628     libucrt:environment_initialization.obj
 0003:0000a62c       __wenviron_table           1002d62c     libucrt:environment_initialization.obj
 0003:0000a630       ___dcrt_initial_wide_environment 1002d630     libucrt:environment_initialization.obj
 0003:0000a634       ___dcrt_initial_narrow_environment 1002d634     libucrt:environment_initialization.obj
 0003:0000a638       ___acrt_atexit_table       1002d638     libucrt:onexit.obj
 0003:0000a644       ___acrt_at_quick_exit_table 1002d644     libucrt:onexit.obj
 0003:0000a654       ___acrt_locale_changed_data 1002d654     libucrt:wsetlocale.obj
 0003:0000a658       ___acrt_current_locale_data 1002d658     libucrt:nlsdata.obj
 0003:0000a65c       __nstream                  1002d65c     libucrt:_file.obj
 0003:0000a660       ___piob                    1002d660     libucrt:_file.obj
 0003:0000a668       ___acrt_stdout_buffer      1002d668     libucrt:_sftbuf.obj
 0003:0000a66c       ___acrt_stderr_buffer      1002d66c     libucrt:_sftbuf.obj
 0003:0000a670       ___pioinfo                 1002d670     libucrt:ioinit.obj
 0003:0000a870       __nhandle                  1002d870     libucrt:ioinit.obj
 0003:0000aa8c       ___mblocalename            1002da8c     libucrt:mbctype.obj
 0003:0000aa90       ___mbcodepage              1002da90     libucrt:mbctype.obj
 0003:0000aa94       ___ismbcodepage            1002da94     libucrt:mbctype.obj
 0003:0000aa98       ___mbulinfo                1002da98     libucrt:mbctype.obj
 0003:0000aaac       ___argc                    1002daac     libucrt:argv_data.obj
 0003:0000aab0       ___argv                    1002dab0     libucrt:argv_data.obj
 0003:0000aab4       ___wargv                   1002dab4     libucrt:argv_data.obj
 0003:0000aab8       __acmdln                   1002dab8     libucrt:argv_data.obj
 0003:0000aabc       __wcmdln                   1002dabc     libucrt:argv_data.obj
 0003:0000aac0       __pgmptr                   1002dac0     libucrt:argv_data.obj
 0003:0000aac4       ___acrt_heap               1002dac4     libucrt:heap_handle.obj
 0003:0000aae0       ___acrt_lconv_static_null  1002dae0     libucrt:localeconv.obj
 0003:0000aae4       ___acrt_lconv_static_W_null 1002dae4     libucrt:localeconv.obj
 0003:0000aaf0       ___fastflag                1002daf0     libucrt:fp_flags.obj
 0003:0000aaf8       ___scrt_ucrt_dll_is_in_use 1002daf8     <common>
 0003:0000aafc       ___dyn_tls_init_callback   1002dafc     <common>
 0003:0000ab00       __pmatherr                 1002db00     <common>
 0003:0000ab04       ___use_sse2_mathfcns       1002db04     <common>

 entry point at        0001:00007574

 Static symbols

 0000:fffcf000       .debug$S                   10000000     kernel32:KERNEL32.dll
 0000:fffcf000       .debug$S                   10000000     ole32:ole32.dll
 0000:fffcf000       .debug$S                   10000000     gdi32:GDI32.dll
 0000:fffcf000       .debug$S                   10000000     gdi32:GDI32.dll
 0000:fffcf000       .debug$S                   10000000     gdi32:GDI32.dll
 0000:fffcf000       .debug$S                   10000000     gdi32:GDI32.dll
 0000:fffcf000       .debug$S                   10000000     gdi32:GDI32.dll
 0000:fffcf000       .debug$S                   10000000     ole32:ole32.dll
 0000:fffcf000       .debug$S                   10000000     advapi32:ADVAPI32.dll
 0000:fffcf000       .debug$S                   10000000     advapi32:ADVAPI32.dll
 0000:fffcf000       .debug$S                   10000000     advapi32:ADVAPI32.dll
 0000:fffcf000       .debug$S                   10000000     advapi32:ADVAPI32.dll
 0000:fffcf000       .debug$S                   10000000     advapi32:ADVAPI32.dll
 0000:fffcf000       .debug$S                   10000000     gdi32:GDI32.dll
 0000:fffcf000       .debug$S                   10000000     gdi32:GDI32.dll
 0000:fffcf000       .debug$S                   10000000     version:VERSION.dll
 0000:fffcf000       .debug$S                   10000000     version:VERSION.dll
 0000:fffcf000       .debug$S                   10000000     version:VERSION.dll
 0000:fffcf000       .debug$S                   10000000     kernel32:KERNEL32.dll
 0000:fffcf000       .debug$S                   10000000     kernel32:KERNEL32.dll
 0000:fffcf000       .debug$S                   10000000     kernel32:KERNEL32.dll
 0000:fffcf000       .debug$S                   10000000     ConEmuBg.exp
 0000:fffcf000       .debug$S                   10000000     kernel32:KERNEL32.dll
 0000:fffcf000       .debug$S                   10000000     kernel32:KERNEL32.dll
 0000:fffcf000       .debug$S                   10000000     kernel32:KERNEL32.dll
 0000:fffcf000       .debug$S                   10000000     kernel32:KERNEL32.dll
 0000:fffcf000       .debug$S                   10000000     kernel32:KERNEL32.dll
 0000:fffcf000       .debug$S                   10000000     kernel32:KERNEL32.dll
 0000:fffcf000       .debug$S                   10000000     kernel32:KERNEL32.dll
 0000:fffcf000       .debug$S                   10000000     kernel32:KERNEL32.dll
 0000:fffcf000       .debug$S                   10000000     kernel32:KERNEL32.dll
 0000:fffcf000       .debug$S                   10000000     kernel32:KERNEL32.dll
 0000:fffcf000       .debug$S                   10000000     kernel32:KERNEL32.dll
 0000:fffcf000       .debug$S                   10000000     kernel32:KERNEL32.dll
 0000:fffcf000       .debug$S                   10000000     kernel32:KERNEL32.dll
 0000:fffcf000       .debug$S                   10000000     kernel32:KERNEL32.dll
 0000:fffcf000       .debug$S                   10000000     kernel32:KERNEL32.dll
 0000:fffcf000       .debug$S                   10000000     kernel32:KERNEL32.dll
 0000:fffcf000       .debug$S                   10000000     kernel32:KERNEL32.dll
 0000:fffcf000       .debug$S                   10000000     kernel32:KERNEL32.dll
 0000:fffcf000       .debug$S                   10000000     kernel32:KERNEL32.dll
 0000:fffcf000       .debug$S                   10000000     kernel32:KERNEL32.dll
 0000:fffcf000       .debug$S                   10000000     kernel32:KERNEL32.dll
 0000:fffcf000       .debug$S                   10000000     kernel32:KERNEL32.dll
 0000:fffcf000       .debug$S                   10000000     kernel32:KERNEL32.dll
 0000:fffcf000       .debug$S                   10000000     kernel32:KERNEL32.dll
 0000:fffcf000       .debug$S                   10000000     kernel32:KERNEL32.dll
 0000:fffcf000       .debug$S                   10000000     kernel32:KERNEL32.dll
 0000:fffcf000       .debug$S                   10000000     kernel32:KERNEL32.dll
 0000:fffcf000       .debug$S                   10000000     kernel32:KERNEL32.dll
 0000:fffcf000       .debug$S                   10000000     kernel32:KERNEL32.dll
 0000:fffcf000       .debug$S                   10000000     kernel32:KERNEL32.dll
 0000:fffcf000       .debug$S                   10000000     kernel32:KERNEL32.dll
 0000:fffcf000       .debug$S                   10000000     kernel32:KERNEL32.dll
 0000:fffcf000       .debug$S                   10000000     kernel32:KERNEL32.dll
 0000:fffcf000       .debug$S                   10000000     kernel32:KERNEL32.dll
 0000:fffcf000       .debug$S                   10000000     kernel32:KERNEL32.dll
 0000:fffcf000       .debug$S                   10000000     kernel32:KERNEL32.dll
 0000:fffcf000       .debug$S                   10000000     kernel32:KERNEL32.dll
 0000:fffcf000       .debug$S                   10000000     kernel32:KERNEL32.dll
 0000:fffcf000       .debug$S                   10000000     kernel32:KERNEL32.dll
 0000:fffcf000       .debug$S                   10000000     kernel32:KERNEL32.dll
 0000:fffcf000       .debug$S                   10000000     kernel32:KERNEL32.dll
 0000:fffcf000       .debug$S                   10000000     kernel32:KERNEL32.dll
 0000:fffcf000       .debug$S                   10000000     kernel32:KERNEL32.dll
 0000:fffcf000       .debug$S                   10000000     kernel32:KERNEL32.dll
 0000:fffcf000       .debug$S                   10000000     kernel32:KERNEL32.dll
 0000:fffcf000       .debug$S                   10000000     kernel32:KERNEL32.dll
 0000:fffcf000       .debug$S                   10000000     kernel32:KERNEL32.dll
 0000:fffcf000       .debug$S                   10000000     kernel32:KERNEL32.dll
 0000:fffcf000       .debug$S                   10000000     kernel32:KERNEL32.dll
 0000:fffcf000       .debug$S                   10000000     kernel32:KERNEL32.dll
 0000:fffcf000       .debug$S                   10000000     kernel32:KERNEL32.dll
 0000:fffcf000       .debug$S                   10000000     kernel32:KERNEL32.dll
 0000:fffcf000       .debug$S                   10000000     kernel32:KERNEL32.dll
 0000:fffcf000       .debug$S                   10000000     kernel32:KERNEL32.dll
 0000:fffcf000       .debug$S                   10000000     kernel32:KERNEL32.dll
 0000:fffcf000       .debug$S                   10000000     kernel32:KERNEL32.dll
 0000:fffcf000       .debug$S                   10000000     kernel32:KERNEL32.dll
 0000:fffcf000       .debug$S                   10000000     kernel32:KERNEL32.dll
 0000:fffcf000       .debug$S                   10000000     kernel32:KERNEL32.dll
 0000:fffcf000       .debug$S                   10000000     kernel32:KERNEL32.dll
 0000:fffcf000       .debug$S                   10000000     kernel32:KERNEL32.dll
 0000:fffcf000       .debug$S                   10000000     kernel32:KERNEL32.dll
 0000:fffcf000       .debug$S                   10000000     kernel32:KERNEL32.dll
 0000:fffcf000       .debug$S                   10000000     kernel32:KERNEL32.dll
 0000:fffcf000       .debug$S                   10000000     kernel32:KERNEL32.dll
 0000:fffcf000       .debug$S                   10000000     kernel32:KERNEL32.dll
 0000:fffcf000       .debug$S                   10000000     kernel32:KERNEL32.dll
 0000:fffcf000       .debug$S                   10000000     kernel32:KERNEL32.dll
 0000:fffcf000       .debug$S                   10000000     kernel32:KERNEL32.dll
 0000:fffcf000       .debug$S                   10000000     kernel32:KERNEL32.dll
 0000:fffcf000       .debug$S                   10000000     kernel32:KERNEL32.dll
 0000:fffcf000       .debug$S                   10000000     kernel32:KERNEL32.dll
 0000:fffcf000       .debug$S                   10000000     kernel32:KERNEL32.dll
 0000:fffcf000       .debug$S                   10000000     kernel32:KERNEL32.dll
 0000:fffcf000       .debug$S                   10000000     kernel32:KERNEL32.dll
 0000:fffcf000       .debug$S                   10000000     kernel32:KERNEL32.dll
 0000:fffcf000       .debug$S                   10000000     kernel32:KERNEL32.dll
 0000:fffcf000       .debug$S                   10000000     kernel32:KERNEL32.dll
 0000:fffcf000       .debug$S                   10000000     kernel32:KERNEL32.dll
 0000:fffcf000       .debug$S                   10000000     kernel32:KERNEL32.dll
 0000:fffcf000       .debug$S                   10000000     kernel32:KERNEL32.dll
 0000:fffcf000       .debug$S                   10000000     kernel32:KERNEL32.dll
 0000:fffcf000       .debug$S                   10000000     kernel32:KERNEL32.dll
 0000:fffcf000       .debug$S                   10000000     kernel32:KERNEL32.dll
 0000:fffcf000       .debug$S                   10000000     kernel32:KERNEL32.dll
 0000:fffcf000       .debug$S                   10000000     kernel32:KERNEL32.dll
 0000:fffcf000       .debug$S                   10000000     kernel32:KERNEL32.dll
 0000:fffcf000       .debug$S                   10000000     kernel32:KERNEL32.dll
 0000:fffcf000       .debug$S                   10000000     kernel32:KERNEL32.dll
 0000:fffcf000       .debug$S                   10000000     kernel32:KERNEL32.dll
 0000:fffcf000       .debug$S                   10000000     kernel32:KERNEL32.dll
 0000:fffcf000       .debug$S                   10000000     kernel32:KERNEL32.dll
 0000:fffcf000       .debug$S                   10000000     kernel32:KERNEL32.dll
 0000:fffcf000       .debug$S                   10000000     kernel32:KERNEL32.dll
 0000:fffcf000       .debug$S                   10000000     kernel32:KERNEL32.dll
 0000:fffcf000       .debug$S                   10000000     kernel32:KERNEL32.dll
 0000:fffcf000       .debug$S                   10000000     kernel32:KERNEL32.dll
 0000:fffcf000       .debug$S                   10000000     gdi32:GDI32.dll
 0000:fffcf000       .debug$S                   10000000     kernel32:KERNEL32.dll
 0000:fffcf000       .debug$S                   10000000     kernel32:KERNEL32.dll
 0000:fffcf000       .debug$S                   10000000     kernel32:KERNEL32.dll
 0000:fffcf000       .debug$S                   10000000     kernel32:KERNEL32.dll
 0000:fffcf000       .debug$S                   10000000     kernel32:KERNEL32.dll
 0000:fffcf000       .debug$S                   10000000     kernel32:KERNEL32.dll
 0000:fffcf000       .debug$S                   10000000     kernel32:KERNEL32.dll
 0000:fffcf000       .debug$S                   10000000     kernel32:KERNEL32.dll
 0000:fffcf000       .debug$S                   10000000     kernel32:KERNEL32.dll
 0000:fffcf000       .debug$S                   10000000     kernel32:KERNEL32.dll
 0000:fffcf000       .debug$S                   10000000     kernel32:KERNEL32.dll
 0000:fffcf000       .debug$S                   10000000     kernel32:KERNEL32.dll
 0000:fffcf000       .debug$S                   10000000     kernel32:KERNEL32.dll
 0000:fffcf000       .debug$S                   10000000     kernel32:KERNEL32.dll
 0000:fffcf000       .debug$S                   10000000     kernel32:KERNEL32.dll
 0000:fffcf000       .debug$S                   10000000     kernel32:KERNEL32.dll
 0000:fffcf000       .debug$S                   10000000     kernel32:KERNEL32.dll
 0000:fffcf000       .debug$S                   10000000     kernel32:KERNEL32.dll
 0000:fffcf000       .debug$S                   10000000     kernel32:KERNEL32.dll
 0000:fffcf000       .debug$S                   10000000     kernel32:KERNEL32.dll
 0000:fffcf000       .debug$S                   10000000     user32:USER32.dll
 0000:fffcf000       .debug$S                   10000000     user32:USER32.dll
 0000:fffcf000       .debug$S                   10000000     user32:USER32.dll
 0000:fffcf000       .debug$S                   10000000     user32:USER32.dll
 0000:fffcf000       .debug$S                   10000000     user32:USER32.dll
 0000:fffcf000       .debug$S                   10000000     user32:USER32.dll
 0000:fffcf000       .debug$S                   10000000     user32:USER32.dll
 0000:fffcf000       .debug$S                   10000000     gdi32:GDI32.dll
 0000:fffcf000       .debug$S                   10000000     gdi32:GDI32.dll
 0000:fffcf000       .debug$S                   10000000     gdi32:GDI32.dll
 0001:00000196       ?ChangeExports@@YA_NPBUExportFunc@@PAUHINSTANCE__@@@Z 10001196 f   ConEmuBg.obj
 0001:000027e2       ?LoadFarVersion@@YA_NAAUFarVersion@@AAY0CAA@_W@Z 100037e2 f   ConEmuBg.obj
 0001:00002872       ?LoadFarVersion@@YA_NPB_WAAUFarVersion@@AAY0CAA@_W@Z 10003872 f   ConEmuBg.obj
 0001:000028f6       ?LoadModuleVersion@@YA_NPB_WAAUtagVS_FIXEDFILEINFO@@PA_WI@Z 100038f6 f   ConEmuBg.obj
 0001:00004664       ?StringCopyWorkerW@@YGJPA_WIPAIPB_WI@Z 10005664 f   ConEmuBg.obj
 0001:000046c9       ?StringLengthWorkerW@@YGJPB_WIPAI@Z 100056c9 f   ConEmuBg.obj
 0001:00004710       ?StringValidateDestAndLengthW@@YGJPB_WIPAII@Z 10005710 f   ConEmuBg.obj
 0001:000048d5       ?ConfigDlgProc@@YGHPAXHH0@Z 100058d5 f   ConEmuBg1900.obj
 0001:00004979       ?ConfigureProc@@YAHH@Z     10005979 f   ConEmuBg1900.obj
 0001:00005066       ?ConfigDlgProc@@YGHPAXHH0@Z 10006066 f   ConEmuBg2800.obj
 0001:0000510a       ?ConfigureProc@@YAHH@Z     1000610a f   ConEmuBg2800.obj
 0001:00005854       ?ConfigDlgProc@@YGJPAXHHJ@Z 10006854 f   ConEmuBg995.obj
 0001:000058f8       ?ConfigureProc@@YAHH@Z     100068f8 f   ConEmuBg995.obj
 0001:00005dfc       ?ConfigDlgProc@@YGJPAXHHJ@Z 10006dfc f   ConEmuBgA.obj
 0001:00005eaa       ?ConfigureProc@@YAHH@Z     10006eaa f   ConEmuBgA.obj
 0001:00006f10       $$000000                   10007f10     LIBCMT:llmul.obj
 0001:00006f50       $$000000                   10007f50     LIBCMT:ulldiv.obj
 0001:00006fdb       ?__scrt_initialize_thread_safe_statics@@YAHXZ 10007fdb f   LIBCMT:thread_safe_statics.obj
 0001:0000701f       ?__scrt_initialize_thread_safe_statics_platform_specific@@YAXXZ 1000801f f   LIBCMT:thread_safe_statics.obj
 0001:0000710e       ?__scrt_uninitialize_thread_safe_statics@@YAXXZ 1000810e f   LIBCMT:thread_safe_statics.obj
 0001:00007268       ?dllmain_crt_dispatch@@YGHQAUHINSTANCE__@@KQAX@Z 10008268 f   LIBCMT:dll_dllmain.obj
 0001:000072bb       ?dllmain_crt_process_attach@@YAHQAUHINSTANCE__@@QAX@Z 100082bb f   LIBCMT:dll_dllmain.obj
 0001:000073b8       ?dllmain_crt_process_detach@@YAH_N@Z 100083b8 f   LIBCMT:dll_dllmain.obj
 0001:0000743e       ?dllmain_dispatch@@YAHQAUHINSTANCE__@@KQAX@Z 1000843e f   LIBCMT:dll_dllmain.obj
 0001:000075a0       $$000000                   100085a0     LIBCMT:_sehprolg4_.obj
 0001:000075fb       ?find_pe_section@@YAPAU_IMAGE_SECTION_HEADER@@QAEI@Z 100085fb f   LIBCMT:utility.obj
 0001:00007a61       ___get_entropy             10008a61 f   LIBCMT:gs_support.obj
 0001:000084e0       $$000000                   100094e0     libvcruntime:memmove.obj
 0001:00008744       TrailingUpVec              10009744     libvcruntime:memmove.obj
 0001:000087f0       TrailingDownVec            100097f0     libvcruntime:memmove.obj
 0001:00008a60       $$000000                   10009a60     libvcruntime:memset.obj
 0001:00008bc0       $$000000                   10009bc0     libvcruntime:strchr.obj
 0001:00008cf0       $$000000                   10009cf0     libvcruntime:strrchr.obj
 0001:00008e30       _ValidateLocalCookies      10009e30 f   libvcruntime:_chandler4_.obj
 0001:000091f0       $$000000                   1000a1f0     libvcruntime:lowhelpr.obj
 0001:000092f8       ?CallCatchBlock@@YAPAXPAUEHExceptionRecord@@PAUEHRegistrationNode@@PAU_CONTEXT@@PBU_s_FuncInfo@@PAXHK@Z 1000a2f8 f   libvcruntime:frame.obj
 0001:000094b4       ?CallUnexpected@@YAXPBU_s_ESTypeList@@@Z 1000a4b4 f   libvcruntime:frame.obj
 0001:000094d4       __catch$?CallUnexpected@@YAXPBU_s_ESTypeList@@@Z$0 1000a4d4 f   libvcruntime:frame.obj
 0001:000094ee       ?CatchIt@@YAXPAUEHExceptionRecord@@PAUEHRegistrationNode@@PAU_CONTEXT@@PAXPBU_s_FuncInfo@@PBU_s_HandlerType@@PBU_s_CatchableType@@PBU_s_TryBlockMapEntry@@H1E@Z 1000a4ee f   libvcruntime:frame.obj
 0001:00009567       ?ExFilterRethrow@@YAHPAU_EXCEPTION_POINTERS@@@Z 1000a567 f   libvcruntime:frame.obj
 0001:000095b1       ?FindHandler@@YAXPAUEHExceptionRecord@@PAUEHRegistrationNode@@PAU_CONTEXT@@PAXPBU_s_FuncInfo@@EH1@Z 1000a5b1 f   libvcruntime:frame.obj
 0001:00009932       ?FindHandlerForForeignException@@YAXPAUEHExceptionRecord@@PAUEHRegistrationNode@@PAU_CONTEXT@@PAXPBU_s_FuncInfo@@HH1@Z 1000a932 f   libvcruntime:frame.obj
 0001:00009a4d       ?IsInExceptionSpec@@YAEPAUEHExceptionRecord@@PBU_s_ESTypeList@@@Z 1000aa4d f   libvcruntime:frame.obj
 0001:00009fa0       $$000000                   1000afa0     libvcruntime:_exsup4_.obj
 0001:0000a030       __unwind_handler4          1000b030 f   libvcruntime:_exsup4_.obj
 0001:0000a172       ?try_get_first_available_module@@YAPAUHINSTANCE__@@QBW4module_id@?A0x9a4b7766@@0@Z 1000b172 f   libvcruntime:winapi_downlevel.obj
 0001:0000a238       ?try_get_function@@YAPAXW4function_id@?A0x9a4b7766@@QBDQBW4module_id@2@2@Z 1000b238 f   libvcruntime:winapi_downlevel.obj
 0001:0000a450       $$000000                   1000b450     libvcruntime:_exsup_.obj
 0001:0000a471       __unwind_handler           1000b471 f   libvcruntime:_exsup_.obj
 0001:0000a7d0       $$000000                   1000b7d0     libvcruntime:memcpy.obj
 0001:0000aa34       TrailingUpVec              1000ba34     libvcruntime:memcpy.obj
 0001:0000aae0       TrailingDownVec            1000bae0     libvcruntime:memcpy.obj
 0001:0000b872       ??$common_vsprintf@Vstandard_base@__crt_stdio_output@@D@@YAH_KQADIQBDQAU__crt_locale_pointers@@1@Z 1000c872 f   libucrt:output.obj
 0001:0000b9ee       ??$common_vsprintf@Vstandard_base@__crt_stdio_output@@_W@@YAH_KQA_WIQB_WQAU__crt_locale_pointers@@QAD@Z 1000c9ee f   libucrt:output.obj
 0001:0000c29a       $LN54                      1000d29a     libucrt:output.obj
 0001:0000c3ba       $LN54                      1000d3ba     libucrt:output.obj
 0001:0000cd7d       $LN19                      1000dd7d     libucrt:output.obj
 0001:0000db1f       ?atexit_exception_filter@@YAHK@Z 1000eb1f f   libucrt:exit.obj
 0001:0000db32       ?common_exit@@YAXHW4_crt_exit_cleanup_mode@@W4_crt_exit_return_mode@@@Z 1000eb32 f   libucrt:exit.obj
 0001:0000dc4b       ?exit_or_terminate_process@@YAXI@Z 1000ec4b f   libucrt:exit.obj
 0001:0000dc8c       ?is_managed_app@@YA_NXZ    1000ec8c f   libucrt:exit.obj
 0001:0000dcd0       ?try_cor_exit_process@@YAXI@Z 1000ecd0 f   libucrt:exit.obj
 0001:0000dd74       ??$common_configure_argv@D@@YAHW4_crt_argv_mode@@@Z 1000ed74 f   libucrt:argv_parsing.obj
 0001:0000de98       ??$parse_command_line@D@@YAXPADPAPAD0PAI2@Z 1000ee98 f   libucrt:argv_parsing.obj
 0001:0000e06d       ??$common_initialize_environment_nolock@D@@YAHXZ 1000f06d f   libucrt:environment_initialization.obj
 0001:0000e0c6       ??$create_environment@D@@YAQAPADQAD@Z 1000f0c6 f   libucrt:environment_initialization.obj
 0001:0000e197       ??$free_environment@_W@@YAXQAPA_W@Z 1000f197 f   libucrt:environment_initialization.obj
 0001:0000e197       ??$free_environment@D@@YAXQAPAD@Z 1000f197 f   libucrt:environment_initialization.obj
 0001:0000e206       ??$uninitialize_environment_internal@D@@YAXAAPAPAD@Z 1000f206 f   libucrt:environment_initialization.obj
 0001:0000e221       ??$uninitialize_environment_internal@_W@@YAXAAPAPA_W@Z 1000f221 f   libucrt:environment_initialization.obj
 0001:0000e3ba       ??R<lambda_275893d493268fdec8709772e3fcec0e>@@QBEHXZ 1000f3ba f   libucrt:onexit.obj
 0001:0000e4da       ??R<lambda_4e60a939b0d047cfe11ddc22648dfba9>@@QBEHXZ 1000f4da f   libucrt:onexit.obj
 0001:0000e6af       _initialize_global_variables 1000f6af f   libucrt:initialization.obj
 0001:0000e6c1       _initialize_c              1000f6c1 f   libucrt:initialization.obj
 0001:0000e6db       _uninitialize_c            1000f6db f   libucrt:initialization.obj
 0001:0000e6db       _initialize_environment    1000f6db f   libucrt:initialization.obj
 0001:0000e6db       _report_memory_leaks       1000f6db f   libucrt:initialization.obj
 0001:0000e6db       _initialize_global_state_isolation 1000f6db f   libucrt:initialization.obj
 0001:0000e6db       _uninitialize_global_state_isolation 1000f6db f   libucrt:initialization.obj
 0001:0000e6de       _uninitialize_environment  1000f6de f   libucrt:initialization.obj
 0001:0000e6e6       _initialize_pointers       1000f6e6 f   libucrt:initialization.obj
 0001:0000e723       _uninitialize_vcruntime    1000f723 f   libucrt:initialization.obj
 0001:0000e72c       _uninitialize_allocated_memory 1000f72c f   libucrt:initialization.obj
 0001:0000e8e0       $$000000                   1000f8e0     libucrt:strncmp.obj
 0001:0000ef2c       ?construct_ptd@@YAXQAU__acrt_ptd@@QAPAU__crt_locale_data@@@Z 1000ff2c f   libucrt:per_thread_data.obj
 0001:0000efa5       ?destroy_fls@@YGXPAX@Z     1000ffa5 f   libucrt:per_thread_data.obj
 0001:0000efc6       ?destroy_ptd@@YAXQAU__acrt_ptd@@@Z 1000ffc6 f   libucrt:per_thread_data.obj
 0001:0000f06f       ?replace_current_thread_locale_nolock@@YAXQAU__acrt_ptd@@QAU__crt_locale_data@@@Z 1001006f f   libucrt:per_thread_data.obj
 0001:0000f351       ??$common_tox_l@$1?internal_isupper_l@@YA_NHQAU__crt_locale_pointers@@@Z$1?internal_map_lower@@YAHH0@Z@@YAHHKQAU__crt_locale_pointers@@@Z 10010351 f   libucrt:tolower_toupper.obj
 0001:0000f49b       ?internal_isupper_l@@YA_NHQAU__crt_locale_pointers@@@Z 1001049b f   libucrt:tolower_toupper.obj
 0001:0000fb44       ?fp_format_a@@YAHQBNPADIQADIH_NIQAU__crt_locale_pointers@@@Z 10010b44 f   libucrt:cvt.obj
 0001:0000fe47       ?fp_format_e@@YAHQBNQADI1IH_NIQAU__crt_locale_pointers@@@Z 10010e47 f   libucrt:cvt.obj
 0001:0000fee2       ?fp_format_e_internal@@YAHQADIH_NIQAU_strflt@@1QAU__crt_locale_pointers@@@Z 10010ee2 f   libucrt:cvt.obj
 0001:0001002d       ?fp_format_f@@YAHQBNQADI1IHQAU__crt_locale_pointers@@@Z 1001102d f   libucrt:cvt.obj
 0001:000100ba       ?fp_format_f_internal@@YAHQADIHQAU_strflt@@_NQAU__crt_locale_pointers@@@Z 100110ba f   libucrt:cvt.obj
 0001:00010191       ?fp_format_g@@YAHQBNQADI1IH_NIQAU__crt_locale_pointers@@@Z 10011191 f   libucrt:cvt.obj
 0001:00010259       ?fp_format_nan_or_infinity@@YAHW4__acrt_fp_class@@_NPADI1@Z 10011259 f   libucrt:cvt.obj
 0001:00010351       ?shift_bytes@@YAXQADI0H@Z  10011351 f   libucrt:cvt.obj
 0001:00010646       ?initialize_inherited_file_handles_nolock@@YAXXZ 10011646 f   libucrt:ioinit.obj
 0001:000106fc       ?initialize_stdio_handles_nolock@@YAXXZ 100116fc f   libucrt:ioinit.obj
 0001:000108d4       ?try_get_function@@YAPAXW4function_id@?A0x352e5c4b@@QBDQBW4module_id@2@2@Z 100118d4 f   libucrt:winapi_thunks.obj
 0001:00010970       ?try_get_module@@YAPAUHINSTANCE__@@W4module_id@?A0x352e5c4b@@@Z 10011970 f   libucrt:winapi_thunks.obj
 0001:00010dcc       ?<helper_func_cdecl>@<lambda_62bb7ecb46d0a77b591a051c43eb5ad1>@@CAHPBX0@Z 10011dcc f   libucrt:argv_wildcards.obj
 0001:00010de4       ??$common_expand_argv_wildcards@D@@YAHQAPADQAPAPAD@Z 10011de4 f   libucrt:argv_wildcards.obj
 0001:00010f74       ??$copy_and_add_argument_to_buffer@D@@YAHQBD0IAAV?$argument_list@D@?A0xb0e4b824@@@Z 10011f74 f   libucrt:argv_wildcards.obj
 0001:0001100a       ??$expand_argument_wildcards@D@@YAHQAD0AAV?$argument_list@D@?A0xb0e4b824@@@Z 1001200a f   libucrt:argv_wildcards.obj
 0001:000112e5       ??R<lambda_ad1ced32f4ac17aa236e5ef05d6b3b7c>@@QBEXXZ 100122e5 f   libucrt:mbctype.obj
 0001:000113a9       ?CPtoLocaleName@@YAPB_WH@Z 100123a9 f   libucrt:mbctype.obj
 0001:000113e7       ?getSystemCP@@YAHH@Z       100123e7 f   libucrt:mbctype.obj
 0001:0001145a       ?setSBCS@@YAXPAU__crt_multibyte_data@@@Z 1001245a f   libucrt:mbctype.obj
 0001:000114bf       ?setSBUpLow@@YAXPAU__crt_multibyte_data@@@Z 100124bf f   libucrt:mbctype.obj
 0001:00011653       ?setmbcp_internal@@YAHH_N@Z 10012653 f   libucrt:mbctype.obj
 0001:00011a05       _memcpy_s                  10012a05 f   libucrt:mbctype.obj
 0001:00011a05       _memcpy_s                  10012a05 f   libucrt:cfout.obj
 0001:00011a86       ?x_ismbbtype_l@@YAHPAU__crt_locale_pointers@@IHH@Z 10012a86 f   libucrt:ismbbyte.obj
 0001:00011b10       ?find_end_of_double_null_terminated_sequence@@YAPB_WQB_W@Z 10012b10 f   libucrt:get_environment_from_os.obj
 0001:00011e59       ?get_global_action_nolock@@YAPAP6AXH@ZH@Z 10012e59 f   libucrt:signal.obj
 0001:00011e9b       ?siglookup@@YAPAU__crt_signal_action_t@@HQAU1@@Z 10012e9b f   libucrt:signal.obj
 0001:0001280a       ?free_crt_array_internal@@YAXQAPBXI@Z 1001380a f   libucrt:inittime.obj
 0001:0001292a       ?__acrt_LCMapStringA_stat@@YAHPAU__crt_locale_pointers@@PB_WKPBDHPADHHH@Z 1001392a f   libucrt:lcmapstringa.obj
 0001:00014620       _common_flush_all          10015620 f   libucrt:fflush.obj
 0001:00014a14       ?GetTableIndexFromLocaleName@@YAHPB_W@Z 10015a14 f   libucrt:lcidtoname_downlevel.obj
 0001:00014b00       ?shortsort@@YAXPAD0IP6AHPBX1@Z@Z 10015b00 f   libucrt:qsort.obj
 0001:00014ba0       ?swap@@YAXPAD0I@Z          10015ba0 f   libucrt:qsort.obj
 0001:00014f7a       ??$common_tcsncpy_s@D@@YAHQADIQBDI@Z 10015f7a f   libucrt:strncpy_s.obj
 0001:00015040       $$000000                   10016040     libucrt:strpbrk.obj
 0001:00015124       ?initialize_multibyte@@YAHXZ 10016124 f   libucrt:multibyte_initializer.obj
 0001:000152a0       $$000000                   100162a0     libucrt:log10.obj
 0001:000153f0       $$000000                   100163f0     libucrt:ceil_pentium4.obj
 0001:0001550d       ?write_double_translated_ansi_nolock@@YA?AUwrite_result@?A0x47fa6670@@HQBDI@Z 1001650d f   libucrt:write.obj
 0001:000156c0       ?write_double_translated_unicode_nolock@@YA?AUwrite_result@?A0x47fa6670@@QBDI@Z 100166c0 f   libucrt:write.obj
 0001:0001572d       ?write_requires_double_translation_nolock@@YA_NH@Z 1001672d f   libucrt:write.obj
 0001:000157a3       ?write_text_ansi_nolock@@YA?AUwrite_result@?A0x47fa6670@@HQBDI@Z 100167a3 f   libucrt:write.obj
 0001:00015882       ?write_text_utf16le_nolock@@YA?AUwrite_result@?A0x47fa6670@@HQBDI@Z 10016882 f   libucrt:write.obj
 0001:00015970       ?write_text_utf8_nolock@@YA?AUwrite_result@?A0x47fa6670@@HQBDI@Z 10016970 f   libucrt:write.obj
 0001:00015d94       ??$common_lseek_nolock@_J@@YA_JH_JH@Z 10016d94 f   libucrt:lseek.obj
 0001:00016058       ___get_abstract_control_sse2 10017058 f   libucrt:_fenvutils.obj
 0001:000160d5       ___get_abstract_control_x87 100170d5 f   libucrt:_fenvutils.obj
 0001:00016148       ___get_machine_control     10017148 f   libucrt:_fenvutils.obj
 0001:000161b9       ___get_machine_control_sse2 100171b9 f   libucrt:_fenvutils.obj
 0001:00016239       ___get_machine_status_sse2 10017239 f   libucrt:_fenvutils.obj
 0001:0001629a       ___get_machine_status_x87  1001729a f   libucrt:_fenvutils.obj
 0001:000165e0       $$000000                   100175e0     libucrt:log10_pentium4.obj
 0001:00016870       $$000000                   10017870     libucrt:87tran.obj
 0001:00016a70       $$000000                   10017a70     libucrt:87disp.obj
 0001:00016c70       $$000000                   10017c70     libucrt:common.obj
 0001:00016e00       $$000000                   10017e00     libucrt:genexcep.obj
 0001:00017370       $$000000                   10018370     libucrt:_strnicm.obj
 0001:00018190       $$000000                   10019190     LIBCMT:ulldvrm.obj
 0001:00018230       $$000000                   10019230     LIBCMT:_sehprolg4gs_.obj
 0001:00018290       $$000000                   10019290     LIBCMT:lldvrm.obj
 0001:00018370       $$000000                   10019370     LIBCMT:ullshr.obj
 0001:00018390       $$000000                   10019390     LIBCMT:alloca16.obj
 0001:000183c0       $$000000                   100193c0     LIBCMT:llshl.obj
 0001:000183e0       $$000000                   100193e0     LIBCMT:_ftol2_.obj
 0001:000184a0       $$000000                   100194a0     LIBCMT:chkstk.obj
 0001:000184cd       __unwindfunclet$?CheckXmlFile@@YA_N_N@Z$1 100194cd f   ConEmuBg.obj
 0001:000184d8       __ehhandler$?CheckXmlFile@@YA_N_N@Z 100194d8 f   ConEmuBg.obj
 0001:00018500       __unwindfunclet$?FillPanelParams@@YAHPAUPaintBackgroundArg@@PAUBkPanelInfo@@PAUDrawInfo@@@Z$2 10019500 f   ConEmuBg.obj
 0001:0001850b       __unwindfunclet$?FillPanelParams@@YAHPAUPaintBackgroundArg@@PAUBkPanelInfo@@PAUDrawInfo@@@Z$3 1001950b f   ConEmuBg.obj
 0001:00018516       __ehhandler$?FillPanelParams@@YAHPAUPaintBackgroundArg@@PAUBkPanelInfo@@PAUDrawInfo@@@Z 10019516 f   ConEmuBg.obj
 0001:0001853e       __unwindfunclet$?GdipDone@@YAXXZ$0 1001953e f   ConEmuBg.obj
 0001:00018546       __ehhandler$?GdipDone@@YAXXZ 10019546 f   ConEmuBg.obj
 0001:00018561       __unwindfunclet$?StartPlugin@@YAXH@Z$0 10019561 f   ConEmuBg.obj
 0001:0001856e       __ehhandler$?StartPlugin@@YAXH@Z 1001956e f   ConEmuBg.obj
 0001:00018589       __ehhandler$?__scrt_initialize_thread_safe_statics_platform_specific@@YAXXZ 10019589 f   LIBCMT:thread_safe_statics.obj
 0001:000185a4       __ehhandler$?CallUnexpected@@YAXPBU_s_ESTypeList@@@Z 100195a4 f   libvcruntime:frame.obj
 0002:0000023c       ?__scrt_initialize_tss_var@@3P6AHXZA 1001a23c     LIBCMT:thread_safe_statics.obj
 0002:00001490       _GS_ExceptionPointers      1001b490     LIBCMT:gs_report.obj
 0002:00001594       ?module_names@?A0x9a4b7766@@3QBQB_WB 1001b594     libvcruntime:winapi_downlevel.obj
 0002:0000164c       ?candidate_modules@?1??try_get_FlsAlloc@@YAP6GKP6GXPAX@Z@ZXZ@4QBW4module_id@?A0x9a4b7766@@B 1001b64c     libvcruntime:winapi_downlevel.obj
 0002:00001660       ?candidate_modules@?1??try_get_FlsFree@@YAP6GHK@ZXZ@4QBW4module_id@?A0x9a4b7766@@B 1001b660     libvcruntime:winapi_downlevel.obj
 0002:00001670       ?candidate_modules@?1??try_get_FlsGetValue@@YAP6GPAXK@ZXZ@4QBW4module_id@?A0x9a4b7766@@B 1001b670     libvcruntime:winapi_downlevel.obj
 0002:00001684       ?candidate_modules@?1??try_get_FlsSetValue@@YAP6GHKPAX@ZXZ@4QBW4module_id@?A0x9a4b7766@@B 1001b684     libvcruntime:winapi_downlevel.obj
 0002:00001698       ?candidate_modules@?1??try_get_InitializeCriticalSectionEx@@YAP6GHPAU_RTL_CRITICAL_SECTION@@KK@ZXZ@4QBW4module_id@?A0x9a4b7766@@B 1001b698     libvcruntime:winapi_downlevel.obj
 0002:000016c0       ?tokenTable@@3QBQBDB       1001b6c0     libvcruntime:undname.obj
 0002:000016fc       ?rttiTable@@3QBQBDB        1001b6fc     libvcruntime:undname.obj
 0002:00001710       ?nameTable@@3QBQBDB        1001b710     libvcruntime:undname.obj
 0002:00001e48       ?ExceptionTemplate@?1??_CxxThrowException@@9@8@4UEHExceptionRecord@@B 1001be48     libvcruntime:throw.obj
 0002:00001fa8       ___acrt_initializers       1001bfa8     libucrt:initialization.obj
 0002:00002020       _errtable                  1001c020     libucrt:errno.obj
 0002:00002ea0       _module_names              1001cea0     libucrt:winapi_thunks.obj
 0002:00003354       ?candidate_modules@?1??try_get_FlsAlloc@@YAP6GKP6GXPAX@Z@ZXZ@4QBW4module_id@?A0x352e5c4b@@B 1001d354     libucrt:winapi_thunks.obj
 0002:0000335c       ?candidate_modules@?1??try_get_FlsFree@@YAP6GHK@ZXZ@4QBW4module_id@?A0x352e5c4b@@B 1001d35c     libucrt:winapi_thunks.obj
 0002:00003364       ?candidate_modules@?1??try_get_FlsGetValue@@YAP6GPAXK@ZXZ@4QBW4module_id@?A0x352e5c4b@@B 1001d364     libucrt:winapi_thunks.obj
 0002:0000336c       ?candidate_modules@?1??try_get_FlsSetValue@@YAP6GHKPAX@ZXZ@4QBW4module_id@?A0x352e5c4b@@B 1001d36c     libucrt:winapi_thunks.obj
 0002:00003374       ?candidate_modules@?1??try_get_GetCurrentPackageId@@YAP6GJPAIPAE@ZXZ@4QBW4module_id@?A0x352e5c4b@@B 1001d374     libucrt:winapi_thunks.obj
 0002:00003390       ?candidate_modules@?1??try_get_InitializeCriticalSectionEx@@YAP6GHPAU_RTL_CRITICAL_SECTION@@KK@ZXZ@4QBW4module_id@?A0x352e5c4b@@B 1001d390     libucrt:winapi_thunks.obj
 0002:00003398       ?candidate_modules@?1??try_get_LCMapStringEx@@YAP6GHPB_WK0HPA_WHPAU_nlsversioninfo@@PAXJ@ZXZ@4QBW4module_id@?A0x352e5c4b@@B 1001d398     libucrt:winapi_thunks.obj
 0002:000033b0       ?candidate_modules@?1??try_get_LocaleNameToLCID@@YAP6GKPB_WK@ZXZ@4QBW4module_id@?A0x352e5c4b@@B 1001d3b0     libucrt:winapi_thunks.obj
 0002:000033cc       __mb_locale_names          1001d3cc     libucrt:mbctype.obj
 0002:00003e00       _LcidToLocaleNameTable     1001de00     libucrt:lcidtoname_downlevel.obj
 0002:00004f20       _LocaleNameToIndexTable    1001ef20     libucrt:lcidtoname_downlevel.obj
 0002:00005e70       LOG_name                   1001fe70     libucrt:log10.obj
 0002:00005e80       _One                       1001fe80     libucrt:ceil_pentium4.obj
 0002:00005e90       _Bns                       1001fe90     libucrt:ceil_pentium4.obj
 0002:00005ea0       _Zero                      1001fea0     libucrt:ceil_pentium4.obj
 0002:00005eb0       _S                         1001feb0     libucrt:ceil_pentium4.obj
 0002:00005ec0       _NegZero                   1001fec0     libucrt:ceil_pentium4.obj
 0002:00005ed0       emask                      1001fed0     libucrt:log10_pentium4.obj
 0002:00005ee0       CC                         1001fee0     libucrt:log10_pentium4.obj
 0002:00005ef0       Magic                      1001fef0     libucrt:log10_pentium4.obj
 0002:00005f00       hi_mask                    1001ff00     libucrt:log10_pentium4.obj
 0002:00005f10       LOG10_2                    1001ff10     libucrt:log10_pentium4.obj
 0002:00005f20       place_L                    1001ff20     libucrt:log10_pentium4.obj
 0002:00005f40       One                        1001ff40     libucrt:log10_pentium4.obj
 0002:00005f50       Zero                       1001ff50     libucrt:log10_pentium4.obj
 0002:00005f60       Two52                      1001ff60     libucrt:log10_pentium4.obj
 0002:00005f70       Infs                       1001ff70     libucrt:log10_pentium4.obj
 0002:00005f80       NaN                        1001ff80     libucrt:log10_pentium4.obj
 0002:00005f90       coeff                      1001ff90     libucrt:log10_pentium4.obj
 0002:00005fee       _log2max                   1001ffee     libucrt:87tran.obj
 0002:00005ff8       _smallarg                  1001fff8     libucrt:87tran.obj
 0002:00006002       _half                      10020002     libucrt:87tran.obj
 0002:0000604e       One                        1002004e     libucrt:87disp.obj
 0002:00006056       Three                      10020056     libucrt:87disp.obj
 0002:0000605e       XAMtoTagTab                1002005e     libucrt:87disp.obj
 0002:00006070       One                        10020070     libucrt:common.obj
 0002:00006084       DblMax                     10020084     libucrt:common.obj
 0002:0000608c       DblMin                     1002008c     libucrt:common.obj
 0002:00006094       IeeeAdjO                   10020094     libucrt:common.obj
 0002:0000609c       IeeeAdjU                   1002009c     libucrt:common.obj
 0002:000060a4       _infinity                  100200a4     libucrt:common.obj
 0002:000060ac       _zero                      100200ac     libucrt:common.obj
 0002:000060e8       _over                      100200e8     libucrt:fpctrl.obj
 0002:000060f4       _under                     100200f4     libucrt:fpctrl.obj
 0002:000069b8       ?_names@?1??_get_fname@@9@9 100209b8     libucrt:fpexcept.obj
 0002:00007198       __unwindtable$?CheckXmlFile@@YA_N_N@Z 10021198     ConEmuBg.obj
 0002:000071a0       __ehfuncinfo$?CheckXmlFile@@YA_N_N@Z 100211a0     ConEmuBg.obj
 0002:000071c4       __unwindtable$?StartPlugin@@YAXH@Z 100211c4     ConEmuBg.obj
 0002:000071cc       __ehfuncinfo$?StartPlugin@@YAXH@Z 100211cc     ConEmuBg.obj
 0002:000071f0       __unwindtable$?GdipDone@@YAXXZ 100211f0     ConEmuBg.obj
 0002:000071f8       __ehfuncinfo$?GdipDone@@YAXXZ 100211f8     ConEmuBg.obj
 0002:0000721c       __unwindtable$?FillPanelParams@@YAHPAUPaintBackgroundArg@@PAUBkPanelInfo@@PAUDrawInfo@@@Z 1002121c     ConEmuBg.obj
 0002:0000722c       __ehfuncinfo$?FillPanelParams@@YAHPAUPaintBackgroundArg@@PAUBkPanelInfo@@PAUDrawInfo@@@Z 1002122c     ConEmuBg.obj
 0002:00007250       __sehtable$?SetThreadName@@YAXKPAD@Z 10021250     common-kernel32:WThreads.obj
 0002:0000726c       __ehfuncinfo$?__scrt_initialize_thread_safe_statics_platform_specific@@YAXXZ 1002126c     LIBCMT:thread_safe_statics.obj
 0002:00007290       __sehtable$?dllmain_crt_process_attach@@YAHQAUHINSTANCE__@@QAX@Z 10021290     LIBCMT:dll_dllmain.obj
 0002:000072b0       __sehtable$?dllmain_crt_process_detach@@YAH_N@Z 100212b0     LIBCMT:dll_dllmain.obj
 0002:000072d0       __sehtable$?dllmain_dispatch@@YAHQAUHINSTANCE__@@KQAX@Z 100212d0     LIBCMT:dll_dllmain.obj
 0002:000072f0       __sehtable$___scrt_is_nonwritable_in_current_image 100212f0     LIBCMT:utility.obj
 0002:00007310       __sehtable$___BuildCatchObject 10021310     libvcruntime:frame.obj
 0002:00007330       __sehtable$___FrameUnwindToState 10021330     libvcruntime:frame.obj
 0002:00007358       __sehtable$?CallCatchBlock@@YAPAXPAUEHExceptionRecord@@PAUEHRegistrationNode@@PAU_CONTEXT@@PBU_s_FuncInfo@@PAXHK@Z 10021358     libvcruntime:frame.obj
 0002:00007380       __catchsym$?CallUnexpected@@YAXPBU_s_ESTypeList@@@Z$2 10021380     libvcruntime:frame.obj
 0002:00007390       __unwindtable$?CallUnexpected@@YAXPBU_s_ESTypeList@@@Z 10021390     libvcruntime:frame.obj
 0002:000073a0       __tryblocktable$?CallUnexpected@@YAXPBU_s_ESTypeList@@@Z 100213a0     libvcruntime:frame.obj
 0002:000073b4       __ehfuncinfo$?CallUnexpected@@YAXPBU_s_ESTypeList@@@Z 100213b4     libvcruntime:frame.obj
 0002:000073d8       __sehtable$___BuildCatchObjectHelper 100213d8     libvcruntime:frame.obj
 0002:00007448       __sehtable$___DestructExceptionObject 10021448     libvcruntime:ehhelpers.obj
 0002:00007468       __sehtable$?common_exit@@YAXHW4_crt_exit_cleanup_mode@@W4_crt_exit_return_mode@@@Z 10021468     libucrt:exit.obj
 0002:00007490       __sehtable$??$?RV<lambda_800076c951b434888f4765a74a194fcc>@@AAV<lambda_4e60a939b0d047cfe11ddc22648dfba9>@@V<lambda_6dbb1268764f43b569ce7b67e331d33a>@@@?$__crt_seh_guarded_call@H@@QAEH$$QAV<lambda_800076c951b434888f4765a74a194fcc>@@AAV<lambda_4e60a939b0d047cfe11ddc22648dfba9>@@$$QAV<lambda_6dbb1268764f43b569ce7b67e331d33a>@@@Z 10021490     libucrt:onexit.obj
 0002:000074b0       __sehtable$??$?RV<lambda_995298e7d72eb4c2aab26c0585b3abe5>@@AAV<lambda_275893d493268fdec8709772e3fcec0e>@@V<lambda_293819299cbf9a7022e18b56a874bb5c>@@@?$__crt_seh_guarded_call@H@@QAEH$$QAV<lambda_995298e7d72eb4c2aab26c0585b3abe5>@@AAV<lambda_275893d493268fdec8709772e3fcec0e>@@$$QAV<lambda_293819299cbf9a7022e18b56a874bb5c>@@@Z 100214b0     libucrt:onexit.obj
 0002:000074d0       __sehtable$_terminate      100214d0     libucrt:terminate.obj
 0002:000074f0       __sehtable$??$?RV<lambda_9df27f884b057bc3edfc946cb5b7cf47>@@AAV<lambda_e69574bed617af4e071282c136b37893>@@V<lambda_cc0d902bcbbeb830f749456577db4721>@@@?$__crt_seh_guarded_call@X@@QAEX$$QAV<lambda_9df27f884b057bc3edfc946cb5b7cf47>@@AAV<lambda_e69574bed617af4e071282c136b37893>@@$$QAV<lambda_cc0d902bcbbeb830f749456577db4721>@@@Z 100214f0     libucrt:per_thread_data.obj
 0002:00007510       __sehtable$??$?RV<lambda_3518db117f0e7cdb002338c5d3c47b6c>@@AAV<lambda_b2ea41f6bbb362cd97d94c6828d90b61>@@V<lambda_abdedf541bb04549bc734292b4a045d4>@@@?$__crt_seh_guarded_call@X@@QAEX$$QAV<lambda_3518db117f0e7cdb002338c5d3c47b6c>@@AAV<lambda_b2ea41f6bbb362cd97d94c6828d90b61>@@$$QAV<lambda_abdedf541bb04549bc734292b4a045d4>@@@Z 10021510     libucrt:per_thread_data.obj
 0002:00007530       __sehtable$??$?RV<lambda_51b6e8b1eb166f2a3faf91f424b38130>@@AAV<lambda_6250bd4b2a391816dd638c3bf72b0bcb>@@V<lambda_0b5a4a3e68152e1d9b943535f5f47bed>@@@?$__crt_seh_guarded_call@X@@QAEX$$QAV<lambda_51b6e8b1eb166f2a3faf91f424b38130>@@AAV<lambda_6250bd4b2a391816dd638c3bf72b0bcb>@@$$QAV<lambda_0b5a4a3e68152e1d9b943535f5f47bed>@@@Z 10021530     libucrt:per_thread_data.obj
 0002:00007550       __sehtable$??$?RV<lambda_5b71d36f03204c0beab531769a5b5694>@@AAV<lambda_be2b3da3f62db62e9dad5dc70221a656>@@V<lambda_8f9ce462984622f9bf76b59e2aaaf805>@@@?$__crt_seh_guarded_call@X@@QAEX$$QAV<lambda_5b71d36f03204c0beab531769a5b5694>@@AAV<lambda_be2b3da3f62db62e9dad5dc70221a656>@@$$QAV<lambda_8f9ce462984622f9bf76b59e2aaaf805>@@@Z 10021550     libucrt:per_thread_data.obj
 0002:00007570       __sehtable$___acrt_uninitialize_locale 10021570     libucrt:wsetlocale.obj
 0002:00007590       __sehtable$___acrt_initialize_lowio 10021590     libucrt:ioinit.obj
 0002:000075b0       __sehtable$___acrt_update_thread_multibyte_data 100215b0     libucrt:mbctype.obj
 0002:000075d0       __sehtable$??$?RV<lambda_978dc153c237d78434369da87b74ff60>@@AAV<lambda_ad1ced32f4ac17aa236e5ef05d6b3b7c>@@V<lambda_4a8533e2866a575feecb8298ce776b0d>@@@?$__crt_seh_guarded_call@X@@QAEX$$QAV<lambda_978dc153c237d78434369da87b74ff60>@@AAV<lambda_ad1ced32f4ac17aa236e5ef05d6b3b7c>@@$$QAV<lambda_4a8533e2866a575feecb8298ce776b0d>@@@Z 100215d0     libucrt:mbctype.obj
 0002:000075f0       __sehtable$__query_new_handler 100215f0     libucrt:new_handler.obj
 0002:00007610       __sehtable$_raise          10021610     libucrt:signal.obj
 0002:00007630       __sehtable$??$?RV<lambda_a048d3beccc847880fc8490e18b82769>@@AAV<lambda_ec61778202f4f5fc7e7711acc23c3bca>@@V<lambda_f7496a158712204296dd6628a163878e>@@@?$__crt_seh_guarded_call@P6AXH@Z@@QAEP6AXH@Z$$QAV<lambda_a048d3beccc847880fc8490e18b82769>@@AAV<lambda_ec61778202f4f5fc7e7711acc23c3bca>@@$$QAV<lambda_f7496a158712204296dd6628a163878e>@@@Z 10021630     libucrt:signal.obj
 0002:00007650       __sehtable$___acrt_update_thread_locale_data 10021650     libucrt:locale_refcounting.obj
 0002:00007670       __sehtable$__fcloseall     10021670     libucrt:closeall.obj
 0002:00007690       __sehtable$_common_flush_all 10021690     libucrt:fflush.obj
 0002:000076b8       __sehtable$___acrt_lowio_ensure_fh_exists 100216b8     libucrt:osfinfo.obj
 0002:000076d8       __sehtable$__write         100216d8     libucrt:write.obj
 0002:000076f8       __sehtable$_fclose         100216f8     libucrt:fclose.obj
 0002:00007718       __sehtable$??$?RV<lambda_61cee617f5178ae960314fd4d05640a0>@@AAV<lambda_6978c1fb23f02e42e1d9e99668cc68aa>@@V<lambda_9cd88cf8ad10232537feb2133f08c833>@@@?$__crt_seh_guarded_call@H@@QAEH$$QAV<lambda_61cee617f5178ae960314fd4d05640a0>@@AAV<lambda_6978c1fb23f02e42e1d9e99668cc68aa>@@$$QAV<lambda_9cd88cf8ad10232537feb2133f08c833>@@@Z 10021718     libucrt:commit.obj
 0002:00007738       __sehtable$??$?RV<lambda_123407a5e2ac06da108355a851863b7a>@@AAV<lambda_2fe9b910cf3cbf4a0ab98a02ba45b3ec>@@V<lambda_ae55bdf541ad94d75914d381c370e64d>@@@?$__crt_seh_guarded_call@H@@QAEH$$QAV<lambda_123407a5e2ac06da108355a851863b7a>@@AAV<lambda_2fe9b910cf3cbf4a0ab98a02ba45b3ec>@@$$QAV<lambda_ae55bdf541ad94d75914d381c370e64d>@@@Z 10021738     libucrt:close.obj
 0002:00007758       __sehtable$__IsNonwritableInCurrentImage 10021758     LIBCMT:pesect.obj
 0002:00007780       .edata                     10021780     ConEmuBg.exp
 0002:000077a8       rgpv                       100217a8     ConEmuBg.exp
 0002:000077e4       rgszName                   100217e4     ConEmuBg.exp
 0002:00007820       rgwOrd                     10021820     ConEmuBg.exp
 0002:0000783e       szName                     1002183e     ConEmuBg.exp
 0002:0000784b       $N00001                    1002184b     ConEmuBg.exp
 0002:0000785a       $N00002                    1002185a     ConEmuBg.exp
 0002:00007869       $N00003                    10021869     ConEmuBg.exp
 0002:0000786f       $N00004                    1002186f     ConEmuBg.exp
 0002:00007879       $N00005                    10021879     ConEmuBg.exp
 0002:00007884       $N00006                    10021884     ConEmuBg.exp
 0002:0000788c       $N00007                    1002188c     ConEmuBg.exp
 0002:00007895       $N00008                    10021895     ConEmuBg.exp
 0002:000078a4       $N00009                    100218a4     ConEmuBg.exp
 0002:000078b5       $N00010                    100218b5     ConEmuBg.exp
 0002:000078c7       $N00011                    100218c7     ConEmuBg.exp
 0002:000078d5       $N00012                    100218d5     ConEmuBg.exp
 0002:000078e0       $N00013                    100218e0     ConEmuBg.exp
 0002:000078ec       $N00014                    100218ec     ConEmuBg.exp
 0002:000078fb       $N00015                    100218fb     ConEmuBg.exp
 0002:00007c06       .idata$6                   10021c06     version:VERSION.dll
 0002:00007ee0       .idata$6                   10021ee0     kernel32:KERNEL32.dll
 0002:00007f4c       .idata$6                   10021f4c     user32:USER32.dll
 0002:00008012       .idata$6                   10022012     gdi32:GDI32.dll
 0002:00008072       .idata$6                   10022072     advapi32:ADVAPI32.dll
 0002:000080a2       .idata$6                   100220a2     ole32:ole32.dll
 0003:00000058       ?items@?1??ConfigureProc@@YAHH@Z@4PAUFarDialogItem@@A 10023058     ConEmuBg1900.obj
 0003:00000258       ?items@?1??ConfigureProc@@YAHH@Z@4PAUFarDialogItem@@A 10023258     ConEmuBg2800.obj
 0003:00000458       ?items@?1??ConfigureProc@@YAHH@Z@4PAUFarDialogItem@@A 10023458     ConEmuBg995.obj
 0003:000005b8       ?items@?1??ConfigureProc@@YAHH@Z@4PAUFarDialogItem@@A 100235b8     ConEmuBgA.obj
 0003:00001700       ?__vcrt_flsindex@@3KA      10024700     libvcruntime:per_thread_data.obj
 0003:00001730       _errno_no_memory           10024730     libucrt:errno.obj
 0003:00001734       _doserrno_no_memory        10024734     libucrt:errno.obj
 0003:0000173c       ___acrt_flsindex           1002473c     libucrt:per_thread_data.obj
 0003:000018b0       ___rgctypeflag             100248b0     libucrt:mbctype.obj
 0003:000018b8       ___rgcode_page_info        100248b8     libucrt:mbctype.obj
 0003:00002164       ?gfRegisterBackground@@3P6GHPAURegisterBackgroundArg@@@ZA 10025164     ConEmuBg.obj
 0003:00002170       ?bWasRegistered@?1??StartPlugin@@YAXH@Z@4_NA 10025170     ConEmuBg.obj
 0003:0000217c       ?szMenu@?1??GetPluginInfoW1900@@YAXPAX@Z@4PAPA_WA 1002517c     ConEmuBg1900.obj
 0003:00002180       ?szMenu1@?1??GetPluginInfoW1900@@YAXPAX@Z@4PA_WA 10025180     ConEmuBg1900.obj
 0003:00002380       ?$TSS0@?1??ConfigureProc@@YAHH@Z@4HA 10025380     ConEmuBg1900.obj
 0003:0000238c       ?szMenu@?1??GetPluginInfoW2800@@YAXPAX@Z@4PAPA_WA 1002538c     ConEmuBg2800.obj
 0003:00002390       ?szMenu1@?1??GetPluginInfoW2800@@YAXPAX@Z@4PA_WA 10025390     ConEmuBg2800.obj
 0003:00002590       ?$TSS0@?1??ConfigureProc@@YAHH@Z@4HA 10025590     ConEmuBg2800.obj
 0003:0000259c       ?gszRootKeyW995@@3PA_WA    1002559c     ConEmuBg995.obj
 0003:000025a0       ?szMenu@?1??GetPluginInfoW995@@YAXPAX@Z@4PAPA_WA 100255a0     ConEmuBg995.obj
 0003:000025a8       ?szMenu1@?1??GetPluginInfoW995@@YAXPAX@Z@4PA_WA 100255a8     ConEmuBg995.obj
 0003:000027a8       ?$TSS0@?1??ConfigureProc@@YAHH@Z@4HA 100257a8     ConEmuBg995.obj
 0003:000027b4       ?gszRootKeyA@@3PA_WA       100257b4     ConEmuBgA.obj
 0003:000027b8       ?szMenu@?1??GetPluginInfo@@9@4@4PAPADA 100257b8     ConEmuBgA.obj
 0003:000027c0       ?szMenu1@?1??GetPluginInfo@@9@4@4PADA 100257c0     ConEmuBgA.obj
 0003:000028c0       ?$TSS0@?1??ConfigureProc@@YAHH@Z@4HA 100258c0     ConEmuBgA.obj
 0003:000028d4       ?gh_UnknownTerminatedThread@@3PAXA 100258d4     common-kernel32:WThreads.obj
 0003:000028d8       ?g_Threads@@3PAUConEmuThreadInfo@@A 100258d8     common-kernel32:WThreads.obj
 0003:0000a0d8       _GS_ExceptionRecord        1002d0d8     LIBCMT:gs_report.obj
 0003:0000a128       _GS_ContextRecord          1002d128     LIBCMT:gs_report.obj
 0003:0000a3f4       ?_Tss_mutex@@3U_RTL_CRITICAL_SECTION@@A 1002d3f4     LIBCMT:thread_safe_statics.obj
 0003:0000a40c       ?_Tss_cv@@3U_RTL_CONDITION_VARIABLE@@A 1002d40c     LIBCMT:thread_safe_statics.obj
 0003:0000a410       ?_Tss_event@@3PAXA         1002d410     LIBCMT:thread_safe_statics.obj
 0003:0000a414       ?encoded_sleep_condition_variable_cs@@3P6GHPAU_RTL_CONDITION_VARIABLE@@PAU_RTL_CRITICAL_SECTION@@K@ZA 1002d414     LIBCMT:thread_safe_statics.obj
 0003:0000a418       ?encoded_wake_all_condition_variable@@3P6GXPAU_RTL_CONDITION_VARIABLE@@@ZA 1002d418     LIBCMT:thread_safe_statics.obj
 0003:0000a420       ?__proc_attached@@3HA      1002d420     LIBCMT:dll_dllmain.obj
 0003:0000a424       ?module_local_atexit_table@@3U_onexit_table_t@@A 1002d424     LIBCMT:utility.obj
 0003:0000a430       ?module_local_at_quick_exit_table@@3U_onexit_table_t@@A 1002d430     LIBCMT:utility.obj
 0003:0000a43c       ?module_local_atexit_table_initialized@@3_NA 1002d43c     LIBCMT:utility.obj
 0003:0000a448       ?is_initialized_as_dll@@3_NA 1002d448     LIBCMT:utility.obj
 0003:0000a468       ?__vcrt_startup_thread_ptd@@3U__vcrt_ptd@@A 1002d468     libvcruntime:per_thread_data.obj
 0003:0000a490       ___vcrt_lock_table         1002d490     libvcruntime:locks.obj
 0003:0000a4a8       ___vcrt_locks_initialized  1002d4a8     libvcruntime:locks.obj
 0003:0000a4ac       ?module_handles@@3PAPAUHINSTANCE__@@A 1002d4ac     libvcruntime:winapi_downlevel.obj
 0003:0000a4b8       ?encoded_function_pointers@@3PAPAXA 1002d4b8     libvcruntime:winapi_downlevel.obj
 0003:0000a4f8       ?heap@@3V_HeapManager@@A   1002d4f8     libvcruntime:undname.obj
 0003:0000a510       _c_termination_complete    1002d510     libucrt:exit.obj
 0003:0000a514       _thread_local_exit_callback_func 1002d514     libucrt:exit.obj
 0003:0000a518       ?c_exit_complete@?5??common_exit@@YAXHW4_crt_exit_cleanup_mode@@W4_crt_exit_return_mode@@@Z@4_NA 1002d518     libucrt:exit.obj
 0003:0000a520       ?program_name@?5???$common_configure_argv@D@@YAHW4_crt_argv_mode@@@Z@4PADA 1002d520     libucrt:argv_parsing.obj
 0003:0000a650       ___acrt_invalid_parameter_handler 1002d650     libucrt:invalid_parameter.obj
 0003:0000a664       _enable_percent_n          1002d664     libucrt:printf_count_output.obj
 0003:0000a878       ___acrt_lock_table         1002d878     libucrt:locks.obj
 0003:0000a9b0       ___acrt_locks_initialized  1002d9b0     libucrt:locks.obj
 0003:0000a9b8       _module_handles            1002d9b8     libucrt:winapi_thunks.obj
 0003:0000aa08       _encoded_function_pointers 1002da08     libucrt:winapi_thunks.obj
 0003:0000aa88       ?state_cache@?1??__acrt_is_packaged_app@@9@4JA 1002da88     libucrt:winapi_thunks.obj
 0003:0000aaa4       _fSystemSet                1002daa4     libucrt:mbctype.obj
 0003:0000aaa8       ?initialized@?1??__acrt_initialize_multibyte@@9@4_NA 1002daa8     libucrt:mbctype.obj
 0003:0000aac8       ___acrt_new_handler        1002dac8     libucrt:new_handler.obj
 0003:0000aacc       _ctrlc_action              1002dacc     libucrt:signal.obj
 0003:0000aad0       _ctrlbreak_action          1002dad0     libucrt:signal.obj
 0003:0000aad4       _abort_action              1002dad4     libucrt:signal.obj
 0003:0000aad8       _term_action               1002dad8     libucrt:signal.obj
 0003:0000aadc       _user_matherr              1002dadc     libucrt:matherr.obj
 0003:0000aae8       ___acrt_global_new_mode    1002dae8     libucrt:new_mode.obj
 0003:0000aaec       ___acrt_app_type           1002daec     libucrt:report_runtime_error.obj
 0003:0000aaf4       __pmatherr_set             1002daf4     libucrt:libm_error.obj
 0004:000000a0       $R000000                   1002e0a0     ConEmuBg.res
 0004:000003b8       $R000318                   1002e3b8     ConEmuBg.res
